:100000000C946B090C948A090C948A090C941C0AB0
:100010000C94520A0C948A090C948A090C948A094B
:100020000C948A090C948A090C948A090C948A0904
:100030000C948A090C948A090C948A090C947D0DFD
:100040000C948A090C948A090C948A090C948A09E4
:100050000C942A6E0C94DD650C948A090C948A0920
:100060000C948A090C94B2660C948A090C94A666C6
:100070000C948A090C948A090C948A090C948A09B4
:100080000C945D790C948A090C948A090C948A0961
:100090000C94F0660C948A090C94E4660C948A091A
:1000A0000C948A090C948A090C948A090C948A0984
:1000B0000C948A090C948A090C948A090C948A0974
:1000C0000C948A090C948A090C948A090C948A0964
:1000D0000C948A090C948A090C948A090C948A0954
:1000E0000C948A090C94E36D0C94ED6D0C94D96D0D
:1000F0000C94996D0C941E6E0C940F6E0C94036E00
:100100000C94F76D0C948A090C948A090C948A0952
:100110000C948A090C948A090C948A090C948A0913
:100120009482B382328321844184618469841684F9
:10013000084AD73B3BCE016E84BCBFFDC12F3D6C4E
:1001400074319ABD56833DDA3D00C77F11BED9E4B4
:10015000BB4C3E916BAAAABE000000803F076342E1
:1001600036B79BD8A71A39685618AEBAAB558C1D4E
:100170003CB7CC5763BD6DEDFD753EF6177231BFD0
:10018000000000803F08000000BE922449123EABF0
:10019000AAAA2ABECDCCCC4C3E00000080BEABAAA1
:1001A000AAAA3E00000000BF000000803F0000003F
:1001B0000000084178D3BB4387D1133D190E3CC3DF
:1001C000BD4282AD2B3E68EC8276BED98FE1A93E5E
:1001D0004C80EFFFBE01C4FF7F3F00000000000025
:1001E00025730A005854414C5F5452494D3D2564D3
:1001F0000025730A0025730A0054657374203620A5
:1002000025730A005465737420352025730A005441
:1002100065737420342025730A0054657374203389
:100220002025730A005465737420322025730A0058
:100230005465737420312025730A006368616E3D34
:1002400025640A0074787077723D25640A003530A1
:10025000306B0A003235306B0A003131356B0A00E1
:1002600035366B0A0033386B0A0025730A00765F57
:100270006C6F773D252D332E32660A0025730A00F8
:1002800073656E743D252D75206475703D252D7543
:100290002069676E6F7265643D252D752074746CDE
:1002A0005F7A65726F3D252D750A0025372E3366FE
:1002B0002025372E33660025352E32662000457204
:1002C000726F72203020566F6C74004E6F74207302
:1002D0007570706F727465640A004572726F722077
:1002E0003020566F6C74004572726F722030205649
:1002F0006F6C74007062323D25730A00256C7500C6
:10030000416C6C6F77656420737065656420312F74
:1003100031302F3130302F343030206B6269742F00
:10032000730025630074746C3D252D642000747483
:100330006C3D252D6420004E65772074746C3D253E
:100340002D6420002563004D533536313120503D5A
:10035000252D372E326620252D372E32666D0A0068
:10036000424D5030383520256C64205061202025C6
:100370002D372E32666D00256300545F4845415489
:100380005F4944583D252D352E32662000545F4488
:1003900045573D252D352E3266200041483D252DFF
:1003A000352E32662000545F53485432583D252D77
:1003B000352E3266200052485F53485432583D254E
:1003C0002D352E32662000545F52483D252D342EA7
:1003D0003166200052483D252D342E3166200025FF
:1003E00063002563002563002563002563007265B3
:1003F000706F72745F616C6C3D007265706F7274C7
:100400003D00256300256300256300256300204F20
:10041000534343414C3D2564200020467573653AA3
:100420002065653D253032782068663D253032787C
:10043000206C663D25303278206C623D2530327864
:10044000004D43553D2530366C78002563007478A7
:100450005F6C656E3D252D6C752C765F6C6F773DFE
:10046000252D6C752C73687432783D252D6C750ABA
:10047000002563004F4B0A002563002563002563B8
:1004800000256300256300256300256300256300C4
:1004900064656275675F616C6C3D00646562756779
:1004A0003D0064656275673D0025730A00646565FB
:1004B000700A006E6F6E650A00707772733D00708F
:1004C00062323D25730A007062313D25730A00696E
:1004D0006E74725F7365635F70313D252D372E3307
:1004E000660A00696E74725F70313D252D6C640A76
:1004F00000696E74725F7365635F70303D252D37E0
:100500002E33660A00696E74725F70303D252D6C63
:10051000640A00765F6D63753D252D352E32660ABF
:1005200000745F6D63753D252D352E32660A0070AF
:100530007077723D25730A0064656275673D0072CD
:10054000636D643D25730A0025730A006175746F3D
:100550000A006C6F675F6D6F64653D007573625F65
:100560007077723D25730A0072656C61793D257361
:100570000A0074746C3D252D640A0052494D455F94
:10058000616464723D252D642E252D640A006E651C
:10059000696768626F725F7461626C655F73697AC4
:1005A000653D25640A00765F6C6F773D252D332EFF
:1005B00032660A00747870773D25640A00636861CA
:1005C0006E3D25640A0069643D006932635F6275AF
:1005D000733D006932635F73706565643D252D6C02
:1005E000750A007478743D25730A00537973746535
:1005F0006D2053756D6D6172790A002530366C7807
:100600000041744D656761323536524652320041C1
:10061000744D656761313238524652320041744D33
:100620006567613634524652320041744D656761E8
:1006300031323852464131004D43553D006D6173B2
:100640006B3D002C00696E74657276616C3D252DE2
:10065000750023252D642C00745F686561745F69E3
:10066000647800745F64657700616800705F6D7323
:10067000353631310072685F736874327800745FA8
:1006800073687432780070610070006164340061D6
:1006900064330061643200616431006133006132AF
:1006A00000613100765F696E0072680065727200E9
:1006B000757074696D650070315F6C7374007031B2
:1006C0005F740070310070305F6C73740070305F65
:1006D0007400703000765F6D637500745F6D6375D4
:1006E00000743100740069640065363400747874F5
:1006F000002D002B006175746F006E6F6E650070C9
:100700006F7765725F736176655F6C65647279009F
:1007100072656C61795F6C65647900636F6D70619F
:10072000737300616363656C007072657300705F62
:10073000707772006165730070315F6C6564790079
:1007400070305F6C656472006576656E74006C6510
:1007500064006F7700706B740074785F6C65647907
:100760000072785F6C656472006F706572006E6F06
:100770006E65002530327800765F6164343D252D4A
:10078000382E3666002000765F6164333D252D38B3
:100790002E3666002000765F6164323D252D382EAE
:1007A0003666002000765F6164313D252D382E3697
:1007B00066002000765F6C696768743D252D382ED1
:1007C0003666002000765F61323D252D372E336678
:1007D000002000765F61313D252D372E33660020E5
:1007E00000765F696E3D252D352E326600204E6500
:1007F0007665722D7573656420737461636B203E3A
:100800002025642062797465730A00757074696DBF
:10081000653D252D642D646179732D253032643A50
:10082000253032643A253032642D686F7572730A50
:100830000074657374205B6F66667C317C327C3338
:100840007C347C355D20202020202020202D207429
:10085000657374206D6F6465730A0D007478205B96
:10086000706B74207061796C6F61645D2020202052
:1008700020202020202020202D2073656E642072EF
:100880006164696F20706B74206B6579626F61724F
:10089000640A0D00776474205B6F6E7C6F66667C03
:1008A000746573745D2020202020202020202020CB
:1008B0002D207761746368646F670A0D00765F6C42
:1008C0006F77205B765F6C6F775D20202020202083
:1008D0002020202020202020202D206C6F77657381
:1008E00074207265706F727420766F6C74616765C6
:1008F0000A0D007570677220202020202020202003
:100900002020202020202020202020202020202DDA
:10091000207265626F6F742076696120626F6F74F8
:100920006C6F616465720A0D0075617274205B33CF
:10093000386B7C35366B7C3131356B7C3235306BC6
:100940007C3530306B5D202D2073657420746572AA
:100950006D2F756172742073706565640A0D006295
:100960006F6F742020202020202020202020202095
:1009700020202020202020202020202D2072656291
:100980006F6F740A0D0070777273205B6465657019
:100990007C6E6F6E655D202020202020202020208E
:1009A00020202D206D637520736C656570206D6F40
:1009B00064650A0D007265737420656570726F6DF1
:1009C0002020202020202020202020202020202027
:1009D000202D20726573746F726520656570726F6B
:1009E0006D0A0D0070707772205B6F6E7C6F6666AB
:1009F0005D202020202020202020202020202020BA
:100A00002D2070726F6772616D6D61626C65207010
:100A100077720A0D0070623220205B6F6E7C6F6609
:100A2000665D202020202020202020202020202043
:100A3000202D2070726F6772616D6D61626C652030
:100A400070696E2062320A0D00747874205B7374D2
:100A500072696E675D202020202020202020202029
:100A600020202020202D20536574207265706F7225
:100A700074207465787420737472696E670A0D004F
:100A800074787077205B31352D305D202020202058
:100A90002020202020202020202020202D205458DD
:100AA000205077722E204869676865737420302063
:100AB000283364426D290A0D0074746C205B302D5C
:100AC00031355D20202020202020202020202020C3
:100AD00020202020202D2074696D652D746F2D6CD1
:100AE00069766520666F72207061636B6574730A46
:100AF0000D00737320202020202020202020202083
:100B000020202020202020202020202020202D20D8
:100B100073797374656D2073756D6D6172790A0DEB
:100B20000072732020202020202020202020202040
:100B3000202020202020202020202020202D207256
:100B40006164696F2073746174730A0D00726920A7
:100B50005B236E5D205B696E745D20202020202069
:100B60002020202020202020202D207265706F72F0
:100B70007420696E74657276616C0A0D0072636D23
:100B800064205B6F6E7C6F66665D202020202020D5
:100B90002020202020202020202D20616C6C6F77C9
:100BA00020636D642066726F6D206E65746F726B6A
:100BB0000A0D007265205B236E5D205B2B7C2D5D32
:100BC000205B6D61736B7C6175746F2C6D61736BF1
:100BD0005D202D206D6F7465207265706F727420BA
:100BE0007365742F6D6F646966790A0D006F7720E5
:100BF00020202020202020202020202020202020F5
:100C00002020202020202020202D206F6E652D7791
:100C10006972652073656E736F72730A0D006C6F75
:100C200067205B6175746F7C6F6E7C6F66665D209C
:100C3000202020202020202020202D206D6F746572
:100C4000732064617461206F6E205553420A0D0059
:100C50006E65205B666C7573685D20202020202007
:100C60002020202020202020202020202D206E65E4
:100C7000696768626F72207461626C650A0D006555
:100C800072722020202020202020202020202020C0
:100C900020202020202020202020202D206572725E
:100CA0006F722073746174730A0D006D6375202078
:100CB0002020202020202020202020202020202034
:100CC000202020202020202D206D637520696E6655
:100CD0006F0A0D00693263205B70726F62657C730E
:100CE0007065656420236E5D202020202020202058
:100CF0002D206932632070726F6265206275737C8B
:100D0000736574206275732073706565640A0D00E5
:100D10006964205B72657365745D2020202020204B
:100D20002020202020202020202020202D20696429
:100D30002068616E646C696E670A0D0068756D20CD
:100D400020202020202020202020202020202020A3
:100D500020202020202020202D2068756D696469C6
:100D600074792073656E736F720A0D0072656C6121
:100D700079205B6F6E7C6F66667C73746174735DE3
:100D800020202020202020202D2072656C617920D9
:100D90006E6574776F726B207265706F7274730A10
:100DA0000D006465205B6D61736B5D202020202049
:100DB00020202020202020202020202020202D2026
:100DC00064656275670A0D006368616E205B31318E
:100DD0002D32365D202020202020202020202020A1
:100DE000202020202D206368616E2031312D323685
:100DF0002028322E3430352D32343830204D687A68
:100E0000290A0D0063616C69205B5B765F696E7C0B
:100E100061317C61325D20766F6C747C72657365C4
:100E2000747C6E6F6E655D202D2063616C696272EB
:100E30006174650A0D006164632020202020202059
:100E400020202020202020202020202020202020A2
:100E500020202D2073686F7720765F696E2C2061CB
:100E6000312C20613220766F6C74616765730A0DD6
:100E7000007520202020202020202020202020203D
:100E8000202020202020202020202020202D207500
:100E90007074696D650A0D007620202020202020C6
:100EA0002020202020202020202020202020202042
:100EB000202020202D2076657273696F6E0A0D0048
:100EC00068202020202020202020202020202020DA
:100ED0002020202020202020202020202D20686578
:100EE0006C700A0D00256300756E6B6E6F776E2057
:100EF000636D640A00484D4335383833002573006C
:100F0000257300202573002025362E32662000250B
:100F10003032780074656D705F65787465726E3D0F
:100F2000252D362E326600202573002025362E32E0
:100F300066204F6E2D426F6172640025303278005A
:100F400074656D705F626F6172643D252D362E325F
:100F500066000A00503A20256C642050612020254C
:100F60002D372E3266206D0A002563002563004967
:100F700032433A2000452025642E256420636C6F9F
:100F8000636B20256C752063707520256C75206C53
:100F9000706D20256C752069727120256C75206735
:100FA0006C656420256C7520796C656420256C75F2
:100FB00020726C656420256C7520747820256C7512
:100FC000206C697374656E20256C752073656E7373
:100FD0006F727320256C752073657269616C2025B2
:100FE0006C750A00532025642E256420636C6F63A2
:100FF0006B20256C7520747820256C752072782004
:10100000256C752072747820256C7520727278209A
:10101000256C75207265786D697420256C7520616A
:10102000636B747820256C75206E6F61636B7478C8
:1010300020256C752061636B727820256C75207497
:10104000696D65646F757420256C752062616461DB
:10105000636B727820256C7520746F6F6C6F6E6790
:1010600020256C7520746F6F73686F727420256C07
:10107000752062616473796E636820256C752062E7
:10108000616463726320256C7520636F6E74656E96
:1010900074696F6E64726F7020256C752073656E55
:1010A00064696E6764726F7020256C75206C6C7457
:1010B0007820256C75206C6C727820256C750A0080
:1010C000257325730A004F6E6C696E650A000A006D
:1010D0002C20636865636B20726174652025752020
:1010E000487A0025732025732C206368616E6E6535
:1010F0006C20257520706F776572202575000A00B9
:1011000025783A004D414320616464726573732011
:101110000052616E646F6D2045554936342061641C
:1011200064726573732067656E6572617465640AC5
:10113000000A2A2A2A2A2A2A2A426F6F74696E67AD
:101140002025732A2A2A2A2A2A2A0A00454550528B
:101150004F4D20697320636F72727570742C20720A
:101160006577726974696E67207769746820646551
:101170006661756C74732E0A006C6F63616C686FC6
:1011800073740041544D45474131323872666131C4
:1011900000020000FFFE0000016E616E00696E66D5
:1011A0000000407A10F35A00A0724E18090010A5F2
:1011B000D4E80000E87648170000E40B5402000071
:1011C000CA9A3B000000E1F50500008096980000F7
:1011D0000040420F000000A0860100000010270020
:1011E000000000E803000000006400000000000AA6
:1011F00000000000000100000000002C76D888DC10
:10120000674F0823DFC1DFAE59E1B1B796E5E3E4EC
:1012100053C63AE651997696E8E6C28426EB898C65
:101220009B62ED407C6FFCEFBC9C9F40F2BAA56FC7
:10123000A5F490055A2AF75C936B6CF9676DC11B96
:10124000FCE0E40D47FEF520E6B500D0ED902E035E
:1012500000943577050080841E080000204E0A00A7
:101260000000C80C333333330F986E12831141EFF3
:101270008D2114893BE65516CFFEE6DB18D1844B51
:10128000381BF77C1D901DA4BBE424203284725EC1
:10129000228100C9F124ECA1E53D274E414E494E83
:1012A000495459494E46CDCCCC3D0AD7233C17B7BB
:1012B000D13877CC2B329595E6241FB14F0A000028
:1012C00020410000C84200401C4620BCBE4CCA1B46
:1012D0000E5AAEC59D7411241FBECFEFD1E4DEBF00
:1012E000CDBF19E0A0E0B2E0E0EAFEE201E00BBF12
:1012F00002C007900D92AE3BB107D9F721E3AEEBE8
:10130000B9E001C01D92A33DB207E1F70E94388504
:101310000C944E970C9400008115910511F00197E3
:10132000F1F7089589EB94E09F938F930E94339493
:101330008091580290915902A0915A02B0915B029B
:101340000F900F9093FF03C083EB94E002C08DEAEF
:1013500094E09F938F930E9433940F900F90089581
:10136000E091771BEF73F0E0E853F44E80838091B7
:10137000771B8F5F8093771B80910D298860809306
:101380000D294EE352E061E1CA010E94BD5580E0A3
:1013900090E00895CF93DF93EC018091C50990917F
:1013A000C60986FF1DC08E811F928F938D811F926B
:1013B0008F938C811F928F938B811F928F938A8141
:1013C0001F928F9385E693E09F938F930E942194C1
:1013D0008DB79EB70C960FB6F8949EBF0FBE8DBF0B
:1013E000BE018CEF99E00E94EF56BE0184E092E0CE
:1013F000DF91CF910C9464568823B9F052985A9893
:101400001DBA80916900806280936900EA9A5398BE
:101410005B98EB9A80916900806880936900809165
:1014200068008160809368000895109269005A9A5C
:10143000EA985B9AEB9808951F920F920FB60F925D
:1014400011248F939F93AF93BF938091680080FF87
:1014500020C08091E8289091E928A091EA28B091D5
:10146000EB280196A11DB11D8093E8289093E928EF
:10147000A093EA28B093EB288091C5099091C60902
:1014800087FF07C0749882E090E090938502809374
:101490008402BF91AF919F918F910F900FBE0F90DB
:1014A0001F9018951F920F920FB60F9211248F93D1
:1014B0009F93AF93BF938091680080FF20C080917D
:1014C000EC289091ED28A091EE28B091EF2801969C
:1014D000A11DB11D8093EC289093ED28A093EE28D8
:1014E000B093EF288091C5099091C60990FF07C07D
:1014F000739882E090E09093850280938402BF917C
:10150000AF919F918F910F900FBE0F901F901895E4
:1015100080937C0080917B00877F80937B0080910B
:101520007C00806C80937C0085E080937A008091C1
:101530007A00806880937A0080917B0087FFFCCFDF
:1015400080917B0085FFFCCF80917A00806480933E
:101550007A0080917A0086FDFCCF1092790010927B
:10156000780084E090E060E070E020917A002064F0
:1015700020937A0020917A0026FDFCCF20917800FC
:1015800030917900620F731F0197009771F71092E5
:101590007C0080917A008F7780937A0076956795AA
:1015A0007695679580E090E00E948E8A089580E0AD
:1015B0000E94880A20917C0230917D0240917E0237
:1015C00050917F020E94728C21EE3AE744E95EE37B
:1015D0000E94278908950F931F93CF93DF93CFE144
:1015E000D0E00BE51EE0C093510187EC90E00E9433
:1015F0008C098091510185FD0DC0C031D10521F0CC
:101600002CF00B54110904C004EC19E00253110929
:101610002197E9CFB80180E090E00E948E8A20E017
:1016200030E04AE754E40E94F189DF91CF911F91A5
:101630000F910895CF93DF93EC01888199810097F2
:1016400099F08B3B904121F01982188283E011C000
:10165000623171F40E94EB0A60933F24709340243E
:1016600080934124909342248BEB90E1998388836B
:1016700081E0DF91CF91089580917B008860809315
:101680007B0089EC80937C0085E080937A008091D8
:101690007A00806880937A0080917B0087FFFCCF7E
:1016A00080917B0085FFFCCF80917A0080648093DD
:1016B0007A0080917A0086FDFCCF80917A00806468
:1016C00080937A0080917A0086FDFCCF609178004B
:1016D0007091790080917A008F7780937A0080E012
:1016E00090E00E948E8A27ED33EA40E95FE30E9492
:1016F000728C26E636E648E853E40E94268908956F
:10170000BF92CF92DF92EF92FF920F931F93CF93EE
:10171000DF93CDB7DEB729970FB6F894DEBF0FBEC3
:10172000CDBF6C011092BE098FEF898708E81BE1DD
:10173000B12C7E0189E0E80EF11C89858823E9F14E
:10174000E8E0BE16E1F1BE016F5F7F4FC7010E9466
:10175000585F89858F3F11F08E3F19F48093BE0941
:101760002CC0CE010196C114D10471F40E94715FA6
:1017700080930A29FE013196A2E0B9E281918D930E
:10178000EE15FF05D9F71DC00E94715FF801808337
:10179000FE01319620E030E0A801485051098191C6
:1017A000DA01A20FB31F8C932F5F3F4F2830310512
:1017B000B1F7B394075F1F4FC0CF8B2D03C088E0F4
:1017C00001C081E029960FB6F894DEBF0FBECDBFF1
:1017D000DF91CF911F910F91FF90EF90DF90CF900D
:1017E000BF90089582E59FE09F938F930E9433946A
:1017F0000F900F9008952F923F924F925F926F92A9
:101800007F928F929F92AF92BF92CF92DF92EF9290
:10181000FF920F931F93CF93DF93EC014B0100973F
:1018200011F427E004C08130910549F426E04AE232
:1018300050E06BE270E089E290E00E94385ECE01F9
:101840000E94800B9E012154364F5901D9018C937F
:10185000CD2B69F098E8C92E9BE1D92EC0E8DBE1D9
:10186000E12CF12C23E0222E2FE0322EA6C082E0C4
:1018700099E20E94A660BC01882777FD8095982F89
:101880000E94908A6B017C01892869F020E030E099
:1018900048EC52E40E94F1899F938F937F936F935A
:1018A00080E49FE0ACC0C2E0D9E20BE31FE0899185
:1018B0001F928F931F930F930E9433940F900F905A
:1018C0000F900F90B9E2CA30DB0789F720E030E0D3
:1018D00048EC52E4C701B6010E94F1899F938F93AF
:1018E0007F936F938BE29FE09F938F930E9433943B
:1018F0000F900F900F900F900F900F9080910A29EA
:10190000882319F084E993E002C088E094E09F9373
:101910008F9387E29FE09F938F930E9433940F9061
:101920000F900F900F9075C000E010E0FE01E00FE7
:10193000F11F80811F928F93AFE0BFE0BF93AF9301
:101940000E9433940F5F1F4F0F900F900F900F90D6
:101950000830110559F720E030E048EC52E4C301AB
:10196000B2010E94F1899F938F937F936F93A7E0B9
:10197000BFE0BF93AF930E9433940F900F900F90EE
:101980000F900F900F90D6018C91882309F455C0C9
:1019900084E993E09F938F933F922F920E94339418
:1019A0000E94F20BBFEFEB1AFB0AE9E0CE0ED11C4E
:1019B00029960F900F900F900F90D5018C9190E089
:1019C000E816F906ECF5CE010E94A660BC01882756
:1019D00077FD8095982F0E94908A2B013C018114FD
:1019E000910409F4A1CF20E030E048EC52E40E94D9
:1019F000F1899F938F937F936F9384E19FE09F93EF
:101A00008F930E9433940F900F900F900F900F9030
:101A10000F90DF91CF911F910F91FF90EF90DF908A
:101A2000CF90BF90AF909F908F907F906F905F907E
:101A30004F903F902F900C94F20B88E094E0AACF47
:101A4000DF91CF911F910F91FF90EF90DF90CF909A
:101A5000BF90AF909F908F907F906F905F904F90CE
:101A60003F902F900895CF93DF9300D0CDB7DEB78E
:101A7000809103298983809109298A83CE01019667
:101A80000E94B1530F900F90DF91CF910895CF93A3
:101A9000DF93EC0120910229309103294091042920
:101AA0005091052960910629709107298091082994
:101AB00090910929AFEF0E94A28FE1F427E04AE25A
:101AC00050E06BE270E089E290E00E94385E80E0D6
:101AD00090E00E94800BC154D64F888349E050E0CB
:101AE0006AE070E082E099E20E94A595DF91CF91D3
:101AF0000C94330DDF91CF9108951F920F920FB682
:101B00000F9211240BB60F92FF920F931F932F93F6
:101B10003F934F935F936F937F938F939F93AF9375
:101B2000BF93CF93DF93EF93FF9380910D29826052
:101B300080930D298091580286FD2B9A809158023E
:101B400087FD2B9A809184029091850218161906C0
:101B500014F4749A739A8091C5099091C60985FF0F
:101B600002C07498739880910202909103020197C9
:101B70009093030280930202892B09F042C1809165
:101B8000D3099091D40901969093D4098093D309F5
:101B90008091432490914424A0914524B0914624FF
:101BA0000196A11DB11D8093432490934424A093DA
:101BB0004524B093462480E190E090930302809303
:101BC00002028091580280FD02C01D9B05C0109248
:101BD000C3091092C20906C081E090E09093C30946
:101BE0008093C2098091C5099091C60997FF08C0EA
:101BF0008091C2099091C309892B49F0749A739816
:101C0000C7E2DBE104E514E2FF24F3941EC0739AFB
:101C10007498F6CF8091D3099091D40901960E94CF
:101C2000428D892BC1F0688579856115710569F54B
:101C30006885798561157105D9F52A960B5F1F4F67
:101C4000FBE1CF34DF0709F449C068857985611568
:101C5000710549F3DFCF4A81417020E030E050E068
:101C600060E070E080E090E0A0E00E94A28FD9F2F6
:101C700077988091C5099091C60992FFD4CF749846
:101C80001092850210928402CECF8091D309909158
:101C9000D40901960E94428D892B51F6F8011482D5
:101CA0001382A80162E186E192E00E94BD55C0CF97
:101CB0008091D3099091D4090E94428D892B09F01B
:101CC000BCCFF801F082D283C18314821382A801B1
:101CD00062E184E392E00E94BD55AFCF60915E0265
:101CE00070915F0261157105A1F18091D309909106
:101CF000D4090E94428D892B61F58091E82890914A
:101D0000E928A091EA28B091EB284091351C509128
:101D1000361C6091371C7091381C841B950BA60BE8
:101D2000B70B80934F1B9093501BA093511BB09304
:101D3000521B8091E8289091E928A091EA28B0915F
:101D4000EB288093351C9093361CA093371CB093DE
:101D5000381C60915C0270915D0261157105A1F102
:101D60008091D3099091D4090E94428D892B61F50D
:101D70008091EC289091ED28A091EE28B091EF2869
:101D80004091391C50913A1C60913B1C70913C1C55
:101D9000841B950BA60BB70B8093531B9093541B7E
:101DA000A093551BB093561B8091EC289091ED2881
:101DB000A091EE28B091EF288093391C90933A1CA3
:101DC000A0933B1CB0933C1C8091580286FD2B983D
:101DD0008091580290915902A0915A02B0915B02F1
:101DE00091FF0FC00E94576A8A3119F0C1E0C80FF5
:101DF00001C0CBE00E9413698C2F0E946F6A0E9481
:101E00005B6940E050E060E086E892E00E94BD55EA
:101E1000FF91EF91DF91CF91BF91AF919F918F9102
:101E20007F916F915F914F913F912F911F910F91F2
:101E3000FF900F900BBE0F900FBE0F901F90189544
:101E40008091771B90915324891B08950E94200F45
:101E5000882371F0E0915324EF73F0E0E853F44EDF
:101E6000808190E0209153242F5F20935324089584
:101E70008FEF9FEF0895CF93DF93EC011092F0095D
:101E80001092EF09888199810097B1F088389340CA
:101E900021F01982188283E0B6C0613109F0B2C026
:101EA0000E94260F99279093EB098093EA098D30C1
:101EB00009F443C08F3F49F40E94200F8111F0CFF5
:101EC00088E893E0998388839DC08231910509F465
:101ED0005AC08F37910509F052C08091E80990915E
:101EE000E909181619060CF56091CD317091CE31C3
:101EF00088E090E00E94EF936091CD317091CE31F7
:101F000080E290E00E94EF936091CD317091CE31EC
:101F100088E090E00E94EF938091E8099091E909B0
:101F200001979093E9098093E8098091E8099091DD
:101F3000E9098F37910509F0BFCF10925324109211
:101F4000771B8091E8099091E909FC01E859FB4D64
:101F500010829093F0098093EF091092E909109292
:101F6000E80980910B2990910C29009709F4A4CFDE
:101F700040E050E06091FE110E94BD559DCF883039
:101F8000910571F5AACF6091CD317091CE318DE080
:101F900090E00E94EF931092E7091092E609809179
:101FA000E6099091E7092091E8093091E909821743
:101FB00093070CF0BACFFC01E859FB4D808160918A
:101FC000CD317091CE3190E00E94EF938091E6097F
:101FD0009091E70901969093E7098093E609DFCF96
:101FE0006091CD317091CE310E94EF938091E809DC
:101FF0009091E9092091EA09FC01E859FB4D208301
:1020000001968FCF81E0DF91CF9108958091C20931
:102010009091C309892BD1F0809158029091590277
:10202000A0915A02B0915B0293FD10C00E94136907
:1020300083B7817F866083BFF89483B7816083BF55
:102040007894889583B78E7F83BF78940895CF93D3
:10205000DF93EC0188819981009719F08E3E9041C1
:1020600099F40E94D0670E94061040E050E065E8B5
:1020700080910212909103120E94BD558EEE90E164
:102080009983888381E003C01982188283E0DF91FD
:10209000CF910895CF93DF9300D0CDB7DEB7892BD2
:1020A00081F05F934F9380E09FE09F938F936983CC
:1020B0007A830E9433940F900F900F900F907A8143
:1020C00069817F936F938DEF9EE09F938F930E9422
:1020D00033940F900F900F900F900F900F90DF910F
:1020E000CF910895FF920F931F93CF93DF930E9498
:1020F000D06780EB0E94336181111CC00E94976100
:1021000080913D2090913E20816090933E2080936D
:102110003D208DE993E09F938F938DEF9EE09F93F9
:102120008F930E9433940F900F900F900F90C1E007
:10213000D0E002C0C0E0D0E0FEB08F2D8470F82E59
:10214000729A0E94D0678EE40E943361811116C09A
:102150000E94976180913D2090913E2082609093F3
:102160003E2080933D208E010F5F1F4F43E259E0D8
:1021700065EA73E0CE010E944A10E801F11001C047
:1021800072980E94D0678EEE0E943361811116C052
:102190000E94976180913D2090913E2084609093B1
:1021A0003E2080933D208E010F5F1F4F43E259E098
:1021B0006DEA73E0CE010E944A10E8010E94D067E8
:1021C00086EA0E943361811116C00E949761809156
:1021D0003D2090913E20886090933E2080933D204A
:1021E0008E010F5F1F4F43E259E064EB73E0CE01B5
:1021F0000E944A10E8010E94D0678CE30E9433617C
:1022000081111EC00E94976180913D2090913E20D7
:10221000806190933E2080933D208E010F5F1F4F81
:1022200043E259E06CEB73E0CE010E944A1085EF67
:102230009EE09F938F930E9433940F900F90E8013C
:102240000E94D06782ED0E943361811116C00E9406
:10225000976180913D2090913E20806290933E2036
:1022600080933D208E010F5F1F4F43E259E064ECE5
:1022700073E0CE010E944A10E8010E94D06780E816
:102280000E943361811116C00E94976180913D20A8
:1022900090913E20916090933E2080933D208E014E
:1022A0000F5F1F4F43E259E06DEC73E0CE010E94D7
:1022B0004A10E8010E94D06780ED0E9433618111CD
:1022C00016C00E94976180913D2090913E208068C9
:1022D00090933E2080933D208E010F5F1F4F43E27D
:1022E00059E063ED73E0CE010E944A10E8010E94BC
:1022F000D0678CEE0E943361811116C00E949761F5
:1023000080913D2090913E20926090933E2080935A
:102310003D208E010F5F1F4F43E259E06BED73E0EC
:10232000CE010E944A10E80107E010E00E94D06749
:102330008CE70E943361811113C00E9497618091E4
:102340003D2090913E20806490933E2080933D20DC
:1023500043E259E062EE73E0CE010E944A1005C0EC
:10236000015011090115110509F70E949761DF91CC
:10237000CF911F910F91FF900C94F20BCF93DF93AD
:1023800000D0CDB7DEB74A8369830E946E61698150
:10239000862F0E949F614A81842F0E949F610F9027
:1023A0000F90DF91CF910C949761AF92BF92DF9223
:1023B000EF92FF920F931F93CF93DF9300D01F9262
:1023C000CDB7DEB7182FD22E4A835B8369830E9474
:1023D0006E616981862F0E949F61812F81600E94BA
:1023E00095614A81A42E5B81B52E00E010E0ED2CB2
:1023F000F12C81E0E81AF1080D1580F40E151F0587
:1024000019F40E94BA6102C00E94B061F501808394
:102410000F5F1F4FFFEFAF1ABF0AEECF0F900F9065
:102420000F90DF91CF911F910F91FF90EF90DF9070
:10243000BF90AF900C949761AF92BF92CF92DF9212
:10244000EF92FF920F931F93CF93DF93CDB7DEB739
:1024500060970FB6F894DEBF0FBECDBFB82EA42E86
:102460006623E9F18E010F5F1F4F80E1F8011192A1
:102470008A95E9F728E0A80168E980EB0E94D51168
:10248000BB2041F02BEE33E03F932F930E94219429
:102490000F900F906E01F8E0CF0ED11C42EFE42EAA
:1024A00043E0F42EF80181918F011F928F93FF92E8
:1024B000EF920E9421940F900F900F900F900C15A7
:1024C0001D0581F788851F928F9327E434E03F93A1
:1024D0002F930E9421940F900F900F900F90AA209D
:1024E000E9F18E010F5F1F4F80E1F80111928A958B
:1024F000E9F728E0A80160E880EB0E94D511BB2035
:1025000041F087EF93E09F938F930E9421940F9067
:102510000F906E01F0E1CF0ED11C32EFE32E33E0CD
:10252000F32EF80181918F011F928F93FF92EF920A
:102530000E9421940F900F900F900F900C151D0585
:1025400081F788851F928F9387E494E09F938F9300
:102550000E9421940F900F900F900F9060960FB6ED
:10256000F894DEBF0FBECDBFDF91CF911F910F91C9
:10257000FF90EF90DF90CF90BF90AF900895CF93F2
:10258000DF9300D0CDB7DEB71A82198222E0AE0108
:102590004F5F5F4F6AEA8EEE0E94D511898190E00D
:1025A000982F88272A81822B9093091C8093081CDE
:1025B00022E0AE014F5F5F4F6CEA8EEE0E94D511B4
:1025C000898190E0982F88272A81822B90930B1C79
:1025D00080930A1C22E0AE014F5F5F4F6EEA8EEEE1
:1025E0000E94D511898190E0982F88272A81822B1B
:1025F00090930D1C80930C1C22E0AE014F5F5F4F47
:1026000060EB8EEE0E94D511898190E0982F88278B
:102610002A81822B90931B1C80931A1C22E0AE010E
:102620004F5F5F4F62EB8EEE0E94D511898190E083
:10263000982F88272A81822B90931D1C80931C1C25
:1026400022E0AE014F5F5F4F64EB8EEE0E94D5112A
:10265000898190E0982F88272A81822B90931F1CD4
:1026600080931E1C22E0AE014F5F5F4F66EB8EEE43
:102670000E94D511898190E0982F88272A81822B8A
:1026800090930F1C80930E1C22E0AE014F5F5F4FB2
:1026900068EB8EEE0E94D511898190E0982F8827F3
:1026A0002A81822B9093111C8093101C22E0AE0192
:1026B0004F5F5F4F6AEB8EEE0E94D511898190E0EB
:1026C000982F88272A81822B9093151C8093141CA5
:1026D00022E0AE014F5F5F4F6CEB8EEE0E94D51192
:1026E000898190E0982F88272A81822B9093171C4C
:1026F0008093161C22E0AE014F5F5F4F6EEB8EEEB3
:102700000E94D511898190E0982F88272A81822BF9
:102710009093191C8093181C0F900F90DF91CF910C
:1027200008952F923F924F925F926F927F928F9275
:102730009F92AF92BF92CF92DF92EF92FF920F9350
:102740001F93CF93DF93CDB7DEB76A970FB6F89498
:10275000DEBF0FBECDBF182F488F298F19821A8276
:102760001B8280912C1C811107C06A8F0E94BF12AE
:1027700081E080932C1C6A8D662309F46CC04EE2C4
:1027800064EF8EEE0E94BE1169E07AE180E090E095
:102790000E94116122E0AE014F5F5F4F66EF8EEE47
:1027A0000E94D5112981822F90E0A0E0B0E022277D
:1027B000382F492F5A2F8A81282B80911E1C9091E7
:1027C0001F1C281B390B41095109A0911C1CB091F9
:1027D0001D1C0E94D68D6B017C018FE0F594E7945F
:1027E000D794C7948A95D1F76091161C7091171CE5
:1027F000882777FD8095982F2BE0660F771F881F1D
:10280000991F2A95D1F72091181C3091191C442743
:1028100037FD4095542F2C0D3D1D4E1D5F1D0E9410
:102820008C8DC20ED31ED092131CC092121C88E055
:10283000C80ED11C34E0D594C7943A95E1F7EE2444
:10284000D7FCE094FE2CC092201CD092211CE09278
:10285000221CF092231C012F0295000F000F007C18
:102860000C5CA12FB0E0BD8BAC8BA3E0B0E0012EDF
:1028700002C0AA0FBB1F0A94E2F725E335E00E94CD
:10288000CF8DDC01CB010296A11DB11D8C879D87E8
:10289000AE87BF8780E593ECA0E0B0E004C0B595BB
:1028A000A795979587951A95D2F7888B998BAA8BC0
:1028B000BB8B10E0188619861A861B86A8E02A2E84
:1028C000312CAC89BD892A1A3B0A988D191709F455
:1028D00036C1402F64EF8EEE0E94BE116C857D855F
:1028E0008E859F850E94116123E0AE014F5F5F4F8F
:1028F00066EF8EEE0E94D511E091121CF091131C30
:10290000E05AFF409F01DF010E94B88D6B017C01FE
:1029100080910A1C90910B1C9F8B8E8BA090081CA1
:10292000B090091C20910C1C30910D1C0E94B88D98
:102930002B013C013DE075946794579447943A9578
:10294000D1F7A0910E1CB0910F1CA70196016CE06D
:1029500055954795379527956A95D1F70E94E18D52
:10296000BB2797FDB095AB2F480E591E6A1E7B1EE4
:1029700092E0490E511C611C711CB2E07594679481
:1029800057944794BA95D1F7A0E85A0E611C711C70
:10299000A0911A1CB0911B1CA30192010E94D68D1C
:1029A000DC01CB012FE0B695A795979587952A95E1
:1029B000D1F78C839D83AE83BF8329818A8190E088
:1029C000A0E0B0E04424582E692E7A2E622A8B8132
:1029D000482A022C04C075946794579447940A942B
:1029E000D2F74501AA2497FCA094BA2C42E0880CA7
:1029F000991CAA1CBB1C4A95D1F7A091101CB09140
:102A0000111CA70196010E94E18D6B017C0157E129
:102A1000F594E794D794C7945A95D1F72E893F89B6
:102A2000DF010E94B88DEBE09595879577956795C6
:102A3000EA95D1F7C60ED71EE81EF91E8C0C9D1C18
:102A4000AE1CBF1C0C8804C0880C991CAA1CBB1CA3
:102A50000A94D2F792E0890E911CA11CB11CF2E0FD
:102A6000B594A79497948794FA95D1F74818590884
:102A70006A087B08A3019201688979898A899B8900
:102A80000E94328D97FD0DC0660F771F881F991F1A
:102A90002C813D814E815F810E946A8D49015A01DE
:102AA0000CC02C813D814E815F810E946A8D49015D
:102AB0005A01880C991CAA1CBB1C9927B7FC9A9533
:102AC0008B2D7A2D692D9B01AC010E94328D9B01CB
:102AD000AC01AEEDBBE00E94D68D6C01FF24D7FCAB
:102AE000F094EF2CA3E4B3EEA50194010E94E48DD1
:102AF000BB2797FDB095AB2FC80ED91EEA1EFB1E53
:102B0000AFECCA0EAEE0DA1EE11CF11CA4E0F594B5
:102B1000E794D794C794AA95D1F7C80CD91CEA1C9E
:102B2000FB1C88859985AA85BB858C0D9D1DAE1DD6
:102B3000BF1D88879987AA87BB871F5FC6CE1123D1
:102B400091F0212F30E040E050E0688579858A855A
:102B50009B850E946A8D2093241C3093251C4093F2
:102B6000261C5093271CA98DAA2389F16091241C4F
:102B70007091251C8091261C9091271C6115710570
:102B80008105910521F10E94908A20E836EE45ECFE
:102B900057E40E94F18921E03EED42E45EE30E94A9
:102BA000D58C9B01AC0160E070E080E89FE30E945F
:102BB00026892BE43AE34DEB57E30E94F1896093B9
:102BC000281C7093291C80932A1C90932B1C6A96B6
:102BD0000FB6F894DEBF0FBECDBFDF91CF911F912E
:102BE0000F91FF90EF90DF90CF90BF90AF909F90AC
:102BF0008F907F906F905F904F903F902F900895AF
:102C00000F931F93CF93DF9300D000D000D0CDB7A8
:102C1000DEB78E010F5F1F4F86E0F80111928A9593
:102C2000E9F780911E1B811113C040E061E386EA41
:102C30000E94BE114AE06CE286EA0E94BE1181E069
:102C400080931E1B6CE77EE380E090E00E941161A0
:102C500048E06DE286EA0E94BE116CE77EE380E008
:102C600090E00E94116126E0A80162E386EA0E94DA
:102C7000D51147E06DE286EA0E94BE118A8190E09C
:102C8000982F88272981822B9093191B8093181BDA
:102C90002C8130E0322F22274B81242B30931B1BB9
:102CA00020931A1B4E8150E0542F44276D81462BF0
:102CB00050931D1B40931C1B5F934F933F932F9387
:102CC0009F938F938BEF93E09F938F930E94219418
:102CD0000FB6F894DEBF0FBECDBF26960FB6F894A0
:102CE000DEBF0FBECDBFDF91CF911F910F91089531
:102CF000CF92DF92EF92FF920F931F93CF93DF93C8
:102D0000CDB7DEB72A970FB6F894DEBF0FBECDBFA2
:102D10008E010F5F1F4F86E0F80111928A95E9F747
:102D200041E062E08CE30E94BE1148E560E08CE384
:102D30000E94BE1162E174E380E090E00E941161A4
:102D400026E0A80163E08CE30E94D51143E062E035
:102D50008CE30E94BE11098110E0102F00278A81A8
:102D6000082B1093F91A0093F81AEB80F12CFE2C23
:102D7000EE248C81E82AF092FB1AE092FA1ACD80B8
:102D8000D12CDC2CCC248E81C82AD092FD1AC09282
:102D9000FC1AB801882777FD8095982F0E94908AA9
:102DA0009B01AC01B701882777FD8095982F2F8371
:102DB000388749875A870E94908A2F8138854985AC
:102DC0005A850E949A8920EE3EE245E652E40E942E
:102DD000728C20E030E044E353E40E9427899F9303
:102DE0008F937F936F93DF92CF92FF92EF921F9317
:102DF0000F9389E094E09F938F930E9421940FB6E4
:102E0000F894DEBF0FBECDBF2A960FB6F894DEBF92
:102E10000FBECDBFDF91CF911F910F91FF90EF902B
:102E2000DF90CF900895CF93DF93EC018881998153
:102E30000097F9F0873D904121F01982188283E0D4
:102E400063C085ED99E00E946358892BE1F0809181
:102E5000C5099091C60993FD18C08091C50990914C
:102E6000C60994FD43C08091C5099091C60995FD9E
:102E700044C060E870E085ED99E00E943C5887ED21
:102E800090E19983888381E03FC080913D2082FF5B
:102E9000E4CF21E048E061E083E00E94911380915B
:102EA0002B1C8F9380912A1C8F938091291C8F93C8
:102EB0008091281C8F938091271C8F938091261CD2
:102EC0008F938091251C8F938091241C8F9384E590
:102ED0009FE09F938F930E9433948DB79EB70A967D
:102EE0000FB6F8949EBF0FBE8DBFB7CF80913D2027
:102EF00083FFB9CF0E940016B6CF80913D2084FF9A
:102F0000B8CF0E947816B5CFDF91CF910895CF93B7
:102F1000C82F8CEE0E9495618C2F0E949F6165E303
:102F200075E080E090E00E9411618DEE0E94956155
:102F30000E94B061C82F0E94BA612C2F30E0322F5E
:102F40002227A901482BCA01CF910895CF93DF937F
:102F5000C82F8CEE0E9495618C2F0E949F6162E1C8
:102F600074E380E090E00E9411618CEE0E94956114
:102F700080E00E949F6165E375E080E090E00E9440
:102F800011618DEE0E9495610E94B061C82F0E9470
:102F9000B061D82F0E94BA614D2F50E060E070E020
:102FA000762F652F542F44276C2B482BCB01BA0169
:102FB000DF91CF9108952F923F924F925F926F923F
:102FC0007F928F929F92AF92BF92CF92DF92EF92B9
:102FD000FF920F931F93CF93DF93CDB7DEB7CD54FE
:102FE000D1090FB6F894DEBF0FBECDBF80910002AD
:102FF00090910102892BD1F11092010210920002EE
:103000008CEE0E9495618EE10E949F616BE17EE4EF
:1030100080E090E00E94116182EA0E9487179093FD
:10302000D2098093D10984EA0E9487179093D0092E
:103030008093CF0986EA0E9487179093CE098093E8
:10304000CD0988EA0E9487179093CC098093CB0919
:103050008AEA0E9487179093CA098093C9098CEA6B
:103060000E9487179093C8098093C70988E40E943B
:10307000A6176FAB78AF89AF9AAF88E50E94A61705
:103080004B015C018091C9099091CA0920E030E0B0
:1030900040E050E0BA0126962FAF269727963FAF23
:1030A000279728964FAF289729965FAF29972A969A
:1030B0006FAF2A972B967FAF2B979C0140E050E093
:1030C00060E070E080E090E008E00E94448F0E94A1
:1030D000FD8E3901B42FA52FF62FE72F8C01940117
:1030E000A50160E070E080E090E05301CB2EDA2E85
:1030F000EF2EFE2E0E947B8F29833A832A011B012B
:103100004C01B101C401315041095F4F6F4F7F4FF6
:103110008F4F9F4FA1E0B0E02596BFAFAEAF259790
:1031200021153F4F4F4F51406105710581059105B4
:1031300009F020F425961FAE1EAE259725966EAC9D
:103140007FAC25978091C7099091C8095C01C12C7B
:10315000D12CE12CF12C00E010E029813A81A20170
:10316000B101C4010E94E98DD22EE32EF42E052F69
:10317000162FB72FF82FE92FA0E00E94A28F84F41A
:103180002150310940485F4F6F4F7F4F8F4F9F4F06
:10319000D22EE32EF42E052F162FB72FF82FE92F5E
:1031A0002D2D3E2D4F2D502F612F7B2F8F2F9E2F9A
:1031B00007E10E945D8F2B8F3C8F4D8F5E8F6F8F4D
:1031C00078A389A39AA32053384F4F4F5F4F6F4F77
:1031D0007F4F8F4F9F4F2B8B3C8B4D8B5E8B6F8B1D
:1031E000788F898F9A8F2056304F4F4F5F4F6F4F98
:1031F0007F4F8F4F9F4F243D30434105510561055F
:1032000071058105910541F038F025966EAC7FACD3
:103210002597FFEF6F1A7F0A8091CF099091D0090F
:103220009C0140E050E060E070E080E090E000E170
:103230000E94448F2B833C834D835E836A8779870A
:103240008F8398874091CB095091CC09A980BA808F
:103250006201710184019A0140E050E060E070E099
:1032600080E090E00E94E98DD22EE32EF42E052F0F
:10327000162FB72FF82FE92FA0E00E94A28F5CF441
:10328000AFE70E94848FD22EE32EF42E052F162F47
:10329000B72FF82FE92F2D2D3E2D4F2D502F612FB9
:1032A0007B2F8F2F9E2F07E00E945D8F59016A01AF
:1032B0007B018C012B813C814D815E816A85798502
:1032C0008F8198850E947B8F2B833C834D835E8307
:1032D0006F8378878F87988B2E5F3F4F43405109CC
:1032E0006E4F7F4F8F4F9F4F22303105494F5F4FB9
:1032F000644071058105910521F018F01FEF611AF6
:10330000710A8091D1099091D209BC0180E090E0CE
:1033100020E030E840E050E00E94428E29873A8762
:103320004B875C876A8B798B8D879E874091CD090F
:103330005091CE09A980BA806201710184019A017D
:1033400040E050E060E070E080E090E00E94E98DB5
:10335000D22EE32EF42E052F162FB72FF82FE92F9C
:10336000A0E00E94A28F84F421503F4F4F4F5F4F47
:103370006F4F7F4F8F4F9F4FD22EE32EF42E052F8E
:10338000162FB72FF82FE92F2D2D3E2D4F2D502F13
:10339000612F7B2F8F2F9E2F08E00E945D8F590198
:1033A0006A017B018C0129853A854B855C856A8998
:1033B00079898D859E850E947B8F29873A874B87E7
:1033C0005C876D877E87898B9A8B2F5F3F4F41404B
:1033D00051096109710981099109213030484C4F27
:1033E0005F47614071058105910521F018F0BFEF3D
:1033F0006B1A7B0A2B893C894D895E896F89788D90
:10340000898D9A8D2F3C3740410551056105710525
:103410008105910511F00CF0A5C1A980BA80620167
:10342000710184019501A201B101C4010E94E98DDD
:10343000A12CB12CC12C10E8D12EE12CF12C00E0F4
:1034400010E00E946F8E2BAF3CAF4DAF5EAF6FAF01
:1034500021967FAF219722968FAF229723969FAF19
:103460002397AB8CBC8CCD8CDE8CEF8CF8A009A1A3
:103470001AA19501A601B701C8010E94E98D590161
:103480006A017B01E82F192F02E00E94448F0E2F62
:103490000E947B8F69017A01162F272EF82FE92FC2
:1034A000322E8D2C942EAF2CB62E072F582EB92FDE
:1034B000A0E00E94A28F5CF4A1E00E94848F322ED3
:1034C000832E942EA52EB62E072F582EB92F232DDE
:1034D000382D492D5A2D6B2D702F852D9B2F01E0F6
:1034E0000E945D8F2E962FAF2E972D963FAF2D9772
:1034F00049A75AA76BA77CA78DA79EA7522E432E3C
:103500004BA35CA36DA37EA38FA398A7B22D9601B6
:10351000A701612F722D8F2F9E2FA0E00E94A28FF6
:103520004CF4A3E00E94848F69017A01162FB72F13
:10353000F82FE92F9601A701612F7B2F8F2F9E2F48
:1035400002E00E945D8F2FA738AB49AB5AAB6BAB43
:103550007CAB8DAB9EAB19014A01B62FA72F2496E9
:103560008FAF2497F92F2B893C894D895E896F890C
:10357000788D898D9A8D24323A4F4F4F5F4F6F4F20
:103580007F4F8F4F9F4F0CF08CC02B8D3C8D4D8DFE
:103590005E8D6F8D78A189A19AA12455324F4F4F2E
:1035A0005F4F6F4F7F4F8F4F9F4F59016A017B01D4
:1035B0008C010E94E98D19014A01B62FA72FFC0149
:1035C00003E00E94448F51016401EB2EFA2E8F011B
:1035D0000E94908F59016A017B018C012E962FADBC
:1035E0002E972D963FAD2D9749A55AA56BA57CA585
:1035F0008DA59EA50E947B8F522E432E4BA35CA3CC
:103600006DA37EA38FA398A79101A4016B2F7A2F9E
:10361000CF0102E00E94448F51016401EB2EFA2E8B
:103620008F010E94908F02E00E94448F0E2F0E9413
:10363000908FF22E032F142FD52EE62EB72FF82FB2
:10364000E92FA0E00E94A28F5CF4A1E00E94848F89
:10365000F22E032F142FD52EE62EB72FF82FE92F99
:103660002F2D302F412F5D2D6E2D7B2F8F2F9E2FD5
:1036700001E00E945D8F59016A017B018C012FA539
:1036800038A949A95AA96BA97CA98DA99EA90E940C
:103690007B8F19014A01B62FA72F24968FAF24974D
:1036A000F92F2B813C814D815E816F8178858F85DB
:1036B0009889A52CB42CCBA0DCA0EDA0FEA00FA176
:1036C00018A50E94908F2B833C834D835E836F836C
:1036D00078878F87988B29853A854B855C856D85A2
:1036E0007E8589899A8951016401EB2EFA2E2496F0
:1036F0000FAD24971F2F0E94908F29873A874B8701
:103700005C876D877E87898B9A8B2B893C894D8955
:103710005E896F89788D898D9A8DABACBCACCDAC50
:10372000DEACEFAC2196FFAC219722960FAD22972D
:1037300023961FAD23970E94908F2056304F4F4FF6
:103740005F4F6F4F7F4F8F4F9F4F243D3043410559
:103750005105610571058105910521F018F02FEFE4
:10376000621A720A6FA978AD89AD9AADAB01BC013E
:1037700080E090E0DC0124964FAF249725965FAF60
:10378000259726966FAF269727967FAF279728967F
:103790008FAF289729969FAF29972A96AFAF2A9780
:1037A0002B96BFAF2B97A984BA84CB84DC84ED849D
:1037B000FE8409891A899A01AB0160E070E080E01B
:1037C00090E00E94E98DF22E032F142FD52EE62EC5
:1037D000B72FF82FE92FA0E00E94A28F84F4215088
:1037E0003109404E5F4F6F4F7F4F8F4F9F4FF22EEB
:1037F000032F142FD52EE62EB72FF82FE92F2F2DBC
:10380000302F412F5D2D6E2D7B2F8F2F9E2F05E1A9
:103810000E945D8FAB80BC80CD80DE80EF80F8841D
:103820000F8518890E94908FF22E032F142FD52E0A
:10383000E62EB72FF82FE92FA0E00E94A28F84F484
:10384000215030484F4F5F4F6F4F7F4F8F4F9F4FEB
:10385000F22E032F142FD52EE62EB72FF82FE92F97
:103860002F2D302F412F5D2D6E2D7B2F8F2F9E2FD3
:103870000FE00E945D8F69017A018B018A83998331
:1038800029011A014B015C01285E334041095109AD
:103890006109710981099109283D304D4140510567
:1038A000610571058105910521F018F0BFEF6B1AD4
:1038B0007B0A0E949761672859F09601A701B80119
:1038C0008A8199810E94FD8E29011A014B015C01B8
:1038D0009201A101B401C5010E948A8A20E030E072
:1038E00048EC52E40E94F189C35BDF4F0FB6F894B5
:1038F000DEBF0FBECDBFDF91CF911F910F91FF9023
:10390000EF90DF90CF90BF90AF909F908F907F907F
:103910006F905F904F903F902F9008954F925F92DD
:103920006F927F928F929F92AF92BF92CF92DF92CF
:10393000EF92FF922B013C0169017A0123EC35EFF4
:103940004CE851E4C701B6010E94728C4B015C0146
:1039500028EB3EE143E753E4C701B6010E94278903
:103960009B01AC01C501B4010E94F1890E945E8AED
:103970004B015C0120E030E048EC52E4C301B201AD
:103980000E94F18921E835E943EC50E40E94728CF1
:10399000A50194010E94728C4B015C0123E333E981
:1039A00048E853E4C701B6010E9427899B01AC0196
:1039B000C501B4010E94F18923E333EB48E553E4E8
:1039C0000E94728CFF90EF90DF90CF90BF90AF90ED
:1039D0009F908F907F906F905F904F9008954F923F
:1039E0005F926F927F928F929F92AF92BF92CF928F
:1039F000DF92EF92FF9269017A010E94F48B20E03E
:103A000030E040E050E40E94268922E93CE54EED9A
:103A10005EE30E94F1894B015C0123EC35EF4CE839
:103A200051E4C701B6010E94728C2B013C0128EBC6
:103A30003EE143E753E4C701B6010E9427899B0199
:103A4000AC01C301B2010E94F1899B01AC01C50127
:103A5000B4010E9427896B017C0128EB3EE143E71A
:103A600053E40E94728C4B015C01A701960163EC48
:103A700075EF8CE891E40E9426899B01AC01C50199
:103A8000B4010E94F189FF90EF90DF90CF90BF903A
:103A9000AF909F908F907F906F905F904F90089520
:103AA0004F925F926F927F928F929F92AF92BF924E
:103AB000CF92DF92EF92FF922B013C0169017A01D4
:103AC00023EC35EF4CE851E4C701B6010E94728C3B
:103AD0004B015C0128EB3EE143E753E4C701B6012B
:103AE0000E9427899B01AC01C501B4010E94F189A4
:103AF0000E945E8A4B015C0120E030E048EC52E419
:103B0000C301B2010E94F189A50194010E94728C47
:103B100020E030E040E251E40E94268924EE38E3C0
:103B20004EE05FE30E94728C9B01AC01C701B601BD
:103B30000E942789FF90EF90DF90CF90BF90AF90C9
:103B40009F908F907F906F905F904F90089580E846
:103B50000E94956181110DC08EEF0E949F618111BD
:103B600008C06BE17EE480E090E00E9411610C945B
:103B700097610E94976180914F2490915024A09169
:103B80005124B09152240196A11DB11D80934F2460
:103B900090935024A0935124B09352240895FC0193
:103BA000DC0182E020E041E39D91292798E0322F5B
:103BB000330F27FF03C0232F242701C0232F915049
:103BC000B1F7815089F781E090E03281231711F03D
:103BD00080E090E00895DF92EF92FF920F931F93A1
:103BE000CF93DF930E94A71D80E80E949561811109
:103BF0006DC08AEF0E949F61811168C08FE00E94B2
:103C00009F61811163C065E375E080E090E00E94F0
:103C1000116181E80E949561811158C00E94B061D4
:103C2000C82F0E94B0610E94B061D82F0E94B0617D
:103C30000E94B061182F0E94B0610E94BA61082FE3
:103C400080E80E949561811141C08CEF0E949F61C4
:103C500081113CC089EC0E949F61811137C065E3EE
:103C600075E080E090E00E94116181E80E9495611A
:103C70000E94B061E82E0E94B061D82E0E94B0610F
:103C80000E94B061F82E0E94BA611F92DF921F92CB
:103C9000EF921F920F931F921F931F92DF931F9219
:103CA000CF931F928F931F92FF928EE194E09F9388
:103CB0008F930E9421940E9497618DB79EB7429680
:103CC0000FB6F8949EBF0FBE8DBF17C00E949761BC
:103CD00080914F2490915024A0915124B09152246E
:103CE0000196A11DB11D80934F2490935024A09361
:103CF0005124B09352240E94A71D20E030E040E000
:103D000050E060E070E080E090E0DF91CF911F91A3
:103D10000F91FF90EF90DF900895EF92FF920F9335
:103D20001F93CF93DF9300D01F92CDB7DEB78C01E6
:103D300080E80E949561811154C00115110551F070
:103D400085EE0E949F6181114CC061E077E980E0BF
:103D500090E009C083EE0E949F61811142C069E931
:103D60007AEB81E090E00E94116181E80E94956108
:103D7000811137C00E94B061F82E89830E94B06122
:103D8000E82E8A830E94BA618B830E949761CE01DC
:103D900001960E94CF1D892B21F16E2D70E07F29A5
:103DA0006C7F80E090E0012B69F00E948E8A20E019
:103DB00030E04AEF5AE30E94728C20E030E040ECA1
:103DC00050E40CC00E948E8A22E538EB4FE25BE3A0
:103DD0000E94728C26E636E64BE352E40E94268966
:103DE0001BC00E94976180914F2490915024A09114
:103DF0005124B09152240196A11DB11D80934F24EE
:103E000090935024A0935124B09352240E94A71D54
:103E100060EF7FEF89E794E40F900F900F90DF91B0
:103E2000CF911F910F91FF90EF9008950F931F93E3
:103E3000CF93DF93729A8091580283FF08C08EE47B
:103E40000E943361811167C0C0E5D0E00AC0C0E5BF
:103E5000D0E087EE93E00E948C0921972097C9F764
:103E6000EECF87EE93E00E948C0921972097C9F747
:103E70008FE40E9433610E94B061082F0F730E948B
:103E8000B061182F0E94B061D82F0E94BA61C82F6C
:103E90000E9497618091580283FF7298602F70E0B2
:103EA000762F6627610F711D80E090E00E948E8A58
:103EB00020E134E048EC5BE30E94728C6093311C9B
:103EC0007093321C8093331C9093341C6D2F70E0E0
:103ED000762F66276C0F711D769567957695679599
:103EE00080E090E00E948E8A24EA3CEF44E25CE3AA
:103EF0000E94728C20E030E040E252E40E94268969
:103F000060930E2970930F298093102990931129A3
:103F100080E090E002C081E090E0DF91CF911F91BE
:103F20000F9108957298729A8EE40E94336180EA2C
:103F30000E949F6180E00E949F6180E00E949F61DB
:103F40008FE40E9433610E94B0618EE40E9433616D
:103F500080E80E949F6180E00E949F6180E00E9453
:103F60009F610E94976180E090E0089588EE9EE056
:103F70009F938F930E943394809173020F900F90C0
:103F8000882361F01F928F9385EE9EE09F938F931D
:103F90000E9433940F900F900F900F90089580EC33
:103FA0009EE09F938F930E94339488E99EE09F93B5
:103FB0008F930E94339481E79EE09F938F930E949A
:103FC000339486E39EE09F938F930E94339484E022
:103FD0009EE09F938F930E94339488EC9DE09F9383
:103FE0008F930E94339482EA9DE09F938F930E9467
:103FF00033948CE69DE09F938F930E94339480913D
:104000003D2090913E20827091702DB73EB7205F89
:104010003F4F0FB6F8943EBF0FBE2DBF892B41F026
:104020008CE39DE09F938F930E9433940F900F90A9
:1040300080E19DE09F938F930E94339484ED9CE0F8
:104040009F938F930E9433948BEA9CE09F938F936E
:104050000E9433948FE79CE09F938F930E94339448
:1040600080E59CE09F938F930E9433948EE19CE0C7
:104070009F938F930E9433948DEE9BE09F938F9339
:104080000E94339483EB9BE09F938F930E94339421
:104090008DE79BE09F938F930E9433948DE49BE088
:1040A0009F938F930E94339481E29BE09F938F9321
:1040B0000E94339482EF9AE09F938F930E943394EF
:1040C00089EB9AE09F938F930E94339480E89AE063
:1040D0009F938F930E94339489E49AE09F938F93E8
:1040E0000E94339485E19AE09F938F930E943394CA
:1040F0008DB79EB780960FB6F8949EBF0FBE8DBF4A
:1041000084EE99E09F938F930E94339485EB99E01E
:104110009F938F930E94339486E899E09F938F93A7
:104120000E9433948FE599E09F938F930E9433947C
:1041300089E299E09F938F930E94339483EF98E0F4
:104140009F938F930E9433948DEB98E09F938F936E
:104150000E94339484E998E09F938F930E94339454
:104160008CE598E09F938F930E94339481E398E0CD
:104170009F938F930E9433942DB73EB72C5E3F4F91
:104180000FB6F8943EBF0FBE2DBF08958DE494E0A6
:104190000C9457944F925F926F927F928F929F925E
:1041A000AF92BF92CF92DF92EF92FF92CF93DF93C5
:1041B000CDB7DEB728970FB6F894DEBF0FBECDBFE0
:1041C0008091432490914424A0914524B0914624A9
:1041D00089839A83AB83BC834090432450904424CA
:1041E000609045247090462480914324909144240B
:1041F000A0914524B09146248D839E83AF83B887D8
:1042000060914324709144248091452490914624E8
:104210002CE3822E912CA12CB12CA50194010E949B
:104220006A8D7F936F9330E1C32E3EE0D32EE12C55
:10423000F12C6D817E818F819885A70196010E9466
:104240006A8DA50194010E946A8D3F932F9340E8E7
:10425000842E41E5942EAA24A394B12CC301B2016B
:10426000A50194010E946A8DA70196010E946A8DA2
:104270003F932F9369817A818B819C81A501940161
:104280000E946A8D3F932F938BE098E09F938F93CA
:104290000E9433940FB6F894DEBF0FBECDBF2896B0
:1042A0000FB6F894DEBF0FBECDBFDF91CF91FF9068
:1042B000EF90DF90CF90BF90AF909F908F907F90C6
:1042C0006F905F904F900895E3EDF1E380819181CD
:1042D0008234924479F0E35DF143FF93EF938DEEE6
:1042E00097E09F938F930E9433940F900F900F90BD
:1042F0000F9008953A96E53F81E4F80738F3089562
:10430000CF93DF93EC018C9A0E94D70A9F938F93EF
:104310007F936F9381EE97E09F938F930E943394E6
:104320000F900F900F900F900F900F90209719F013
:104330000E94F20B08C08FED97E09F938F930E942D
:1043400033940F900F9081E00E94880A20917802A8
:104350003091790240917A0250917B020E94728CD6
:104360009F938F937F936F9383ED97E09F938F93AA
:104370000E9433940F900F900F900F900F900F901A
:10438000209719F00E94F20B08C081ED97E09F93EF
:104390008F930E9433940F900F9082E00E94880ABE
:1043A000209174023091750240917602509177020B
:1043B0000E94728C9F938F937F936F9385EC97E00D
:1043C0009F938F930E9433940F900F900F900F90B4
:1043D0000F900F90209719F00E94F20B08C083EC09
:1043E00097E09F938F930E9433940F900F9083E0F8
:1043F0000E94880A9F938F937F936F9384EB97E03B
:104400009F938F930E9433948C980F900F900F90EE
:104410000F900F900F90209719F00E94F20B08C098
:1044200082EB97E09F938F930E9433940F900F90AD
:1044300080913D2087FF83C021E042E161E080ED73
:104440000E94F7629F938F937F936F9385EA97E023
:104450009F938F930E9433940F900F900F900F9023
:104460000F900F90209719F00E94F20B08C083EA7A
:1044700097E09F938F930E9433940F900F9021E0C9
:1044800042E162E080ED0E94F7629F938F937F93F9
:104490006F9386E997E09F938F930E9433940F90D8
:1044A0000F900F900F900F900F90209719F00E948F
:1044B000F20B08C084E997E09F938F930E94339496
:1044C0000F900F9021E042E163E080ED0E94F762DF
:1044D0009F938F937F936F9387E897E09F938F933A
:1044E0000E9433940F900F900F900F900F900F90A9
:1044F000CD2B19F00E94F20B08C085E897E09F933E
:104500008F930E9433940F900F9021E042E164E07A
:1045100080ED0E94F7629F938F937F936F9388E75C
:1045200097E09F938F930E9433940F900F900F907A
:104530000F900F900F90DF91CF910C94F20BCD2B39
:10454000D1F3DF91CF9108950F931F93CF93DF9312
:10455000882389F049E050E06FEF70E082E099E253
:104560000E94759349E050E06AE070E082E099E2D1
:104570000E94A59513C0C2E0D9E203E717E0899134
:104580001F928F931F930F930E9433940F900F905D
:104590000F900F9089E2CA30D80789F7DF91CF9149
:1045A0001F910F910C94F20B882311F02A9A089511
:1045B0002A980895882311F02B9A08952B9808952E
:1045C000CF92DF92EF92FF92CF93DF936B017C014A
:1045D00060FF11C08AE894E09F938F938DEF9EE077
:1045E0009F938F930E9433940F900F900F900F9092
:1045F00081E090E002C080E090E0C1FE09C0EC01E3
:10460000219643E259E06FE874E00E944A10CE011F
:10461000C2FE09C0EC01219643E259E067E974E06B
:104620000E944A10CE01C3FE09C0EC01219643E26C
:1046300059E06FE974E00E944A10CE01C4FE09C03F
:10464000EC01219643E259E063EA74E00E944A10CB
:10465000CE01C5FE09C0EC01219643E259E066EAAD
:1046600074E00E944A10CE01C6FE09C0EC012196FA
:1046700043E259E06AEA74E00E944A10CE01C7FEA4
:1046800009C0EC01219643E259E060EB74E00E941E
:104690004A10CE01D0FE09C0EC01219643E259E058
:1046A00068EB74E00E944A10CE01D1FE09C0EC0113
:1046B000219643E259E060EC74E00E944A10CE017A
:1046C000D2FE09C0EC01219643E259E064EC74E0AB
:1046D0000E944A10CE0120913D2030913E2024704E
:1046E0003270232B59F0D3FE09C0EC01219643E22E
:1046F00059E06AEC74E00E944A10CE0120913D20FE
:1047000023FF0BC0D4FE09C0EC01219643E259E01F
:104710006FEC74E00E944A10CE0120913D2024FFEE
:104720000BC0D5FE09C0EC01219643E259E065EDCE
:1047300074E00E944A10CE01D6FE09C0EC01219619
:1047400043E259E06DED74E00E944A10CE01B701DA
:10475000A60144275078452B462B472B61F043E2B6
:1047600059E068EE74E0DF91CF91FF90EF90DF9019
:10477000CF900C944A10CD28CE28CF2841F48EE655
:1047800097E09F938F930E9433940F900F90DF9147
:10479000CF91FF90EF90DF90CF9008950F931F93EC
:1047A000CF93DF938C01C0E0D0E00115110509F42F
:1047B0008AC069E677E0C8010E945493892B09F406
:1047C000C16061E677E0C8010E945493892B09F427
:1047D000C26069E577E0C8010E945493892B09F40F
:1047E000C46065E577E0C8010E945493892B09F401
:1047F000C86062E577E0C8010E945493892B09F4F0
:10480000C0616EE477E0C8010E945493892B09F4DB
:10481000C06268E477E0C8010E945493892B09F4D0
:10482000C06460E477E0C8010E945493892B09F4C6
:10483000C06868E377E0C8010E945493892B09F4AB
:10484000D16064E377E0C8010E945493892B09F496
:10485000D2606EE277E0C8010E945493892B09F47C
:10486000D46069E277E0C8010E945493892B09F46F
:10487000D86063E277E0C8010E945493892B09F461
:10488000D0616BE177E0C8010E945493892B09F451
:10489000D06260E177E0C8010E945493892B09F44B
:1048A000D0646FEF76E0C8010E945493892B09F41D
:1048B000D068609171027091720280E090E00E9475
:1048C00068938C0172CFCE01DF91CF911F910F9130
:1048D0000895AF92BF92CF92DF92EF92FF920F9323
:1048E0001F93CF93DF93F22E032F142FE52ED62E96
:1048F000A72EB82EC92E217030E040E050E060E0D5
:1049000070E080E090E0A0E00E94A28F89F0E9EFE3
:10491000F4E0FF93EF93EDEFFEE0FF93EF930E943F
:1049200033940F900F900F900F90E1E0F0E002C0F1
:10493000E0E0F0E080913D2080FF17C02F2D247033
:1049400030E040E050E060E070E080E090E0A0E027
:104950000E94A28F51F0EF01219643E259E06DEFE2
:1049600074E0CF010E944A10FE012F2D227030E02A
:1049700040E050E060E070E080E090E0A0E00E9465
:10498000A28F51F0EF01219643E259E061E075E01A
:10499000CF010E944A10FE012F2D287030E040E028
:1049A00050E060E070E080E090E0A0E00E94A28F24
:1049B00051F0EF01219643E259E069E175E0CF0142
:1049C0000E944A10FE012F2D207130E040E050E09F
:1049D00060E070E080E090E0A0E00E94A28F51F0E3
:1049E000EF01219643E259E064E075E0CF010E94B7
:1049F0004A10FE012F2D207230E040E050E060E0D0
:104A000070E080E090E0A0E00E94A28F51F0EF0102
:104A1000219643E259E067E075E0CF010E944A1019
:104A2000FE012F2D207430E040E050E060E070E0A7
:104A300080E090E0A0E00E94A28F51F0EF0121966B
:104A400043E259E06DE075E0CF010E944A10FE019B
:104A50002F2D207830E040E050E060E070E080E012
:104A600090E0A0E00E94A28F51F0EF01219643E276
:104A700059E063E175E0CF010E944A10FE0120E099
:104A8000302F317040E050E060E070E080E090E076
:104A9000A0E00E94A28F51F0EF01219643E259E07D
:104AA00066E175E0CF010E944A10FE0120E0302F40
:104AB000327040E050E060E070E080E090E0A0E024
:104AC0000E94A28F51F0EF01219643E259E06BE181
:104AD00075E0CF010E944A10FE0120E0302F3470B3
:104AE00040E050E060E070E080E090E0A0E00E94F4
:104AF000A28F51F0EF01219643E259E062E275E0A6
:104B0000CF010E944A10FE0120E0302F387040E0B3
:104B100050E060E070E080E090E0A0E00E94A28FB2
:104B200051F0EF01219643E259E065E275E0CF01D3
:104B30000E944A10FE0120E0302F307140E050E02A
:104B400060E070E080E090E0A0E00E94A28F51F071
:104B5000EF01219643E259E06AE275E0CF010E943D
:104B60004A10FE0120E0302F307240E050E060E05B
:104B700070E080E090E0A0E00E94A28F51F0EF0191
:104B8000219643E259E061E375E0CF010E944A10AB
:104B9000FE0120E030E040E050E06D2D647070E0F8
:104BA00080E090E0A0E00E94A28F51F0EF012196FA
:104BB00043E259E068E375E0CF010E944A10FE012C
:104BC00080913D2081FF17C020E0302F307440E0FD
:104BD00050E060E070E080E090E0A0E00E94A28FF2
:104BE00051F0EF01219643E259E06CE375E0CF010B
:104BF0000E944A10FE0180913D2090913E2090FF3E
:104C000017C020E030E040E05E2D507160E070E0C1
:104C100080E090E0A0E00E94A28F51F0EF01219689
:104C200043E259E06FE375E0CF010E944A10FE01B4
:104C300080913D2090913E2090FF17C020E030E011
:104C400040E05E2D507260E070E080E090E0A0E017
:104C50000E94A28F51F0EF01219643E259E062E4F5
:104C600075E0CF010E944A10FE0180913D20909195
:104C70003E2090FF17C020E030E040E05E2D5074F1
:104C800060E070E080E090E0A0E00E94A28F51F030
:104C9000EF01219643E259E068E475E0CF010E94FC
:104CA0004A10FE0120E0302F307840E050E060E014
:104CB00070E080E090E0A0E00E94A28F51F0EF0150
:104CC000219643E259E063E575E0CF010E944A1066
:104CD000FE0120E030E0412F417050E060E070E0E4
:104CE00080E090E0A0E00E94A28F51F0EF012196B9
:104CF00043E259E068E575E0CF010E944A10FE01E9
:104D000020E030E0412F427050E060E070E080E051
:104D100090E0A0E00E94A28F51F0EF01219643E2C3
:104D200059E06BE575E0CF010E944A10FE0120E0DA
:104D300030E0412F447050E060E070E080E090E0AF
:104D4000A0E00E94A28F51F0EF01219643E259E0CA
:104D50006EE575E0CF010E944A10FE0180913D2072
:104D600087FF17C020E030E0412F487050E060E03E
:104D700070E080E090E0A0E00E94A28F51F0EF018F
:104D8000219643E259E061E675E0CF010E944A10A6
:104D9000FE0180913D2087FF17C020E030E0412FC9
:104DA000407150E060E070E080E090E0A0E00E94A0
:104DB000A28F51F0EF01219643E259E065E675E0DC
:104DC000CF010E944A10FE0180913D2087FF17C04D
:104DD00020E030E0412F407250E060E070E080E081
:104DE00090E0A0E00E94A28F51F0EF01219643E2F3
:104DF00059E069E675E0CF010E944A10FE018091FA
:104E00003D2087FF17C020E030E0412F407450E084
:104E100060E070E080E090E0A0E00E94A28F51F09E
:104E2000EF01219643E259E06DE675E0CF010E9463
:104E30004A10FE0180913D2082FF17C020E030E043
:104E4000412F407850E060E070E080E090E0A0E02A
:104E50000E94A28F51F0EF01219643E259E06DE3E9
:104E600076E0CF010E944A10FE0180913D2082FF32
:104E700017C020E030E040E05E2D517060E070E04F
:104E800080E090E0A0E00E94A28F51F0EF01219617
:104E900043E259E061E775E0CF010E944A10FE014C
:104EA00080913D2090913E2090FF17C020E030E09F
:104EB00040E05E2D527060E070E080E090E0A0E0A5
:104EC0000E94A28F51F0EF01219643E259E064E77E
:104ED00075E0CF010E944A10FE0180913D20909123
:104EE0003E2090FF17C020E030E040E05E2D54707F
:104EF00060E070E080E090E0A0E00E94A28F51F0BE
:104F0000EF01219643E259E06CE775E0CF010E9482
:104F10004A10FE0180913D2090913E2091FF1EC0DD
:104F200020E030E040E05E2D587060E070E080E00E
:104F300090E0A0E00E94A28F89F043E259E065E88A
:104F400075E0CF01DF91CF911F910F91FF90EF900E
:104F5000DF90CF90BF90AF900C944A102F2D302F40
:104F6000412F5E2D6D2D7A2D8B2D9C2DA0E00E9462
:104F7000A28F41F48AEF96E09F938F930E9433941F
:104F80000F900F90DF91CF911F910F91FF90EF90B5
:104F9000DF90CF90BF90AF9008958F929F92BF9275
:104FA000DF92EF920F931F93CF93DF93EC014B01AE
:104FB000FB01108265EF76E00E945493892B61F526
:104FC00080913D207DE4D72EE0E8EE2E82FD02C0E8
:104FD00004E001C004E810E0B12C81FF02C060ECE5
:104FE000E62E26E04AE250E06BE270E089E290E0D3
:104FF0000E94385E81E090E00E94800B882311F0CF
:105000005DE5D52E80913D2090913E2090FD16E0EB
:1050100091FF07C0186005C0D12CE12C00E010E022
:10502000B12C63EF76E0CE010E945493892B61F49A
:1050300081E0F4018083609171027091720280E0DE
:1050400090E00E946893EC0161EF76E0CE010E944F
:105050005493892B61F48FEFF40180836091710286
:105060007091720280E090E00E946893EC012097BA
:1050700009F424C16DEE76E0CE010E945493892B91
:1050800019F4FD2DF160DF2E69EE76E0CE010E946D
:105090005493892B19F48D2D8460D82E66EE76E01A
:1050A000CE010E945493892B19F4ED2DE260DE2E7F
:1050B00064EE76E0CE010E945493892B19F4FD2D05
:1050C000F860DF2E61EE76E0CE010E945493892BCA
:1050D00019F48D2D8061D82E6BED76E0CE010E9403
:1050E0005493892B19F4ED2DE062DE2E65ED76E008
:1050F000CE010E945493892B19F4FD2DF064DF2E0C
:1051000062ED76E0CE010E945493892B19F48D2D27
:105110008068D82E6DEC76E0CE010E945493892BE6
:1051200019F4EE2DE160EE2E66EC76E0CE010E94E1
:105130005493892B19F4FE2DF260EF2E63EC76E088
:10514000CE010E945493892B19F48E2D8460E82E91
:105150006EEB76E0CE010E945493892B19F4EE2D6C
:10516000E860EE2E67EB76E0CE010E945493892B27
:1051700019F4FE2DF061EF2E60EB76E0CE010E9477
:105180005493892B19F48E2D8062E82E6CEA76E018
:10519000CE010E945493892B19F4EB2DE460BE2EAE
:1051A00069EA76E0CE010E945493892B19F4FE2D12
:1051B000F064EF2E64EA76E0CE010E945493892BCE
:1051C00019F48E2D8068E82E61EA76E0CE010E9407
:1051D0005493892B09F401606EE976E0CE010E94B8
:1051E0005493892B09F402606BE976E0CE010E94AA
:1051F0005493892B09F4046067E976E0CE010E949C
:105200005493892B09F4086063E976E0CE010E948B
:105210005493892B09F400616FE876E0CE010E9477
:105220005493892B09F400626BE876E0CE010E946A
:105230005493892B09F4006469E876E0CE010E945A
:105240005493892B09F4006866E876E0CE010E9449
:105250005493892B09F411606EE776E0CE010E9429
:105260005493892B09F4126065E776E0CE010E9421
:105270005493892B09F414606CE676E0CE010E9409
:105280005493892B09F4186069E676E0CE010E94F8
:105290005493892B09F4106163E676E0CE010E94F5
:1052A0005493892B09F4106268E576E0CE010E94E0
:1052B0005493892B09F0D2CE1064D0CE2D2D3E2DE3
:1052C000A8016B2D70E080E090E0DF91CF911F91FD
:1052D0000F91EF90DF90BF909F908F9008955F9215
:1052E0006F927F928F929F92AF92BF92CF92DF92F6
:1052F000EF92FF920F931F93CF93DF93782EC7E225
:10530000DBE100E010E0F2E5EF2EF6E0FF2E817029
:10531000582E872D8270682EADE3CA2EA6E0DA2EB5
:10532000B5E4AB2EB6E0BB2E83E4882E86E0982E43
:10533000772051F01F930F93FF92EF920E943394C6
:105340000F900F900F900F905520A1F089858F93AB
:1053500088858F93BF92AF920E9433940F900F90E5
:105360000F900F906620C1F09F928F920E9433940D
:105370000F900F90662081F0DF92CF920E943394BD
:10538000288139814A815B816C817D818E819F81F9
:105390000E9469240F900F900E94F20B0F5F1F4F25
:1053A0002A960430110521F6DF91CF911F910F91BC
:1053B000FF90EF90DF90CF90BF90AF909F908F9035
:1053C0007F906F905F90089588E396E09F938F930E
:1053D0000E94339480912D1C90912E1CA0912F1C23
:1053E000B091301C0F900F90813027EA92072EE188
:1053F000A207B10519F48AE296E01DC0823026EAC0
:1054000092072EE1A207B10519F48DE196E013C0D1
:10541000823027EA92072EE1A207B10519F48FE046
:1054200096E009C0823028EA92072EE1A207B10572
:1054300049F481E096E09F938F930E9433940F90FC
:105440000F900895BF93AF939F938F938BEF95E049
:105450009F938F930E9433940F900F900F900F9013
:105460000F900F9008958BEE95E09F938F930E947D
:1054700033940E94C6200E94E4290E94F20B8EE021
:105480009BE19F938F9383EE95E09F938F930E9470
:105490003394609152027091530280915402909122
:1054A000550228EE33E040E050E00E946A8D5F93A1
:1054B0004F933F932F9383ED95E09F938F930E949B
:1054C00033948AEC95E09F938F930E9433940E94CB
:1054D000721080913D202DB73EB7225F3F4F0FB62F
:1054E000F8943EBF0FBE2DBF80FF05C041E061E0D4
:1054F00081E00E941C1286EC95E09F938F930E949E
:10550000339480E00E94A4220E94CA208091570216
:105510001F928F938DEB95E09F938F930E9433940E
:105520008091C1091F928F9384EB95E09F938F9395
:105530000E943394809183028F93809182028F9393
:10554000809181028F93809180028F9386EA95E00B
:105550009F938F930E9433941F9280E48F938EE8E1
:1055600095E09F938F930E943394809113291F920B
:105570008F93809112291F928F938BE795E09F93D1
:105580008F930E943394809156021F928F9382E7EB
:1055900095E09F938F930E9433948091580290914D
:1055A0005902A0915A02B0915B022DB73EB7225E1C
:1055B0003F4F0FB6F8943EBF0FBE2DBF96FF03C0FE
:1055C0008EE895E002C081E995E09F938F9388E68D
:1055D00095E09F938F930E94339483E00E946F29FC
:1055E0000F900F900F900F901D9B03C08EE895E0D9
:1055F00002C081E995E09F938F938CE595E09F939E
:105600008F930E94339482E595E09F938F930E943D
:105610003394809158020F900F900F900F900F903D
:105620000F9081FF09C08CE495E09F938F930E94B7
:1056300033940F900F9013C080FF03C08EE895E065
:1056400002C081E995E09F938F9388E495E09F9352
:105650008F930E9433940F900F900F900F90809132
:10566000580290915902A0915A02B0915B0297FFA3
:1056700003C08EE895E002C081E995E09F938F9387
:105680008FE395E09F938F930E94339488E395E096
:105690009F938F930E9433946091C5097091C609BE
:1056A00080E090E00E94E0220E94F20B0F900F90A9
:1056B0000F900F900F900F90779903C08EE895E0B0
:1056C00002C081E995E09F938F938FE295E09F93CD
:1056D0008F930E9433940E9492090E943C0B9F93E7
:1056E0008F937F936F9381E295E09F938F930E94B6
:1056F00033940E94EB0A9F938F937F936F9383E180
:1057000095E09F938F930E94339481E090E00E94F4
:1057100080218091E8289091E928A091EA28B09111
:10572000EB28BF93AF939F938F9385E095E09F9372
:105730008F930E9433948091FD288F938091FC2851
:105740008F938091FB288F938091FA288F9381EF1C
:1057500094E09F938F930E9433948091EC289091D2
:10576000ED28A091EE28B091EF28BF93AF939F93BF
:105770008F9383EE94E09F938F930E9433948DB721
:105780009EB782960FB6F8949EBF0FBE8DBF8091D4
:1057900001298F93809100298F938091FF288F9307
:1057A0008091FE288F938FEC94E09F938F930E94BB
:1057B000339461E070E080E090E00E94FB0B61E0D8
:1057C00070E081E090E00E94FB0B0F900F900F9033
:1057D0000F900F900F90299B03C08EE895E002C0B8
:1057E00081E995E09F938F9387EC94E09F938F934B
:1057F0000E9433940F900F900F900F902A9B03C03C
:105800008EE895E002C081E995E09F938F938FEB3E
:1058100094E09F938F930E9433940F900F900F907A
:105820000F900895F894E0E0F0E081E28093570053
:105830008491E2E0F0E041E2409357004491E4E0DB
:10584000F0E091E290935700E49190E0A0E0B0E0A6
:10585000DC019927882750E060E070E0762F652F03
:10586000542F4427840F951FA61FB71F8E0F911D1D
:10587000A11DB11D80932D1C90932E1CA0932F1C55
:10588000B093301C78940895CF93DF93CDB7DEB7F3
:1058900061970FB6F894DEBF0FBECDBF48E250E06F
:1058A0006EE170E087E29BE10E9487952091271BC3
:1058B0003091281B4091291B50912A1B60912B1B72
:1058C00070912C1B80912D1B90912E1BAFEF0E948D
:1058D000A28F09F05DC08DE48093271B80E8809340
:1058E000281B84E08093291B10922A1B10922B1BEB
:1058F00010922C1B10922D1B10922E1B8CE390E00B
:105900009093301B80932F1B1092311B1092321BEF
:105910001092331B1092341B1092351B1092361BC1
:105920001092371B1092381B10923A1B1092391BA1
:1059300010923B1B10923C1B10923D1B10923E1B81
:1059400010923F1B1092401B1092411B1092421B61
:105950001092441B1092431B1092451B1092461B41
:105960001092471B1092481B1092491B10924A1B21
:1059700010924B1B10924C1B10924E1B10924D1B01
:1059800048E250E06EE170E087E29BE10E94A5955D
:1059900044E050E06AE170E0CE010B960E948795EA
:1059A0008B859C85AD85BE858F3F2FEF9207A20723
:1059B000B207A9F48AE090E4A0E0B0E08093580236
:1059C00090935902A0935A02B0935B0244E050E0D6
:1059D0006AE170E088E592E00E94A59508C0809396
:1059E000580290935902A0935A02B0935B0280919F
:1059F000580290915902A0915A02B0915B02A2FF05
:105A000002C02A9A03C080E00E94D42242E050E003
:105A100066E570E0CE010F960E9487958F85988984
:105A20008F3F2FEF920769F41092C6091092C509B3
:105A300042E050E066E570E085EC99E00E94A595B3
:105A400004C09093C6098093C50949E050E06AE01C
:105A500070E082E099E20E9487950E94330D44E055
:105A600050E06AE470E0CE010B960E9487958B852A
:105A70009C85AD85BE8544E050E06AE470E08F3FD0
:105A80009F4FAF4FBF4F29F488E792E00E94A59542
:105A900004C088E792E00E94879544E050E066E405
:105AA00070E0CE010B960E9487958B859C85AD8515
:105AB000BE8544E050E066E470E08F3F9F4FAF4FFB
:105AC000BF4F29F484E792E00E94A59504C084E7C3
:105AD00092E00E94879544E050E06EE470E0CE01D1
:105AE0000B960E9487958B859C85AD85BE8544E08D
:105AF00050E06EE470E08F3F9F4FAF4FBF4F29F4EF
:105B00008CE792E00E94A59504C08CE792E00E9489
:105B1000879541E050E069E170E0CE0141960E9436
:105B20008795898941E050E069E170E08F3F29F471
:105B300081EC99E00E94A59504C081EC99E00E9457
:105B4000879541E050E068E170E0CE0141960E9407
:105B50008795898941E050E068E170E08F3F29F442
:105B600087E592E00E94A59504C087E592E00E9437
:105B7000879541E050E067E170E0CE0141960E94D8
:105B80008795898941E050E067E170E08F3F29F413
:105B900086E592E00E94A59504C086E592E00E9409
:105BA00087954AE050E060E070E0CE0101960E94E7
:105BB000879589814AE050E060E070E08F3F29F4EA
:105BC0008EE09BE10E94A59504C08EE09BE10E94BF
:105BD000879544E050E062E570E0CE010B960E94AC
:105BE00087958B859C85AD85BE8544E050E062E558
:105BF00070E08F3F9F4FAF4FBF4F29F480E892E096
:105C00000E94A59504C080E892E00E94879544E038
:105C100050E063E170E0CE010B960E9487958B8582
:105C20009C85AD85BE8544E050E063E170E08F3F28
:105C30009F4FAF4FBF4F29F482E592E00E94A59598
:105C400004C082E592E00E94879561960FB6F894B1
:105C5000DEBF0FBECDBFDF91CF910895CF92DF920F
:105C6000EF92FF92609171027091720280E090E079
:105C70000E94689365E975E00E947C93892B09F086
:105C80001FC18DE48093271B80E88093281B84E04C
:105C90008093291B10922A1B10922B1B10922C1BF5
:105CA00010922D1B10922E1B8CE390E09093301BD2
:105CB00080932F1B1092311B1092321B1092331BBA
:105CC0001092341B1092351B1092361B1092371B0A
:105CD0001092381B10923A1B1092391B10923B1BEA
:105CE00010923C1B10923D1B10923E1B10923F1BCA
:105CF0001092401B1092411B1092421B1092441BA9
:105D00001092431B1092451B1092461B1092471B8A
:105D10001092481B1092491B10924A1B10924B1B69
:105D200010924C1B10924E1B10924D1B48E250E0FB
:105D30006EE170E087E29BE10E94A5958AE090E425
:105D4000A0E0B0E08093580290935902A0935A02C9
:105D5000B0935B0244E050E06AE170E088E592E0D5
:105D60000E94A5951092C6091092C50942E050E024
:105D700066E570E085EC99E00E94A59542E2C42EAC
:105D8000DD24DA944CECE42E4BE3F42EC09278023E
:105D9000D0927902E0927A02F0927B0244E050E0E5
:105DA0006AE470E088E792E00E94A595C0927402D0
:105DB000D0927502E0927602F092770244E050E0D1
:105DC00066E470E084E792E00E94A59587ED94E395
:105DD000AFEEBCE380937C0290937D02A0937E02A1
:105DE000B0937F0244E050E06EE470E08CE792E014
:105DF0000E94A5958AE999E9A9E1B0E4809380021F
:105E000090938102A0938202B093830244E050E019
:105E100062E570E080E892E00E94A5951092C109C9
:105E200080E00E94B36B41E050E069E170E081ECFA
:105E300099E00E94A5958AE1809357020E945A6AD0
:105E400041E050E068E170E087E592E00E94A595AE
:105E50008FE08093560241E050E067E170E086E514
:105E600092E00E94A5958AE0EEE0FBE1DF011D9241
:105E70008A95E9F74AE050E060E070E0CF010E94C7
:105E8000A59580EA96E8A1E0B0E080935202909355
:105E90005302A0935402B093550244E050E063E1F2
:105EA00070E082E592E00E94A59581E00E94A42224
:105EB00080E090E0FF90EF90DF90CF900C94470D42
:105EC000FF90EF90DF90CF9008952F923F924F92E6
:105ED0005F926F927F928F929F92AF92BF92CF927A
:105EE000DF92EF92FF920F931F93CF93DF93CDB783
:105EF000DEB72B970FB6F894DEBF0FBECDBF9B87E2
:105F00008A874A01FC0180819181892B11F00C94D0
:105F100074426091710270917202CA010E9468938A
:105F200060E870E0C4010E949B93009759F460916F
:105F3000CD317091CE318AE090E00E94EF9381E004
:105F40000C9479428130910561F4F401B0801B2DED
:105F5000110F110B012F412E512E612E712EA12EEA
:105F6000BCC082309105B9F4F4018081992787FD86
:105F70009095982F88272181820F911D27FD9A9552
:105F8000B82E192F092F000F000B402E502E602E17
:105F9000702EA02EA2C083309105B1F5F4012081AE
:105FA000922F990F990B392F492F592F692F792F3C
:105FB000892F00E10E94448F19012A013B01B82F6B
:105FC000A92F2181922F990F990B392F492F592FE2
:105FD000692F792F892F08E00E94448F59016A01A7
:105FE0007B018C019101A201B3018B2F9A2F0E949A
:105FF0007B8FA2801A2D110F110BB12EC12ED12E25
:10600000E12EF12E012F55C004970CF45DC0F40170
:106010002081922F990F990B392F492F592F692FD2
:10602000792F892F08E10E94448F19012A013B0131
:10603000B82FA92F2181922F990F990B392F492F12
:10604000592F692F792F892F00E10E94448F590120
:106050006A017B018C019101A201B3018B2F9A2F60
:106060000E947B8FA3801A2D110F110BB12EC12E10
:10607000D12EE12EF12E012F0E947B8F19012A01D2
:106080003B01B82FA92F2281922F990F990B392FFD
:10609000492F592F692F792F892F08E00E94448FAB
:1060A00059016A017B018C019101A201B3018B2F7F
:1060B0009A2F0E947B8FB22E132F042F452E562E1F
:1060C000672E782EA92E09C07AE0B72E10E000E0E6
:1060D000412C512C612C712CA12C0E94F20B2B2DE8
:1060E000312F402F542D652D762D872D9A2D253754
:1060F000F3E63F07FDE64F07510561057105810590
:10610000910511F40C945C3D2537E3E63E07EDE67E
:106110004E075105610571058105910511F008F0E3
:10612000AAC12337F2E73F07410551056105710513
:106130008105910511F40C94EF3F2337E2E73E0708
:1061400041055105610571058105910511F008F0C2
:10615000B2C02536F4E63F074105510561057105DA
:106160008105910509F4C8C62536E4E63E074105D8
:106170005105610571058105910509F0B8F5A6E79E
:106180000E94A28F11F40C94F3390E94A28F09F09F
:1061900068F4A8E60E94A28F09F4F4C6A5E70E945D
:1061A000A28F11F40C94DD390C9472422B2D312FF7
:1061B000402F542D652D762D872D9A2D2A33F6E20A
:1061C0003F0741055105610571058105910509F4F8
:1061D00033C32436314641055105610571058105FA
:1061E000910511F40C9417400C9472422B2D312F11
:1061F000402F542D652D762D872D9A2D2737FFE6BC
:106200003F0741055105610571058105910511F4AF
:106210000C94C23D2737EFE63E0741055105610565
:1062200071058105910509F0C8F42436F9E63F07A8
:1062300041055105610571058105910511F40C9425
:10624000B63925363E464105510561057105810582
:10625000910511F40C94F63D0C9472422B2D312FC4
:10626000402F542D652D762D872D9A2D2536F2E75A
:106270003F0741055105610571058105910511F43F
:106280000C94C03E2936E2E73E0741055105610501
:1062900071058105910511F40C949E3F233331471C
:1062A00041055105610571058105910511F00C94B9
:1062B00072420C9417402B2D312F402F542D652DF9
:1062C000762D872D9A2D2236E5E63E07E4E64E0729
:1062D0005105610571058105910509F40DC6223648
:1062E000F5E63F07F4E64F075105610571058105A5
:1062F000910511F008F054C02133E4E63E07E1E6D1
:106300004E075105610571058105910509F4A4C287
:106310002133F4E63F07F1E64F07510561057105AA
:106320008105910509F0C0F42337E3E73E074105F5
:106330005105610571058105910511F40C94034027
:1063400028373447410551056105710581059105DF
:1063500009F472C20C9472422B2D312F402F542D10
:10636000652D762D872D9A2D2336E4E63E07E1E64E
:106370004E075105610571058105910511F40C94D5
:10638000174028373446414651056105710581059E
:10639000910511F00C9472420E9400160C94744204
:1063A0002B2D312F402F542D652D762D872D9A2D95
:1063B0002D36E5E73E07E8E64E0751056105710514
:1063C0008105910511F40C942D402D36F5E73F071A
:1063D000F8E64F075105610571058105910509F042
:1063E000E0F42237E2E73E07E5E64E075105610596
:1063F00071058105910511F40C941B3D23363D4632
:1064000048465105610571058105910511F00C940F
:1064100072420E9478160C9474422B2D312F402F1B
:10642000542D652D762D872D9A2D2436E3E63E07D3
:10643000ECE64E075105610571058105910511F4E2
:106440000C947E3C2736FFE63F07FCE64F075105DC
:10645000610571058105910511F40C94813C233689
:10646000324349465105610571058105910511F0D9
:106470000C94724211C22B2D312F402F542D652DBB
:10648000762D872D9A2D2136FDE63F07F5E74F073C
:10649000F8E65F07610571058105910511F40C941B
:1064A000E03D2136EDE63E07E5E74E07E8E65E070C
:1064B000610571058105910511F008F0D9C02437F7
:1064C000F8E73F07F4E74F075105610571058105BE
:1064D000910509F4F4C72437E8E73E07E4E74E07DF
:1064E0005105610571058105910511F008F054C051
:1064F0002133F1E33F07F1E74F07510561057105CE
:106500008105910511F40C945C3D2133E1E33E07D4
:10651000E1E74E075105610571058105910509F017
:10652000C8F42233F2E63F07F0E74F075105610553
:1065300071058105910509F487C220333143414734
:106540005105610571058105910511F40C941B3D00
:106550000C9472422B2D312F402F542D652D762D0A
:10656000872D9A2D2037F5E63F07F2E74F075105B3
:10657000610571058105910511F40C94C03E2C361E
:10658000344744475105610571058105910511F4B2
:106590000C949B410C9472422B2D312F402F542D83
:1065A000652D762D872D9A2D2936FCE63F07F1E6DD
:1065B0004F07F3E65F07610571058105910509F451
:1065C000D9C22936ECE63E07E1E64E07E3E65E0770
:1065D000610571058105910509F0E0F42437F4E6C1
:1065E0003F07F7E74F0751056105710581059105E3
:1065F00011F40C94E94124373F464F465246610559
:1066000071058105910511F00C9472420C94000003
:106610000C9474422B2D312F402F542D652D762D47
:10662000872D9A2D2633F9E63F07F5E74F07F5E664
:106630005F07610571058105910509F4A7C420373D
:10664000ECE63E07E5E64E07E8E65E076105710504
:106650008105910509F496C42E36314648465346C5
:10666000610571058105910509F4FDC60C9472421E
:106670002B2D312F402F542D652D762D872D9A2DC2
:106680002437E3E73E07E5E64E07E2E75E076105EC
:1066900071058105910511F40C94703E2437F3E7E0
:1066A0003F07F5E64F07F2E75F07610571058105D2
:1066B000910511F008F055C02337E2E73E07E7E700
:1066C0004E07E0E75E07610571058105910511F44C
:1066D0000C94733E2337F2E73F07F7E74F07F0E7E5
:1066E0005F07610571058105910509F0C8F422373E
:1066F000E7E73E07E0E74E075E07610571058105A4
:10670000910509F406C223373546424750476105D3
:1067100071058105910511F40C94DD400C947242D1
:106720002B2D312F402F542D652D762D872D9A2D11
:106730002436EDE63E07E3E64E07E2E75E07610535
:1067400071058105910509F42CC521363C46454665
:106750005247610571058105910509F434C40C9413
:1067600072422B2D312F402F542D652D762D872DE4
:106770009A2D2437E2E73E07E1E64E07E5E75E079C
:10678000610571058105910509F466C52437F2E7B5
:106790003F07F1E64F07F5E75F07610571058105E2
:1067A000910509F0C8F42437E3E73E07E5E64E0714
:1067B000E4E75E07610571058105910509F4AAC644
:1067C00027373047484754476105710581059105D2
:1067D00009F41FC60C9472422B2D312F402F542DDB
:1067E000652D762D872D9A2D2F36ECE63E07EFE5A9
:1067F0004E07E6E75E07610571058105910509F41D
:106800007BC42C36F1E63F07F4E74F07F8E75F0754
:10681000610571058105910511F40C9465412237DC
:10682000374640475547610571058105910511F0CF
:106830000C9472420C94593C83E08093F02810929F
:10684000F2281092F12840EF58E262E184E392E0EE
:106850000E94BD550C94744221E042E161E080ED5C
:106860000E94F76221E042E161E080ED0E94F76260
:1068700021E042E161E080ED0E94F76221E042E127
:1068800061E080ED0E94F76221E042E161E080ED8D
:106890000E94F7620C9474426091710270917202CE
:1068A00080E090E00E9468936CE975E00E947C9320
:1068B000892B09F0C5C0609171027091720280E06D
:1068C00090E00E9468935C01009709F497C060EE25
:1068D00073E00E947C93892BE1F488EE93E0A0E0C2
:1068E000B0E08093520290935302A0935402B0936D
:1068F000550268EE73E080E090E00E941E6144E083
:1069000050E063E170E082E592E00E94A5950C946E
:10691000744262EA75E0C5010E947C93892BE1F420
:1069200080E197E2A0E0B0E080935202909353029E
:10693000A0935402B093550260E177E280E090E0CA
:106940000E941E6144E050E063E170E082E592E065
:106950000E94A5950C94744265EA75E0C5010E94F9
:106960007C93892BE1F480EA96E8A1E0B0E0809383
:10697000520290935302A0935402B093550260EADE
:1069800076E881E090E00E941E6144E050E063E11F
:1069900070E082E592E00E94A5950C94744269EA49
:1069A00075E0C5010E947C93892BE1F480E89AE1AF
:1069B000A6E0B0E08093520290935302A093540259
:1069C000B093550260E87AE186E090E00E941E6193
:1069D00044E050E063E170E082E592E00E94A5951A
:1069E0000C94744280E093E09F938F930E943394C1
:1069F0000E94F20B0F900F900C947442609152021F
:106A000070915302809154029091550228EE33E028
:106A100040E050E00E946A8D5F934F933F932F9325
:106A20008CEF92E09F938F930E9433940E94F20B1D
:106A30000F900F900F900F900F900F900C94744246
:106A40000E9472100C9474426091710270917202F3
:106A500080E090E00E9468938C016EE875E00E94EF
:106A60007C93892BE1F48091580290915902A09176
:106A70005A02B0915B02A46080935802909359022D
:106A8000A0935A02B0935B022A9A44E050E06AE174
:106A900070E088E592E00E94A5950C94744261E94B
:106AA00075E0C8010E947C93892BF1F48091580213
:106AB00090915902A0915A02B0915B02AB7F8093F2
:106AC000580290935902A0935A02B0935B0280E05F
:106AD0000E94D42244E050E06AE170E088E592E050
:106AE0000E94A5950C9474422A9B03C08EE895E001
:106AF00002C081E995E09F938F9384EF92E09F938A
:106B00008F930E9433940F900F900F900F900C94DE
:106B10007442609171027091720280E090E00E9474
:106B200068938C016EE875E00E947C93892B19F4C0
:106B300077980C94744261E975E0C8010E947C93D7
:106B4000892B19F4779A0C947442779903C08EE8D4
:106B500095E002C081E995E09F938F9389EA94E0E4
:106B60009F938F930E9433940F900F900F900F90EC
:106B70000C947442609171027091720280E090E016
:106B80000E9468938C0168E575E00E947C93892BD4
:106B900009F077C0609171027091720280E090E01C
:106BA0000E9468938C01009711F40C9474426DEA72
:106BB00075E00E947C93892BB1F482E29FEFACECEC
:106BC000BBE38093780290937902A0937A02B0930A
:106BD0007B0244E050E06AE470E088E792E00E94C3
:106BE000A5950C94744263EB75E0C8010E947C93F8
:106BF000892BB1F482E29FEFACECBAE38093780288
:106C000090937902A0937A02B0937B0244E050E023
:106C10006AE470E088E792E00E94A5950C947442C3
:106C2000C8010E9452922B013C0120E030E0A901F2
:106C30000E94ED898823D9F081E00E94880A9B0197
:106C4000AC01C301B2010E94F18960937802709394
:106C5000790280937A0290937B0244E050E06AE4E8
:106C600070E088E792E00E94A5950C94744287EE4C
:106C700092E09F938F930E9433940F900F900C9407
:106C800074426BE575E0C8010E947C93892B09F082
:106C900077C0609171027091720280E090E00E9472
:106CA00068938C01009711F40C9474426DEA75E0BE
:106CB0000E947C93892BB1F482E29FEFACECBBE3A2
:106CC0008093740290937502A0937602B09377023A
:106CD00044E050E066E470E084E792E00E94A5950D
:106CE0000C94744263EB75E0C8010E947C93892B7D
:106CF000B1F482E29FEFACECBAE38093740290931C
:106D00007502A0937602B093770244E050E066E407
:106D100070E084E792E00E94A5950C947442C8014B
:106D20000E9452922B013C0120E030E0A9010E9418
:106D3000ED898823D9F082E00E94880A9B01AC018A
:106D4000C301B2010E94F1896093740270937502CD
:106D5000809376029093770244E050E066E470E01E
:106D600084E792E00E94A5950C9474428AED92E02B
:106D70009F938F930E9433940F900F900C947442C2
:106D800063E575E0C8010E947C93892B09F073C00C
:106D9000609171027091720280E090E00E946893AD
:106DA0008C01009711F40C9474426DEA75E00E9416
:106DB0007C93892BB1F487ED94E3AFEEBCE3809331
:106DC0007C0290937D02A0937E02B0937F0244E008
:106DD00050E06EE470E08CE792E00E94A5950C9480
:106DE000744263EB75E0C8010E947C93892B51F4D7
:106DF0008BEC92E09F938F930E9433940F900F90AF
:106E00000C947442C8010E9452922B013C0120E074
:106E100030E0A9010E94ED89882319F180E00E94E9
:106E2000880A4B015C0121EE3AE744E95EE3C301C5
:106E3000B2010E942689A50194010E94F189609304
:106E40007C0270937D0280937E0290937F0244E0E7
:106E500050E06EE470E08CE792E00E94A5950C94FF
:106E600074428EEB92E09F938F930E9433940F9025
:106E70000F900C9474420E94D70A9F938F937F9334
:106E80006F9387EB92E09F938F930E94339482E0FD
:106E90000E94880A20917402309175024091760216
:106EA000509177020E94728C162F072FF82EE92E30
:106EB00081E00E94880AEF92FF920F931F93209126
:106EC00078023091790240917A0250917B020E94BF
:106ED000728C9F938F937F936F938BEA92E09F9333
:106EE0008F930E9433940E94F20B0FB6F894DEBF8A
:106EF0000FBECDBF0C94744260917102709172020A
:106F000080E090E00E9468930097C1F00E94CE2339
:106F10002091C5093091C6098217930709F1909312
:106F2000C6098093C50942E050E066E570E085EC53
:106F300099E00E94A59582EA94E002C08BE994E072
:106F40009F938F930E9433946091C5097091C609F5
:106F500080E090E00E94E0220E94F20B0F900F90E0
:106F600080E994E09F938F930E9433946FEF7FEFBB
:106F700080E090E00E94E0220E94F20B0F900F90C0
:106F80000C9474420E94CF1F0C947442F4018481CB
:106F9000843329F440E061E080E00E941C1280917B
:106FA0007302882311F40C9474421F928F938DE81E
:106FB00094E09F938F930E9433940F900F900F90C3
:106FC0000F900C947442F4018481893709F080C0D9
:106FD000609171027091720280E090E00E9468936B
:106FE0008C016EE875E00E947C93892B51F48091AE
:106FF000580290915902A0915A02B0915B0290649C
:1070000010C061E975E0C8010E947C93892BD1F41E
:107010008091580290915902A0915A02B0915B025E
:107020009F7B8093580290935902A0935A02B09389
:107030005B0244E050E06AE170E088E592E00E9483
:10704000A59546C068EB75E0C8010E947C93892B2A
:1070500021F58091261B8F938091251B8F93809122
:10706000241B8F938091231B8F938091221B8F93DE
:107070008091211B8F938091201B8F9380911F1BE8
:107080008F9380E892E09F938F930E9433940FB682
:10709000F894DEBF0FBECDBF1BC080915802909107
:1070A0005902A0915A02B0915B0296FF03C08EE88C
:1070B00095E002C081E995E09F938F938CE792E081
:1070C0009F938F930E9433940F900F900F900F9087
:1070D00080917302882311F40C9474421F928F9351
:1070E0008AE894E09F938F930E9433940F900F90BF
:1070F0000F900F900C947442F40184818737E9F566
:10710000609171027091720280E090E00E94689339
:107110000097D9F00E9452922B013C0120E030E010
:10712000A9010E94ED89882381F04092800250924B
:107130008102609282027092830244E050E062E534
:1071400070E080E892E00E94A595809183028F9381
:10715000809182028F93809181028F93809180022F
:107160008F938EE692E09F938F930E9433940F90BB
:107170000F900F900F900F900F90809173028823C3
:1071800011F40C9474421F928F9387E894E09F93BC
:107190008F930E9433940F900F900F900F900C9448
:1071A0007442609171027091720280E090E00E94DE
:1071B00068938C016EE875E00E947C9340905802C1
:1071C0005090590260905A0270905B02892B19F41A
:1071D000689457F809C061E975E0C8010E947C9382
:1071E000892B99F4E89457F840925802509259022A
:1071F00060925A0270925B0244E050E06AE170E0F3
:1072000088E592E00E94A59513C057FE03C08EE862
:1072100095E002C081E995E09F938F938AE692E022
:107220009F938F930E9433940F900F900F900F9025
:1072300080917302882311F40C9474421F928F93EF
:1072400084E894E09F938F930E9433940F900F9063
:107250000F900F900C9474426091710270917202C1
:1072600080E090E00E9468935C016EEB75E00E9404
:107270007C93892B11F489E108C062EC75E0C501AB
:107280000E947C93892B49F480E18093C400109282
:10729000C50082E08093C00055C066EC75E0C50172
:1072A0000E947C93892B11F488E0EFCF6BEC75E0A2
:1072B000C5010E947C93892B39F060ED75E0C50112
:1072C0000E947C93892B11F483E0DFCF8091C4006E
:1072D000893141F485E692E09F938F930E94339425
:1072E0000F900F908091C400803141F480E692E0CD
:1072F0009F938F930E9433940F900F908091C400BE
:10730000883041F48AE592E09F938F930E943394F2
:107310000F900F908091C400833041F484E592E097
:107320009F938F930E9433940F900F908091C4008D
:10733000883041F48EE492E09F938F930E943394BF
:107340000F900F9080917302882311F40C94744273
:107350001F928F9381E894E09F938F930E943394C0
:107360000F900F900F900F900C94744260917102E7
:107370007091720280E090E00E9468936DEA75E07F
:107380000E947C93892B11F481E001C080E00E946F
:10739000A42280917302882311F40C9474421F92EA
:1073A0008F938EE794E09F938F930E9433940F9076
:1073B0000F900F900F900C9474420E94CA208091FD
:1073C0007302882311F40C9474421F928F938BE7FD
:1073D00094E09F938F930E9433940F900F900F909F
:1073E0000F900C9474420E94C620809173028823EF
:1073F00011F40C9474421F928F9388E794E09F934A
:107400008F930E9433940F900F900F900F900C94D5
:107410007442609171027091720280E090E00E946B
:1074200068930E945692803170F48093C1090E9443
:10743000B36B41E050E069E170E081EC99E00E94BB
:10744000A5950C9474428091C1091F928F9384E496
:1074500092E09F938F930E9433940F900F900F9020
:107460000F900C947442609171027091720280E0EE
:1074700090E00E9468930E94569295EF980F903189
:1074800070F4809357020E945A6A41E050E068E12C
:1074900070E087E592E00E94A5950C94744280917B
:1074A00057021F928F938BE392E09F938F930E94DA
:1074B00033940F900F900F900F900C947442609142
:1074C00071027091720280E090E00E9468930097D0
:1074D00089F04AE050E0BC018EE09BE10E948C9371
:1074E0004AE050E060E070E08EE09BE10E94A595EC
:1074F0000C9474428EE09BE19F938F9385ED95E011
:107500009F938F930E9421940F900F900F900F9054
:107510000C947442609171027091720280E090E06C
:107520000E9468935C0160EE73E00E947C93892B5B
:10753000D9F4219A8091580290915902A0915A024F
:10754000B0915B0280618093580290935902A0939E
:107550005A02B0935B0244E050E06AE170E088E5D3
:1075600092E00E94A595C0C76CE575E0C5010E9438
:107570007C93892BD9F4229A8091580290915902D8
:10758000A0915A02B0915B0280628093580290935E
:107590005902A0935A02B0935B0244E050E06AE1C2
:1075A00070E088E592E00E94A5959EC762EC73E0CA
:1075B000C5010E947C93892BD9F4239A80915802AB
:1075C00090915902A0915A02B0915B02806480931D
:1075D000580290935902A0935A02B0935B0244E080
:1075E00050E06AE170E088E592E00E94A5957CC7D2
:1075F0006FEF74E0C5010E947C93892BD9F4239A24
:107600008091580290915902A0915A02B0915B0268
:1076100080688093580290935902A0935A02B093C5
:107620005B0244E050E06AE170E088E592E00E948D
:10763000A5955AC76CE679E0C5010E947C93892B19
:1076400071F581E08093542487E29BE19093562466
:1076500080935524109258241092572480915802F8
:1076600090915902A0915A02B0915B02916080936F
:10767000580290935902A0935A02B0935B0244E0DF
:1076800050E06AE170E088E592E00E94A59544E54B
:1076900054E262E184E392E00E94BD5525C769EEA1
:1076A00073E0C5010E947C93892B11F5E7E5FBE1AE
:1076B000119211922BE1E737F207D1F7809158022E
:1076C00090915902A0915A02B0915B02926080930E
:1076D000580290935902A0935A02B0935B0244E07F
:1076E00050E06AE170E088E592E00E94A595FCC652
:1076F00061E975E0C5010E947C9340915802509168
:10770000590260915A0270915B02892BC1F44F704B
:107710005C7F409358025093590260935A027093D1
:107720005B022B9A44E050E06AE170E088E592E069
:107730000E94A5958091F9280E946F6AD5C644FFE2
:1077400003C08EE895E002C081E995E09F938F9396
:1077500080E392E09F938F930E943394809158022C
:107760000F900F900F900F9085FF03C08EE895E06B
:1077700002C081E995E09F938F9385E292E09F9309
:107780008F930E943394809158020F900F900F9026
:107790000F9086FF03C08EE895E002C081E995E076
:1077A0009F938F938AE192E09F938F930E943394EB
:1077B000809158020F900F900F900F9087FF03C099
:1077C0008EE895E002C081E995E09F938F938FE06A
:1077D00092E09F938F930E943394809158029091EE
:1077E0005902A0915A02B0915B020F900F900F9036
:1077F0000F9090FF03C08EE895E002C081E995E00C
:107800009F938F9384E092E09F938F930E94339491
:107810008091580290915902A0915A02B0915B0256
:107820000F900F900F900F9091FF03C08EE895E09E
:1078300002C081E995E09F938F9389EF91E09F9338
:107840008F930E9433948091580290915902A09195
:107850005A02B0915B020F900F900F900F9091FF22
:1078600043C68DED95E00E94579457E5A52E5BE148
:10787000B52E0BE010E065EE862E65E0962EF50144
:1078800080819181F2E0AF0EB11C9F938F931F9383
:107890000F939F928F920E9421940F5F1F4F0F9022
:1078A0000F900F900F900F900F900B31110539F73B
:1078B0001BC684E794E09F938F930E94339480913A
:1078C00073020F900F90882361F01F928F9381E7CE
:1078D00094E09F938F930E9433940F900F900F909A
:1078E0000F90F89428E088E190E00FB6F894A895FE
:1078F000809360000FBE20936000FFCF0E94A862BB
:10790000F3C5609171027091720280E090E00E9474
:1079100068938C016EE875E00E947C93892BE9F4F2
:107920000E945B698091580290915902A0915A027D
:10793000B0915B028D7F81608093580290935902D1
:10794000A0935A02B0935B0244E050E06AE170E019
:1079500088E592E00E94A595C7C561E975E0C80178
:107960000E947C93892BE1F40E9413698091580254
:1079700090915902A0915A02B0915B028C7F809342
:10798000580290935902A0935A02B0935B0244E0CC
:1079900050E06AE170E088E592E00E94A595A4C5F8
:1079A00060EF75E0C8010E947C93892BE9F40E9486
:1079B00013698091580290915902A0915A02B09196
:1079C0005B028E7F82608093580290935902A0934D
:1079D0005A02B0935B0244E050E06AE170E088E54F
:1079E00092E00E94A59580C58091580281FF0FC04A
:1079F00080EF95E09F938F9385EF91E09F938F9316
:107A00000E9433940F900F900F900F906DC580FFE0
:107A100003C08EE895E002C081E995E09F938F93C3
:107A200081EF91E09F938F930E9433940F900F907A
:107A30000F900F9059C5809152248F9380915124BB
:107A40008F93809150248F9380914F248F938091B6
:107A50004E248F9380914D248F9380914C248F934B
:107A600080914B248F9380914A248F938091492455
:107A70008F93809148248F93809147248F938EE435
:107A800094E09F938F930E943394809173020FB67A
:107A9000F894DEBF0FBECDBF882309F425C51F9221
:107AA0008F938BE494E09F938F930E9433940F9075
:107AB0000F900F900F9018C5F89481E090E029E0A6
:107AC000FC0120935700C895E02C80E090E0FC0179
:107AD00020935700C895F02C7894F89483E090E0B8
:107AE000FC0120935700C895002D82E090E0FC0136
:107AF00020935700C895102D78948091301C8F9357
:107B000080912F1C8F9380912E1C8F9380912D1C20
:107B10008F9321E434E03F932F930E9433941F927C
:107B2000EF921F92FF921F920F931F921F938AE171
:107B300094E09F938F930E9433940E9464218091DC
:107B400066001F928F938EE094E09F938F930E9424
:107B500033940E94F20B809173020FB6F894DEBF4B
:107B60000FBECDBF882309F4BFC41F928F938BE053
:107B700094E09F938F930E9433940F900F900F90F7
:107B80000F90B2C460E070E080E090E00E94FB0BD8
:107B900060E070E081E090E00E94FB0B8091730256
:107BA000882309F4A1C41F928F9388E094E09F93E7
:107BB0008F930E9433940F900F900F900F9094C466
:107BC0000E94921F0E94F20B80917302882309F495
:107BD0008BC41F928F9385E094E09F938F930E94B4
:107BE00033940F900F900F900F907EC460917102AC
:107BF0007091720280E090E00E94689365EF75E0FA
:107C00000E947C93892B31F5F8948CEF99E00E94C7
:107C1000AA565C01009769F0C5010F960E94AE5903
:107C2000B50184E092E00E946456C5010E9452575B
:107C3000F0CF8CEF99E00E943757892B29F08CEF19
:107C400099E00E94E356F5CF8CEF99E00E94A6568A
:107C5000789434C08CEF99E00E94AA565C010BEF37
:107C600015E0A114B10451F1F50186811F928F93A3
:107C700080851F928F9385811F928F9381851F929C
:107C80008F9387811F928F9384811F928F9383811B
:107C90001F928F9382811F928F9382851F928F9361
:107CA0001F930F930E942194C5010E9452575C01BB
:107CB0000FB6F894DEBF0FBECDBFD3CF8091730255
:107CC000882309F411C41F928F9382E094E09F935C
:107CD0008F930E9433940F900F900F900F9004C4D5
:107CE0000E942E2E01C4609171027091720280E098
:107CF00090E00E9468938C016AE376E00E947C9396
:107D0000892BD1F48091580290915902A0915A0286
:107D1000B0915B02977F8093580290935902A09391
:107D20005A02B0935B0244E050E06AE170E088E5FB
:107D300092E00E94A595D8C363EB75E0C8010E944C
:107D40007C93892BD1F48091580290915902A09193
:107D50005A02B0915B029860809358029093590246
:107D6000A0935A02B0935B0244E050E06AE170E0F5
:107D700088E592E00E94A595B7C30E949209B4C31A
:107D8000609171027091720280E090E00E946893AD
:107D9000FC0120812332B1F44AE050E060E070E061
:107DA00001960E940A901B0160917102709172020B
:107DB00080E090E00E946893F4E02F1631040CF00C
:107DC00094C002C0212C312C009709F48EC0198276
:107DD000BE016F5F7F4F0E94CD2729013A014B0101
:107DE000B82FA92F8AE0829DF001839DF00D112408
:107DF000E95DF44E20812A8331813B8382818C832B
:107E000093819D8324812E8335813F83868188875A
:107E1000978199879201A301B4018B2F9A2FAA8091
:107E2000BB80CC80DD80EE80FF80088519850E94B4
:107E3000998F09F45DC08981882351F18CF02A81E2
:107E4000422A3B81532A8C81682A9D81792A2E817E
:107E5000822A3F81932A8885B82B9985A92B18C03F
:107E6000409450946094709480949094B095A095B0
:107E70002A8142223B8153228C8168229D81792272
:107E80002E8182223F8193228885B8239985A92358
:107E9000408251826282738284829582B683A783F4
:107EA00048E250E06EE170E087E29BE10E94A59518
:107EB0008AEF93E09F938F930E9433948AE0829D90
:107EC000F001839DF00D1124E95DF44E2081318194
:107ED0004281538164817581868197810E946924E2
:107EE0000E94F20B0F900F9003C082E00E946F2956
:107EF0008EEE93E09F938F930E9433942FEF3FEF8A
:107F00004FEF5FEF6FEF7FEF8FEF9FEF0E946924DE
:107F10000E94F20B809173020F900F90882309F456
:107F2000E3C21F928F938BEE93E09F938F930E94F7
:107F300033940F900F900F900F90D6C26091710202
:107F40007091720280E090E00E946893FC012081B1
:107F50002332A1F44AE050E060E070E001960E9414
:107F60000A908B01609171027091720280E090E042
:107F70000E94689304301105ECF402C000E010E0A8
:107F80000097C1F04AE050E060E070E00E943E914E
:107F90002AE0209FF001219FF00D1124E95DF44EAD
:107FA0007187608748E250E06EE170E087E29BE114
:107FB0000E94A59581E00E946F2980917302882319
:107FC00009F492C21F928F9388EE93E09F938F9350
:107FD0000E9433940F900F900F900F9085C20E94D3
:107FE000E75980917302882309F47EC21F928F9310
:107FF00085EE93E09F938F930E9433940F900F90A0
:108000000F900F9071C20E94332A809173028823CF
:1080100009F46AC21F928F9382EE93E09F938F932D
:108020000E9433940F900F900F900F905DC280E0EC
:1080300090E00E94802180917302882309F454C249
:108040001F928F938FED93E09F938F930E943394B1
:108050000F900F900F900F9047C280913D2081FFAD
:108060002DC00E94161F892B49F58091341C8F93D7
:108070008091331C8F938091321C8F938091311C9F
:108080008F9384ED93E09F938F930E94339480911C
:1080900011298F93809110298F9380910F298F93AD
:1080A00080910E298F9387EC93E09F938F930E948A
:1080B00033940FB6F894DEBF0FBECDBF0E94F20B13
:1080C00080913D2090913E2090FF63C081E090E040
:1080D0000E948D1E3B014C0180E090E00E948D1EAD
:1080E0001B012C010E94EB1D9F928F927F926F9239
:1080F00086EB93E09F938F930E9433945F924F920D
:108100003F922F9286EA93E09F938F930E9433943D
:10811000222D332D442D552D662D772D882D992D0B
:108120000E948E1C9F938F937F936F938BE993E0B4
:108130009F938F930E943394222D332D442D552DE0
:10814000662D772D882D992D0E94EF1C9F938F937C
:108150007F936F938DE893E09F938F930E94339466
:10816000222D332D442D552D662D772D882D992DBB
:108170000E94501D9F938F937F936F938AE793E0A4
:108180009F938F930E9433940FB6F894DEBF0FBE77
:10819000CDBF0E94F20B80917302882309F4A4C121
:1081A0001F928F9387E793E09F938F930E9433945E
:1081B0000F900F900F900F9097C180913D2082FFFC
:1081C0002BC021E048E061E083E00E9491138091A0
:1081D0002B1C8F9380912A1C8F938091291C8F9345
:1081E0008091281C8F938091271C8F938091261C4F
:1081F0008F938091251C8F938091241C8F9380E610
:1082000093E09F938F930E9433940E94F20B0FB6DA
:10821000F894DEBF0FBECDBF80913D2090913E20EF
:1082200091FF41C00E94DB17B62EA72E982E892EF3
:1082300020E030E048EC52E4D501F4016B2F7A2FB6
:108240008F2F9E2F0E94728C20E836EE45EC57E46B
:108250000E94F18921E03EED42E45EE30E94D58C6C
:108260009B01AC0160E070E080E89FE30E942689FA
:108270002BE43AE34DEB57E30E94F1899F938F93F0
:108280007F936F938F929F92AF92BF9287E493E018
:108290009F938F930E9433940E94F20B0FB6F89431
:1082A000DEBF0FBECDBF80917302882309F41CC1CD
:1082B0001F928F9384E493E09F938F930E94339453
:1082C0000F900F900F900F900FC1609171027091FD
:1082D000720280E090E00E9468936FE376E00E9473
:1082E0007C93892BB1F4609171027091720280E0ED
:1082F00090E00E946893009709F4F6C00E9456929D
:10830000803108F0F1C090915201982B9093520166
:10831000EBC0809152018F701F928F9384EE91E099
:108320009F938F930E9433940E94F20B0F900F90B3
:108330000F900F90D9C0609171027091720280E02D
:1083400090E00E946893009711F14AE050E060E0ED
:1083500070E00E940A90603198F4609356021F9278
:108360006F9387E393E09F938F930E94339441E050
:1083700050E067E170E086E592E00E94A59511C0AB
:10838000809156021F928F938EE293E006C08091F7
:1083900056021F928F9385E293E09F938F930E94E2
:1083A00033940F900F900F900F900E94F20B8091DA
:1083B0007302882309F498C01F928F9382E293E09E
:1083C0009F938F930E9433940F900F900F900F9074
:1083D0008BC0609171027091720280E090E00E9407
:1083E00068938C016EE875E00E947C93892BE1F420
:1083F0000E94C4678091580290915902A0915A023C
:10840000B0915B0290618093580290935902A093BF
:108410005A02B0935B0244E050E06AE170E088E504
:1084200092E00E94A59560C061E975E0C8010E94D4
:108430007C93892B81F5F8940E94D26788E10FB66E
:10844000F89480936000109260000FBE84B7877F1D
:1084500084BF80916000886180936000109260000A
:1084600078948091580290915902A0915A02B0914B
:108470005B029F7E8093580290935902A0935A0208
:10848000B0935B0244E050E06AE170E088E592E07E
:108490000E94A59529C064E476E0C8010E947C93FF
:1084A000409158025091590260915A0270915B02BA
:1084B000892B21F454FF18C0F894FFCF54FF03C058
:1084C0008EE895E002C081E995E09F938F9380EE5E
:1084D00091E09F938F930E9433940F900F900F9091
:1084E0000F9002C00E94B61FEA85FB8511821082A0
:1084F00083E02B960FB6F894DEBF0FBECDBFDF91A1
:10850000CF911F910F91FF90EF90DF90CF90BF9090
:10851000AF909F908F907F906F905F904F903F9023
:108520002F9008950F931F93CF93DF93EC018A014F
:1085300088819981009711F1853C904121F0198241
:10854000188283E020C06231E9F4A80162E170E0A2
:108550008DEE99E00E94652F84E08093F0281092C0
:10856000F2281092F1281093F4280093F32840EF9A
:1085700058E262E184E392E00E94BD5585EC90E10F
:108580009983888381E0DF91CF911F910F910895A6
:108590000E94B8676C9A6B9A6A9A6F9A729A749AE8
:1085A000739A779A809880B3897F80BB83988498E8
:1085B00087E080937E00549A0E94122C0E94442CE3
:1085C00081E00E94FC0980E090E00E94470D6091EC
:1085D00052027091530280915402909155020E9470
:1085E0001E610E94EB0A60933F24709340248093A5
:1085F0004124909342248091580286FD239A219A27
:10860000229A239A1D9B05C01092C3091092C20999
:10861000089581E090E09093C3098093C209089582
:10862000CF93DF93EC0188819981009741F0803BE3
:10863000904109F48CC01982188283E093C00E9493
:10864000C8428091580280FD05C081FF01C01D9B7A
:108650000E941369809170008C7F809370008091DC
:10866000B60080628093B6001092B20082E08093E0
:10867000B1008091B6008770E1F780917000816051
:108680008093700060EB79E080E090E00E94A26748
:108690000E94C62080E00E94A4228FE69FE09F9364
:1086A0008F930E9433940E94721080913D200F900E
:1086B0000F9086FD0E94546280913D2090913E2053
:1086C00090FD0E94A71D80913D2087FF06C021E0FC
:1086D0004CE061E080ED0E94F7628091C1090E9448
:1086E000B36B809157020E945A6A0E94576A809326
:1086F000EC09809157020E945A6A8091C1091F9229
:108700008F938091EC091F928F9389E496E09F9359
:108710008F930E9421941092EE091092ED090F9010
:108720000F900F900F900F900F9088E492E090932D
:108730000C2980930B2983E290E09093FF118093A2
:10874000FE1180EB90E19983888381E00BC0633256
:10875000E1F748E654E260E070E08DEE99E00E94B7
:10876000652FE3CFDF91CF9108958436910514F101
:108770009F938F938BE596E09F938F930E94219414
:108780008091472490914824A0914924B0914A2493
:108790000196A11DB11D8093472490934824A09376
:1087A0004924B0934A240F900F900F900F9081E0CE
:1087B00090E0089580E090E008952F923F924F92CC
:1087C0005F926F927F928F929F92AF92BF92CF9261
:1087D000DF92EF92FF920F931F93CF93DF93CDB76A
:1087E000DEB7C859D1090FB6F894DEBF0FBECDBFB2
:1087F000C057DF4F99838883C059D0408A016338BE
:1088000071F481EF99E0C856DF4F6883C859D040B2
:108810000E940054C856DF4F6881C859D040C057E5
:10882000DF4FA881B981C059D0402D913C912D35A1
:10883000B0E13B0709F4D3C340F42115310581F0C1
:1088400029393E4009F411C405C42F3640E13407EC
:1088500009F4E1C32637304111F40C940851FAC3EE
:108860004AEE52E061E870E081EF99E00E94E65341
:1088700089E99EE0ABC3E3E0F0E0EC0FFD1FE20FFF
:10888000F31F1082C9010E94B543892B89F720E0AC
:1088900030E040E050E0C357DF4F6881CD58D04012
:1088A000627070E080E090E0A0E00E94A28F09F08A
:1088B0008EC6C557DF4F2881CB58D040287030E096
:1088C00040E050E060E070E080E090E0A0E00E94D6
:1088D000A28FA1F127E04AE250E06BE270E089E26A
:1088E00090E00E94385E82E099E20E94A660BC019E
:1088F000882777FD8095982F0E94908A20E030E0AD
:1089000048EC52E40E94F1899F938F937F936F9379
:108910008FE896E09F938F931F9287E78F93CE0106
:108920008E0D9F1D03969F938F930E948494E80E53
:10893000F91E0FB6F894DEBF0FBECDBFC557DF4F8F
:108940002881CB58D040207130E040E050E060E01A
:1089500070E080E090E0A0E00E94A28FF1F126E0BC
:108960004AE250E06BE270E089E290E00E94385EFB
:1089700081E090E00E94800B8093C00980E89BE139
:108980000E94A660BC01882777FD8095982F0E94E1
:10899000908A20E030E048EC52E40E94F1899F93F5
:1089A0008F937F936F9389E996E09F938F931F92A4
:1089B00087E78F93C7010296E1E0F0E0EC0FFD1F1F
:1089C0008E0F9F1F9F938F930E948494E80EF91E31
:1089D0000FB6F894DEBF0FBECDBF272D30E040E0CC
:1089E00050E060E070E080E090E0A0E00E94A28FA4
:1089F00001F10E943C0B9F938F937F936F9384EAC6
:108A000096E09F938F931F9287E78F93C7010296FB
:108A100041E050E04C0F5D1F840F951F9F938F9393
:108A20000E948494E80EF91E0FB6F894DEBF0FBEC4
:108A3000CDBFC557DF4F2881CB58D040207430E0E0
:108A400040E050E060E070E080E090E0A0E00E9454
:108A5000A28F31F1809142248F93809141248F9392
:108A6000809140248F9380913F248F9382EB96E0F6
:108A70009F938F931F9287E78F93C7010296A1E080
:108A8000B0E0AC0FBD1F8A0F9B1F9F938F930E9476
:108A90008494E80EF91E0FB6F894DEBF0FBECDBF6A
:108AA000C557DF4F2881CB58D040207830E040E0D8
:108AB00050E060E070E080E090E0A0E00E94A28FD3
:108AC00041F1F8948091E8289091E928A091EA2852
:108AD000B091EB287894BF93AF939F938F9380ECE2
:108AE00096E09F938F931F9287E78F93C70102961B
:108AF00021E030E02C0F3D1F820F931F9F938F9337
:108B00000E948494E80EF91E0FB6F894DEBF0FBEE3
:108B1000CDBF20E0C457DF4F3881CC58D0403170F2
:108B200040E050E060E070E080E090E0A0E00E9473
:108B3000A28F09F05EC520E0C457DF4F3881CC58C2
:108B4000D040327040E050E060E070E080E090E0C3
:108B5000A0E00E94A28F09F0BFC520E0C457DF4FFC
:108B60003881CC58D040347040E050E060E070E094
:108B700080E090E0A0E00E94A28F09F0DEC520E036
:108B8000C457DF4F3881CC58D040387040E050E0B7
:108B900060E070E080E090E0A0E00E94A28F09F029
:108BA000FBC520E0C457DF4F3881CC58D04030712E
:108BB00040E050E060E070E080E090E0A0E00E94E3
:108BC000A28F09F05CC620E0C457DF4F3881CC5833
:108BD000D040307240E050E060E070E080E090E033
:108BE000A0E00E94A28F09F07AC620E030E040E0C9
:108BF00050E0C357DF4F6881CD58D040647070E0BB
:108C000080E090E0A0E00E94A28F09F096C620E0EC
:108C1000CB56DF4F3881C559D04040E050E060E08E
:108C200070E080E090E0A0E00E94A28F09F0F2C620
:108C300020E0CA56DF4F3881C659D04040E050E0AE
:108C400060E070E080E090E0A0E00E94A28F09F078
:108C50000FC7502F5170D52E20E030E0452F50E047
:108C600060E070E080E090E0A0E00E94A28F09F058
:108C70002DC720E030E0402F427050E060E070E00F
:108C800080E090E0A0E00E94A28F09F052C720E0AF
:108C900030E0C657DF4F4881CA58D04050E060E00E
:108CA00070E080E090E0A0E00E94A28F09F074C71D
:108CB00020E030E0402F487050E060E070E080E05D
:108CC00090E0A0E00E94A28F09F090C720E030E081
:108CD000402F407150E060E070E080E090E0A0E064
:108CE0000E94A28F09F0B2C720E030E0402F40720E
:108CF00050E060E070E080E090E0A0E00E94A28F91
:108D000009F0D4C720E030E0402F407450E060E02C
:108D100070E080E090E0A0E00E94A28F11F00C943F
:108D2000874EF02FF078AF2E20E030E04F2F50E04C
:108D300060E070E080E090E0A0E00E94A28F11F07F
:108D40000C94BA4E212F2170B22E20E030E040E08A
:108D50005B2D60E070E080E090E0A0E00E94A28FD8
:108D600011F00C94C74E20E030E04A2D50E060E056
:108D700070E080E090E0A0E00E94A28F11F00C94DF
:108D8000D54E20E030E040E05B2D60E070E080E018
:108D900090E0A0E00E94A28F11F00C940A4F20E016
:108DA00030E040E0512F527060E070E080E090E0F1
:108DB000A0E00E94A28F11F00C943F4F20E030E021
:108DC00040E0512F547060E070E080E090E0A0E05F
:108DD0000E94A28F11F00C94724F20E030E040E02E
:108DE000512F507160E070E080E090E0A0E00E94C0
:108DF000A28F11F00C94A54F20E030E040E0512FFD
:108E0000507260E070E080E090E0A0E00E94A28FED
:108E100011F00C94E44F20E030E040E0512F50740A
:108E200060E070E080E090E0A0E00E94A28F11F08E
:108E30000C94235020E030E040E0512F587060E067
:108E400070E080E090E0A0E00E94A28F11F00C940E
:108E5000625020E030E040E05C2D60E070E080E0B7
:108E600090E0A0E00E94A28F11F00C94935020E0BB
:108E700030E04D2D50E060E070E080E090E0A0E058
:108E8000FE0133966F010E94A28F11F00C94CF5017
:108E9000C557DF4F2881CB58D040C457DF4F3881AA
:108EA000CC58D040A801C357DF4F6881CD58D0407F
:108EB000CE56DF4F7881C259D040CD56DF4F8881E2
:108EC000C359D040CC56DF4F9881C459D040A0E060
:108ED0000E94A28F11F00C94D650809156028061AE
:108EE00089838091E5098A83F601EE0DFF1D1082CA
:108EF0008091C5099091C60987010D5F1F4F80FFC2
:108F00000CC01F930F9387E598E09F938F930E9467
:108F100021940F900F900F900F90B801CE01019601
:108F20000E942F5D8091580282FF0AC028EE34E231
:108F3000A801BE016F5F7F4F81E692E00E94C4618D
:108F40008091C5099091C60982FD73980E945B6962
:108F500081EF99E00E940254809158029091590249
:108F6000A0915A02B0915B0290FF40C0FFEFEF1A50
:108F7000FF0A0E94576AD82E89E10E946F6A4091C9
:108F800058025091590260915A0270915B0250FF51
:108F900029C073988091E5098F5F8093E5098A83E2
:108FA000B7016F5F7F4FCE0101960E942F5D81EF69
:108FB00099E00E94025440E050E065E8809102127E
:108FC000909103120E94BD558DE590E1C057DF4F8F
:108FD000A881B981C059D0408D939C9338C0E12CB1
:108FE000F12CCDCF8D2D0E946F6A739A8091C209AA
:108FF0009091C309892B11F00E9413698091E509B2
:109000008F5F8093E5098091C5099091C60982FF21
:109010002FCC739A2DCC8DED99E00E946358892B4B
:10902000B1F00E945B698091580287FD2B9860E443
:1090300070E08DED99E00E943C5886E790E1C057C2
:10904000DF4FE881F981C059D0409183808381E06E
:109050000C941B51C057DF4FA881B981C059D04033
:109060001D921C9283E00C941B51623181F7C090D9
:109070005802D0905902E0905A02F0905B02D1FC65
:10908000F7CBF8018081813091F50180F281E02DEC
:109090002081C557DF4F2883CB58D0403181C4573A
:1090A000DF4F3883CC58D040028113814481C357AD
:1090B000DF4F4883CD58D0405581CE56DF4F58837F
:1090C000C259D0408681CD56DF4F8883C359D040E6
:1090D0009781CC56DF4F9883C459D0402084318487
:1090E000C257DF4F19821882CE58D0406AC08230F2
:1090F000E9F4A381B481C257DF4FB983A883CE5866
:10910000D040212C312CB1E0C557DF4FB883CB586C
:10911000D040C457DF4F1882CC58D04000E010E850
:10912000C357DF4F1882CD58D0403CC08330F9F090
:10913000843009F09DCB212C312CC257DF4F19828E
:109140001882CE58D040E5E0C557DF4FE883CB58B2
:10915000D040C457DF4F1882CC58D04000E010E018
:10916000F2E0C357DF4FF883CD58D0401BC0212C0D
:10917000312CC257DF4F19821882CE58D04025E0DB
:10918000C557DF4F2883CB58D040C457DF4F1882D4
:10919000CC58D04000E010E031E0C357DF4F3883B7
:1091A000CD58D040CE56DF4F1882C259D040CD5650
:1091B000DF4F1882C359D040CC56DF4F1882C459B4
:1091C000D04080903F2490904024A0904124B090C3
:1091D0004224409080025090810260908202709000
:1091E00083022DEC3CEC4CE45EE3C301B2010E942F
:1091F00027899B01AC01C501B4010E94B38B87FD97
:109200000BC0E894E0F8C0925802D0925902E09264
:109210005A02F0925B024AC0A3019201C501B40157
:109220000E94ED8987FF42C080914B2490914C248D
:10923000A0914D24B0914E240196A11DB11D8093A3
:109240004B2490934C24A0934D24B0934E24E0FCE7
:109250000FCB6894E0F8C0925802D0925902E09285
:109260005A02F0925B0245E4C557DF4F4883CB5862
:10927000D04050E2C457DF4F5883CC58D04000E074
:1092800010E084E0C357DF4F8883CD58D040CE56DE
:10929000DF4F1882C259D040CD56DF4F1882C359D4
:1092A000D040CC56DF4F1882C459D040902F9470D4
:1092B000C657DF4F9883CA58D04020E030E0492F8E
:1092C00050E060E070E080E090E0A0E00E94A28FBB
:1092D00009F08C9AC557DF4FA881CB58D040A072B7
:1092E0007A2E2A2F30E040E050E060E070E080E02D
:1092F00090E0A0E00E94A28F11F00E943C0BC457A6
:10930000DF4FB881CC58D040B074CB56DF4FB88314
:10931000C559D04020E03B2F40E050E060E070E0D5
:1093200080E090E0A0E00E94A28F11F00E94161F42
:10933000C457DF4FE881CC58D040E078CA56DF4FA1
:10934000E883C659D04020E03E2F40E050E060E086
:1093500070E080E090E0A0E00E94A28F51F00E94B7
:10936000D70A6093F5287093F6288093F728909396
:10937000F828C557DF4F2881CB58D040217030E006
:1093800040E050E060E070E080E090E0A0E00E940B
:10939000A28FF1F08EE09BE19F938F938FE696E092
:1093A0009F938F931F9287E78F93CE0103969F938E
:1093B0008F930E9484946C010E94B5430FB6F89479
:1093C000DEBF0FBECDBF892B09F052CA760102C0A5
:1093D000E12CF12CC557DF4F2881CB58D0402270AB
:1093E00030E040E050E060E070E080E090E0A0E03D
:1093F0000E94A28FD1F1C701029667E776E041E0B3
:1094000050E04C0F5D1F840F951F0E94859353E021
:10941000E50EF11C22E0A22E29E2B22E32EFC32E7D
:1094200033E0D32E47E7942ED5018D915D011F9235
:109430008F93DF92CF921F929F92C7010296E1E035
:10944000F0E0EC0FFD1F8E0F9F1F9F938F930E94E4
:109450008494E80EF91E0FB6F894DEBF0FBECDBFA0
:109460003AE0A31639E2B306F9F6C557DF4F288173
:10947000CB58D040247030E040E050E060E070E035
:1094800080E090E0A0E00E94A28F09F447C0C701ED
:1094900002966BE776E041E050E04C0F5D1F840FD1
:1094A000951F0E94859354E0E50EF11C4E018AE75A
:1094B000880E911C80E1D4011D928A95E9F728E07D
:1094C000A40168E980EB0E94D5115401B8E0AB0E0D
:1094D000B11C82EFC82E83E0D82E97E7692EF401E5
:1094E00081914F011F928F93DF92CF921F926F92C3
:1094F000C701029621E030E02C0F3D1F820F931F21
:109500009F938F930E948494E80EF91E0FB6F894EF
:10951000DEBF0FBECDBF8A149B0409F7512F5078D0
:10952000C52E20E030E040E060E070E080E090E0B8
:10953000A0E00E94A28FE1F48091C2099091C3093A
:109540009F938F9380E896E09F938F931F9287E776
:109550008F93CE018E0D9F1D03969F938F930E9434
:109560008494E80EF91E0FB6F894DEBF0FBECDBF8F
:1095700020E030E040E050E0C357DF4F6881CD5835
:10958000D040617070E080E090E0A0E00E94A28F87
:1095900009F47DC9E3E0F0E0EC0FFD1FEE0DFF1DC7
:1095A00080E28083EBE6F4E2808197012F5F3F4FFA
:1095B0007901882309F45FC98081A1E0B0E0AC0F94
:1095C000BD1FAE0DBF1D12968C933196EDCFCE010F
:1095D0008E0D9F1D67E876E003960E94859397E0C5
:1095E000E90EF11CC7010E94B543892B09F040C95F
:1095F00060C92114310409F49ECAF8944090E82807
:109600005090E9286090EA287090EB287894809137
:10961000781B9091791BA0917A1BB0917B1BA301C1
:109620009201281B390B4A0B5B0BCA01B9010E943E
:109630008E8A4B015C01B10180E090E00E948E8A2D
:109640009B01AC01C501B4010E94F189B82ED92E4D
:109650009F938F937F936F938BEC96E09F938F9361
:109660001F9287E78F939E012E0D3F1D2D5F3F4F69
:109670003F932F93C856DF4F6883C859D040C956CF
:10968000DF4F7883C759D0400E948494E80EF91EBA
:10969000C856DF4F6881C859D040C956DF4F78811E
:1096A000C759D040862F972FAB2DBD2D8093FA2818
:1096B0009093FB28A093FC28B093FD284092781B40
:1096C0005092791B60927A1B70927B1B0FB6F894B4
:1096D000DEBF0FBECDBF2FCA2114310409F43DCA2D
:1096E000F89480914F1B9091501BA091511BB09109
:1096F000521B78949F938F9380915F028F938091F8
:109700005E028F9388ED96E09F938F931F9287E779
:109710008F93C7010296A1E0B0E0AC0FBD1F8A0F86
:109720009B1F9F938F930E948494E80EF91E0FB69F
:10973000F894DEBF0FBECDBF10CAF8948091EC281C
:109740009091ED28A091EE28B091EF287894BF93E6
:10975000AF939F938F9388EE96E09F938F931F9282
:1097600087E78F93C701029621E030E02C0F3D1F61
:10977000820F931F9F938F930E948494E80EF91E8B
:10978000C7010E94B5430FB6F894DEBF0FBECDBF30
:10979000892B09F06DC8F3C92114310409F401CAF9
:1097A000F8944090EC285090ED286090EE2870904E
:1097B000EF28789480917C1B90917D1BA0917E1B5B
:1097C000B0917F1BA3019201281B390B4A0B5B0B45
:1097D000CA01B9010E948E8A4B015C01B10180E08F
:1097E00090E00E948E8A9B01AC01C501B4010E94E9
:1097F000F189B82ED92E9F938F937F936F9383EF28
:1098000096E09F938F931F9287E78F939E012E0D73
:109810003F1D2D5F3F4F3F932F93C856DF4F688307
:10982000C859D040C956DF4F7883C759D0400E94ED
:109830008494E80EF91EC856DF4F6881C859D0409D
:10984000C956DF4F7881C759D040862F972FAB2D4F
:10985000BD2D8093FE289093FF28A0930029B093FC
:10986000012940927C1B50927D1B60927E1B70925E
:109870007F1B0FB6F894DEBF0FBECDBF92C9232861
:1098800009F4A1C9F8948091531B9091541BA091A5
:10989000551BB091561B78949F938F9380915D02D6
:1098A0008F9380915C028F9380E097E09F938F93DA
:1098B0001F9287E78F93C7010296A1E0B0E0AC0F3B
:1098C000BD1F8A0F9B1F9F938F930E948494E80E65
:1098D000F91E0FB6F894DEBF0FBECDBF74C98091DC
:1098E000432490914424A0914524B0914624BF93F1
:1098F000AF939F938F9380E197E09F938F931F92F5
:1099000087E78F93C701029621E030E02C0F3D1FBF
:10991000820F931F9F938F930E948494E80EF91EE9
:10992000C7010E94B5430FB6F894DEBF0FBECDBF8E
:10993000892B11F00C94384458C980914E248F9390
:1099400080914D248F9380914C248F9380914B2450
:109950008F9380914A248F93809149248F93809193
:1099600048248F93809147248F938BE197E09F93B6
:109970008F931F92B7E7DB2EDF92C7010296A1E01B
:10998000B0E0AC0FBD1F8A0F9B1F9F938F930E9467
:109990008494E80EF91EC7010E94B5430FB6F894EF
:1099A000DEBF0FBECDBF892B11F00C9438448091DF
:1099B0003D2090913E2090FF2AC9809152248F93A0
:1099C000809151248F93809150248F9380914F24C4
:1099D0008F938FE397E09F938F931F92DF92C7013E
:1099E000029621E030E02C0F3D1F820F931F9F93C2
:1099F0008F930E948494E80EF91EC7010E94B5431C
:109A00000FB6F894DEBF0FBECDBF892B11F00C94BA
:109A10003844FDC88091341C8F938091331C8F9300
:109A20008091321C8F938091311C8F9381E597E058
:109A30009F938F931F9287E78F93C7010296A1E0B0
:109A4000B0E0AC0FBD1F8A0F9B1F9F938F930E94A6
:109A50008494E80EF91EC7010E94B5430FB6F8942E
:109A6000DEBF0FBECDBF892B11F00C943844E0C887
:109A70008091F8288F938091F7288F938091F62812
:109A80008F938091F5288F938CE597E09F938F9328
:109A90001F9287E78F93C701029621E030E02C0FD9
:109AA0003D1F820F931F9F938F930E948494E80E13
:109AB000F91EC7010E94B5430FB6F894DEBF0FBE72
:109AC000CDBF892B11F00C943844C3C881E00E94AB
:109AD000880A209178023091790240917A0250915F
:109AE0007B020E94728C9F938F937F936F9389E682
:109AF00097E09F938F931F9287E78F93C7010296FA
:109B0000A1E0B0E0AC0FBD1F8A0F9B1F9F938F9306
:109B10000E948494E80EF91EC7010E94B5430FB657
:109B2000F894DEBF0FBECDBF892B11F00C943844E2
:109B3000A0C882E00E94880A2091740230917502C8
:109B400040917602509177020E94728C9F938F937E
:109B50007F936F9386E797E09F938F931F9287E79A
:109B60008F93C701029621E030E02C0F3D1F820F3A
:109B7000931F9F938F930E948494E80EF91EC70150
:109B80000E94B5430FB6F894DEBF0FBECDBF892B40
:109B900011F00C9438447BC883E00E94880A9F939C
:109BA0008F937F936F9383E897E09F938F931F9298
:109BB00087E78F93C7010296A1E0B0E0AC0FBD1F0D
:109BC0008A0F9B1F9F938F930E948494E80EF91E27
:109BD0008C98C7010E94B5430FB6F894DEBF0FBE44
:109BE000CDBF892B11F00C94384462C880913D2080
:109BF00087FF6CC821E042E161E080ED0E94F762DE
:109C00009F938F937F936F9380E997E09F938F93B8
:109C10001F9287E78F93C701029621E030E02C0F57
:109C20003D1F820F931F9F938F930E948494E80E91
:109C3000F91EC7010E94B5430FB6F894DEBF0FBEF0
:109C4000CDBF892B11F00C94384440C880913D2041
:109C500087FF4AC821E042E162E080ED0E94F7629E
:109C60009F938F937F936F938EE997E09F938F934A
:109C70001F9287E78F93C7010296A1E0B0E0AC0F77
:109C8000BD1F8A0F9B1F9F938F930E948494E80EA1
:109C9000F91EC7010E94B5430FB6F894DEBF0FBE90
:109CA000CDBF892B11F00C9438441EC880913D2003
:109CB00087FF28C821E042E163E080ED0E94F7625F
:109CC0009F938F937F936F938CEA97E09F938F93EB
:109CD0001F9287E78F93C701029621E030E02C0F97
:109CE0003D1F820F931F9F938F930E948494E80ED1
:109CF000F91EC7010E94B5430FB6F894DEBF0FBE30
:109D0000CDBF892B11F00C9438440C94824680917D
:109D10003D2087FD02C00C94914621E042E164E0C1
:109D200080ED0E94F7629F938F937F936F938AEBEE
:109D300097E09F938F931F9287E78F93C7010296B7
:109D4000A1E0B0E0AC0FBD1F8A0F9B1F9F938F93C4
:109D50000E948494E80EF91EC7010E94B5430FB615
:109D6000F894DEBF0FBECDBF892B11F00C943844A0
:109D70000C94914680913D2082FD02C00C94A24635
:109D800046E061E083E00E9491130C94A24680912A
:109D90003D2082FD02C00C94B34621E046E061E024
:109DA00083E00E9491130C94B34680913D2082FD84
:109DB00002C00C94C1468091271C8F938091261C71
:109DC0008F938091251C8F938091241C8F9388EC16
:109DD00097E09F938F931F9287E78F93C701029617
:109DE00041E050E04C0F5D1F840F951F9F938F93B0
:109DF0000E948494E80EF91EC7010E94B5430FB675
:109E0000F894DEBF0FBECDBF892B11F00C943844FF
:109E10000C94C14680913D2082FD02C00C94CF4637
:109E200080912B1C8F9380912A1C8F938091291CE9
:109E30008F938091281C8F9380ED97E09F938F9351
:109E40001F9287E78F93C7010296E1E0F0E0EC0FE5
:109E5000FD1F8E0F9F1F9F938F930E948494E80E87
:109E6000F91EC7010E94B5430FB6F894DEBF0FBEBE
:109E7000CDBF892B11F00C9438440C94CF468091BF
:109E80003D2090913E2090FD02C00C94DE4680E083
:109E900090E00E948D1E9F938F937F936F938BED25
:109EA00097E09F938F931F9287E78F93C701029646
:109EB00041E050E04C0F5D1F840F951F9F938F93DF
:109EC0000E948494E80EF91EC7010E94B5430FB6A4
:109ED000F894DEBF0FBECDBF892B11F00C9438442F
:109EE0000C94DE4680913D2090913E2090FD02C072
:109EF0000C94ED4681E090E00E948D1E9F938F931D
:109F00007F936F938BEE97E09F938F931F9287E7DA
:109F10008F93C7010296E1E0F0E0EC0FFD1F8E0F7A
:109F20009F1F9F938F930E948494E80EF91EC70190
:109F30000E94B5430FB6F894DEBF0FBECDBF892B8C
:109F400011F00C9438440C94ED4680913D20909192
:109F50003E2090FD02C00C94FC4681E090E00E94FF
:109F60008D1E4B015C0180E090E00E948D1E9B01E4
:109F7000AC01C501B4010E948E1C9F938F937F9307
:109F80006F938CEF97E09F938F931F9287E78F9348
:109F9000C701029641E050E04C0F5D1F840F951FF2
:109FA0009F938F930E948494E80EF91EC7010E942C
:109FB000B5430FB6F894DEBF0FBECDBF892B11F0AD
:109FC0000C9438440C94FC4680913D2090913E20A6
:109FD00090FD02C00C940B4781E090E00E948D1E22
:109FE0004B015C0180E090E00E948D1E9B01AC0162
:109FF000C501B4010E94EF1C9F938F937F936F93D1
:10A0000087E098E09F938F931F9287E78F93C70114
:10A010000296E1E0F0E0EC0FFD1F8E0F9F1F9F9373
:10A020008F930E948494E80EF91EC7010E94B543E5
:10A030000FB6F894DEBF0FBECDBF892B11F00C9484
:10A0400038440C940B4780913D2090913E2090FD28
:10A0500002C00C941A4781E090E00E948D1E4B01D3
:10A060005C0180E090E00E948D1E9B01AC01C50167
:10A07000B4010E94501D9F938F937F936F9385E14E
:10A0800098E09F938F931F9287E78F93C701029663
:10A0900041E050E04C0F5D1F840F951F9F938F93FD
:10A0A0000E948494E80EF91EC7010E94B5430FB6C2
:10A0B000F894DEBF0FBECDBF892B11F00C9438444D
:10A0C0000C941A4780913D2090913E2091FD02C052
:10A0D0000C9429470E94DB179F938F937F936F9374
:10A0E00088E298E09F938F931F9287E78F93C70131
:10A0F0000296E1E0F0E0EC0FFD1F8E0F9F1F9F9393
:10A100008F930E948494E80EF91EC7010E94B54304
:10A110000FB6F894DEBF0FBECDBF892B11F00C94A3
:10A1200038440C942947C257DF4FA881B981CE58D3
:10A13000D04016968C9116971F928F9315968C91FE
:10A1400015971F928F9313968C9113971F928F934D
:10A1500012968C911F928F9389E398E09F938F932F
:10A160001F9287E78F93C7010296E1E0F0E0EC0FC2
:10A17000FD1F8E0F9F1F9F938F930E948494E80E64
:10A18000F91EC7010E94B5430FB6F894DEBF0FBE9B
:10A19000CDBF892B11F00C9438440C943747779A33
:10A1A0008091C5099091C60992FD749A8091C50964
:10A1B0009091C60982FD0CC08091580280FD08C0B4
:10A1C00081FD02C00C946D471D9902C00C946D472F
:10A1D000DF92CF9280E598E09F938F930E94219425
:10A1E000809173020F900F900F900F90882311F4BD
:10A1F0000C946D471F928F938CE69FE09F938F93F3
:10A200000E9433940F900F900F900F900C946D4715
:10A210008DED99E00E946358892B11F40C94274826
:10A220000E9413698091580287FD02C00C94384443
:10A230002B9A0C943844C856DF4F0FB6F894DEBF03
:10A240000FBECDBFDF91CF911F910F91FF90EF9087
:10A25000DF90CF90BF90AF909F908F907F906F9046
:10A260005F904F903F902F9008950C9429544F92F7
:10A270005F926F927F928F929F92AF92BF92CF9296
:10A28000DF92EF92FF920F931F93CF93DF93CDB79F
:10A29000DEB760970FB6F894DEBF0FBECDBF6B017F
:10A2A0000E94576AE82FF0E0EE0FFF1FEF5BF44EBD
:10A2B000808191810196918380838091C5099091DD
:10A2C000C60981FD74988090580290905902A09020
:10A2D0005A02B0905B020E94835C7C01FC01808189
:10A2E000982F92959F70913099F48F7051F48091CE
:10A2F000251B9091261B01969093261B8093251B6E
:10A3000007C1B60182E199E20E949F53892B51F067
:10A310008091231B9091241B01969093241B809382
:10A32000231BF6C0D501C4011EE0B695A7959795ED
:10A3300087951A95D1F7F82FF1708F2E8CEF99E051
:10A340000E94AA568C01009709F448C0B601C801C2
:10A3500002960E949F53892BE9F198014AEC59E03B
:10A3600060E074E6C8010F960E942A59F7019181B6
:10A37000F8018481981321C082858F5F8287809144
:10A38000211B9091221B01969093221B8093211BED
:10A3900084E00E94A05DF801208530E0281739078D
:10A3A00008F0A9C184E00E94A05DF8018087F70150
:10A3B00080818F70F8018187ABC0F801128684E03C
:10A3C0000E94A05DF8018087F70180818F70F801FD
:10A3D000818792C1C8010E945257B4CF84E092E0B5
:10A3E0000E943F568C01009709F492C0B601C80143
:10A3F00002960E949653F70181818150F80184836F
:10A4000080E091E0A0E0B0E083879487A587B687DD
:10A41000128684E00E94A05DF8018087F7018081A8
:10A420008F70F8018187B8018CEF99E00E940A577C
:10A4300098014AEC59E060E074E6C8010F960E946A
:10A440002A5999249394F7018181F8018483F701B3
:10A4500080818F70F801878384E00E94A05DF801FD
:10A46000858383E00E94A05D5C01F801868387817B
:10A470008F3009F0912CF7014180F8018481481A4E
:10A48000512C612C712C76E0440C551C661C771CF9
:10A490007A95D1F72385348545855685A0ECB0E0C3
:10A4A0000E94D68DBB27A92F982F872F480E591EA3
:10A4B0006A1E7B1E43865486658676868091C50912
:10A4C0009091C60981FD2EC08091580280FD2AC05E
:10A4D00081FD26C08091580290915902A0915A02A4
:10A4E000B0915B0297FDD2C0992091F082E08093F9
:10A4F00054241092562410925524109358240093FB
:10A50000572444E554E262E184E392E00E94BD55A1
:10A510008091C5099091C60981FFF0C0749AEEC080
:10A520001D9BD8CFA4E6B0E0A30192010E94D68D76
:10A53000672F782F892F992724E630E040E050E0FC
:10A540000E946A8D7F936F93452C562C672C77243D
:10A550005F924F92BB24BF92AF92F80185811F9208
:10A560008F93F70180818F701F928F9381811F924B
:10A570008F93F60181811F928F9380811F928F9319
:10A58000C70102969F938F9388E698E09F938F93DD
:10A590000E942194809173020FB6F894DEBF0FBE23
:10A5A000CDBF882361F01F928F9389E69FE09F9330
:10A5B0008F930E9433940F900F900F900F90809183
:10A5C000580290915902A0915A02B0915B0296FFF5
:10A5D0002DC0882059F1F7012081322F3F70832F41
:10A5E00090E00297D4F08FEF830F207F822B80833F
:10A5F00081EF99E00E94355180911F1B9091201BA3
:10A6000001969093201B80931F1B8091C509909108
:10A61000C60996FF0BC0739809C08091251B9091C5
:10A62000261B01969093261B8093251B80913D202D
:10A6300086FF50CF0E944662C70105960E941262B3
:10A64000F70181811F928F93F80186811F928F936A
:10A6500085811F928F938CEA98E09F938F931F922E
:10A6600080E18F939E012F5F3F4F6901DF922F930F
:10A670000E94849482E00E942C62C6010E941262B1
:10A680000FB6F894DEBF0FBECDBF24CF8EE09BE1A6
:10A6900020910E1B222309F427CF9F938F938FEBDA
:10A6A00098E09F938F93FE0131966F01DF92EF93B5
:10A6B0000E94C1945C01B601C70102960E94A69354
:10A6C0000F900F900F900F900F900F90009709F43C
:10A6D0000BCF95012F5F3F4F280F391FA9012F5F27
:10A6E0003F4FFA0180818032C9F362E18CE092E051
:10A6F0000E94BD55F9CE812C912CA5CE60960FB647
:10A70000F894DEBF0FBECDBFDF91CF911F910F91A7
:10A71000FF90EF90DF90CF90BF90AF909F908F9081
:10A720007F906F905F904F9008950895FB01208176
:10A73000FC012083FB012181FC0121830895FC01A0
:10A740009081DB018C91981309C081E090E0318108
:10A7500011962C91321721F080E0089580E090E06E
:10A760000895BC0182E199E20C949653DC0119969C
:10A77000ED91FC911A970280F381E02D309709F05A
:10A78000099408950F931F93CF93DF9300D0CDB713
:10A79000DEB78C0188E10E94B35DBC01CE01019659
:10A7A0000E949653D8011996ED91FC911A97019049
:10A7B000F081E02DBE016F5F7F4FC80109950F90BA
:10A7C0000F90DF91CF911F910F910895EF92FF921B
:10A7D0000F931F93CF93DF93EC018B017A0142E03B
:10A7E00053E00E940F54FA86E98666E073E0C801E0
:10A7F000DF91CF911F910F91FF90EF900C946854CF
:10A800000C942754CF93DF93EC0162E179E288E165
:10A810000E94A95DCE01DF91CF910C942954EF9253
:10A82000FF920F931F93CF93DF93EC018B017A017B
:10A830000E944454F886EF826AE073E0C801DF9119
:10A84000CF911F910F91FF90EF900C9468540C944E
:10A850004C540C94D16EDC011796ED91FC91189735
:10A860000190F081E02D0994DC011796ED91FC91A7
:10A8700018970280F381E02D309709F0099408952C
:10A8800080E092E10C94A656FC0173836283BC01C4
:10A8900080E092E10C940A57BC0180E092E10C94B4
:10A8A000EF56CF93DF93EC0180E092E10E94AA562D
:10A8B000009749F0FC01228133812C173D0729F0D4
:10A8C0000E945257F5CF80E090E0DF91CF9108953C
:10A8D0000F931F93CF93DF938B010E945154EC0190
:10A8E000009731F01D830C83C8010E9402718E8392
:10A8F000DF91CF911F910F9108951F93CF93DF9315
:10A90000EC01162FEC81FD813097D1F0909303126A
:10A910008093021282E08887CE01069609959927D6
:10A9200087FD90950297029710F0133839F4BE0115
:10A93000CE01DF91CF911F910C94AA5481E08887BA
:10A94000DF91CF911F910895FC01208520FD0C948B
:10A950007D540895CF92DF92EF92FF920F931F9351
:10A96000CF93DF93EC016B01E0900212F0900312A1
:10A970000091041210910512F801EC17FD0739F04F
:10A98000309709F44AC00190F081E02DF6CF20976E
:10A9900009F443C08885882309F11886011511053B
:10A9A00061F0C017D10729F0AE0167E8C8010E9425
:10A9B000A454F80100811181F1CFEC81FD81309721
:10A9C00069F0CC15DD0551F0D0930312C09302124B
:10A9D00040E050E063E8CE0106960995E09104124C
:10A9E000F0910512CE17DF0769F488819981909361
:10A9F0000512809304120DC0808191818C179D07F0
:10AA000021F0FC013097C1F704C0888199819183BE
:10AA10008083F0920312E0920212DF91CF911F9196
:10AA20000F91FF90EF90DF90CF9008951F93CF93F9
:10AA3000DF9310920E12C0910412D091051211E012
:10AA4000209779F08985882341F01887198640E09E
:10AA500050E062E8CE010E947D540990D881C02D5B
:10AA6000EFCFDF91CF911F9108958091B11291E0C6
:10AA7000980F9093B1120895609102127091031291
:10AA80000C94AA548AE88093B1121092AF121092DB
:10AA9000B01210920512109204121092031210922A
:10AAA0000212089580910E1281110E941655709124
:10AAB000B012772309F451C0E091AF122E2F30E08D
:10AAC00085E0E89FF0011124E15FFD4E6081609315
:10AAD0000D124181528150930C1240930B128381CD
:10AAE000948190930A12809309122F5F3F4F2F7128
:10AAF00033272093AF1271507093B012009731F545
:10AB0000809104129091051290930812809307127D
:10AB10008091071290910812892BF9F080910E1202
:10AB200081110E94165540910B1250910C126091A8
:10AB30000D1280910712909108120E94A454E09186
:10AB40000712F091081280819181DECF613819F4EB
:10AB500021E0FC0120870E94A45480910E122091D4
:10AB6000B01290E0820F911D089580910E122091F5
:10AB7000B01290E0820F911D08952091B012203202
:10AB8000B9F0E091AF12E20FEF71E093061235E0F9
:10AB9000E39FF0011124E15FFD4E60835283418306
:10ABA000948383832F5F2093B01280E090E0089518
:10ABB00081E090E00895CF93DF93C0910212D0918D
:10ABC00003120E94A454D0930312C0930212DF9187
:10ABD000CF910895AB013091041220910512E32F1B
:10ABE000F22FE817F907B1F0309721F00190F081CA
:10ABF000E02DF7CF009771F0FC0130832183909313
:10AC000005128093041221E020871782168261E8E2
:10AC10000C94DB550895009749F0FC0120852150E4
:10AC2000223020F421E0218720930E12089521E0A4
:10AC300030E0FC018085811102C020E030E0C901D4
:10AC40000895CF93DF93EC014A815B8160E070E06F
:10AC50008C819D810E9475932A813B818881998195
:10AC6000289FA001299F500D389F500D112460E0AE
:10AC700070E08E819F81DF91CF910C947593FC01E0
:10AC80008281938120E030E028173907D1F0A48138
:10AC9000B581A20FB31F4C91411110C081E08C937C
:10ACA00080819181289FA001299F500D389F500DD0
:10ACB000112486819781840F951F08952F5F3F4F40
:10ACC000E3CF80E090E00895FC0126813781428146
:10ACD000538180E090E084179507C9F02617370765
:10ACE00081F4A481B581A80FB91F2C91121614F418
:10ACF00021502C930480F581E02DE80FF91F80810D
:10AD00000895A081B1812A0F3B1F0196E4CF8FEFF8
:10AD10000895FC018681978168177907A0F0A081CA
:10AD2000B18142815381A49F9001A59F300DB49FB2
:10AD3000300D1124280F391F81E090E0621773074E
:10AD400020F080E0089580E090E00895FC011182F9
:10AD500010820895FC01808191810895FB0120817A
:10AD60003181FC01318320830895DC01ED91FC9158
:10AD7000309731F080819181009729F0FC01FACF62
:10AD800080E090E00895CF010895DC01ED91FC9101
:10AD900011973097A9F020813181232B21F41D9246
:10ADA0001C92CF010895A081B1818D919C91119742
:10ADB000892B11F0FD01F7CF11821082CD0108958A
:10ADC00080E090E00895DC01ED91FC9111973097BF
:10ADD00021F0208131812D933C93CF010895DC0136
:10ADE000ED91FC913097A9F0A0E0B0E02081318195
:10ADF000E617F70741F4109709F4DC012D933C9313
:10AE00001182108208952115310519F0DF01F90131
:10AE1000EDCF08950F931F93CF93DF938C01EB0138
:10AE20000E94EF5619821882C8010E94B5560097F9
:10AE300011F4F80101C0FC01D183C083DF91CF91EF
:10AE40001F910F9108950F931F93CF93DF93EC0100
:10AE50008B010E94EF5688819981F801918380834C
:10AE600019830883DF91CF911F910F910895DC0121
:10AE7000ED91FC9180E090E0309729F001960190EF
:10AE8000F081E02DF9CF0895FB01309719F4BA0154
:10AE90000C94235780819181DA018D939C93518387
:10AEA00040830895009721F0FC01808191810895ED
:10AEB00080E090E008958091B4129091B512892BB2
:10AEC00029F41092B3121092B21208950E945E6695
:10AED000E091B412F091B512228133814081518109
:10AEE000240F351F281B390B0480F581E02D309786
:10AEF00069F04281538160817181460F571F481B61
:10AF0000590B4217530780F79A01EECF280F391FCC
:10AF10003093B3122093B212089586E892E00C9415
:10AF20000B56EF92FF920F931F93CF93DF938C01F9
:10AF3000FC0180819181009799F08A359105D9F0C3
:10AF4000F8011182108283E068C08681978184179E
:10AF5000950709F049C00480F581E02D3097A9F7E5
:10AF60001092B5121092B4128AE590E0F801918324
:10AF7000808381E052C0673891F16238A9F7C091AF
:10AF8000B412D091B512E12CF12C209769F3CE01C7
:10AF90000E94D374892BF1F0AE0168E88E819F8105
:10AFA0000E94BD55892BA1F41F821E828C819D8138
:10AFB000E114F10421F0F7019583848304C0909398
:10AFC000B5128093B4121D821C820E945B57D7CFAA
:10AFD0000E948D577E010C80DD81C02DD6CFE0917F
:10AFE000B412F091B512BACFF093B512E093B41247
:10AFF000A481B581109709F4B7CF16968D919C91D5
:10B0000017978417950711F0FD01F2CF14968D91D3
:10B010009C91159795838483EBCFDF91CF911F91FE
:10B020000F91FF90EF900895CF93DF93EC010E9472
:10B030008D578E819F813091B4122091B512892B4A
:10B0400059F0E32FF22F309739F0EC17FD0781F01C
:10B050000480F581E02DF7CF8091021290910312C8
:10B060009F838E833C832D83D093B512C093B412FB
:10B07000DF91CF910C945B57CF93DF93EC010E944B
:10B08000B374CE01DF91CF910C941458CF93DF931A
:10B09000EC010E94BF74CE01DF91CF910C94145843
:10B0A000CF93DF93EC010E94C974CE01DF91CF9161
:10B0B0000C941458FC0120813181260F371F3183F5
:10B0C00020830C945B5721E030E0FC01868197815E
:10B0D000892B11F020E030E0C9010895FC012281A4
:10B0E000338180819181820F931F0895FC018081BB
:10B0F0009181089581E090E02091B4123091B512D1
:10B10000232B11F480E090E008958091B412909187
:10B11000B512892B29F08091B2129091B312089543
:10B1200080E090E00895CF93DF93EC01E091B412BA
:10B13000F091B5128E179F0769F48C819D819093D1
:10B14000B5128093B4120DC0848195818C179D0730
:10B1500021F0FC013097C1F706C08C819D81958359
:10B1600084830E945B571D821C821F821E82DF9196
:10B17000CF910895EF92FF920F931F93CF93DF9398
:10B180008C017A01FC0180819181009741F08B3420
:10B19000910501F1F8011182108283E048C087EB2C
:10B1A00092E10E94AA56EC01209751F06C817D81BA
:10B1B000CE0102960E943C580990D881C02DF4CF50
:10B1C00081E08093B6128BE490E0F8019183808354
:10B1D00081E02DC06838E1F787EB92E10E94AA5622
:10B1E000EC01209781F3CE010296E816F906D9F416
:10B1F000BE0187EB92E10E94EF56E0900212F090C0
:10B2000003128A859B859093031280930212EC852A
:10B21000FD85309719F08E859F850995F092031270
:10B22000E0920212D0CF0990D881C02DDACFDF9101
:10B23000CF911F910F91FF90EF9008951092B61249
:10B2400087EB92E10E94A65660E070E080E992E010
:10B250000C94EA550F931F93CF93DF93EC01009169
:10B260000212109103121B870A875D874C873F8764
:10B270002E878091B612882379F080E992E090932E
:10B28000031280930212CE0102960E943C58109342
:10B2900003120093021202C07D836C83BE0187EB10
:10B2A00092E10E94EF56BE0187EB92E1DF91CF91D0
:10B2B0001F910F910C940A570F931F93CF93DF9315
:10B2C000EC018091B612882391F000910212109146
:10B2D000031280E992E09093031280930212CE0150
:10B2E00002960E9446581093031200930212BE0168
:10B2F00087EB92E10E94EF56BE0187EB92E1DF916E
:10B30000CF911F910F910C940A570F931F93CF93D6
:10B31000DF93EC018091B612882391F00091021224
:10B320001091031280E992E090930312809302122D
:10B33000CE0102960E9450581093031200930212FD
:10B34000BE0187EB92E10E94EF56BE0187EB92E1CE
:10B35000DF91CF911F910F910C940A57CF93DF93F8
:10B36000EC018091B612882329F0CE0102960E944A
:10B37000935804C01F821E8219861886BE0187EB6F
:10B3800092E1DF91CF910C94EF56CF93DF93EC01D4
:10B390008091B612882331F0CE010296DF91CF91D1
:10B3A0000C94635887EB92E10E94AA56009739F0FB
:10B3B0008C179D0739F0FC0180819181F7CF81E0E6
:10B3C00090E002C080E090E0DF91CF9108952F924D
:10B3D0003F924F925F926F927F928F929F92AF9225
:10B3E000BF92CF92DF92EF92FF920F931F93CF9372
:10B3F000DF93CDB7DEB7E8970FB6F894DEBF0FBE88
:10B40000CDBFE9E4FBE22081318142815381E5E453
:10B41000FBE25080418032802380E1E4FBE28081C6
:10B42000898391819A83A281AB836380EDE3FBE200
:10B43000B081BC8381818D8392819E83A381AF8300
:10B44000E9E3FBE2B081B8878181898792819A879D
:10B45000A381AB87E5E3FBE2B081BC8781818D8767
:10B4600092819E87A381AF87E1E3FBE2B081B88B35
:10B470008181898B92819A8BA381AB8BEDE2FBE278
:10B48000B081BC8B81818D8B92819E8BA381AF8B90
:10B49000E9E2FBE2B081B88F8181898F92819A8F36
:10B4A000A381AB8FE5E2FBE2B081BC8F81818D8F00
:10B4B00092819E8FA381AF8FE1E2FBE2B081B8A3BE
:10B4C000818189A392819AA3A381ABA3EDE1FBE2E1
:10B4D000B081BCA381818DA392819EA3A381AFA3E0
:10B4E000E9E1FBE2B081B8A7818189A792819AA79F
:10B4F000A381ABA7E5E1FBE2B081BCA781818DA769
:10B5000092819EA7A381AFA7E1E1FBE2B081B8AB36
:10B51000818189AB92819AAB7380EDE0FBE2B080D0
:10B52000A18092808380E9E0FBE2F080E180D2801C
:10B53000C380E5E0FBE2A081AFABB181B8AF12817F
:10B5400003812BAB3CAB4DAB5EAB0E948C665EA91E
:10B550005F934DA94F933CA93F932BA92F932F9213
:10B560003F924F925F926F922B812F932A812F935C
:10B5700029812F932F812F932E812F932D812F930C
:10B580002C812F932B852F932A852F9329852F93F9
:10B5900028852F932F852F932E852F932D852F93DD
:10B5A0002C852F932B892F932A892F9329892F93C9
:10B5B00028892F932F892F932E892F932D892F93AD
:10B5C0002C892F932B8D2F932A8D2F93298D2F9399
:10B5D000288D2F932F8D2F932E8D2F932D8D2F937D
:10B5E0002C8D2F932BA12F932AA12F9329A12F9339
:10B5F00028A12F932FA12F932EA12F932DA12F930D
:10B600002CA12F932BA52F932AA52F9329A52F93F8
:10B6100028A52F932FA52F932EA52F932DA52F93DC
:10B620002CA52F937F922AA92F9329A92F9328A97C
:10B630002F938F929F92AF92BF92CF92DF92EF9211
:10B64000FF920F931F9328AD2F932FA92F939F93B2
:10B650008F937F936F93A3E1B9E28C911F928F93A5
:10B66000E2E1F9E280811F928F9384EE9FE09F9345
:10B670008F930E943394E9E7FBE22081318142817C
:10B680005381E5E7FBE25080418032802380E9E688
:10B69000FBE29080818072806380E5E6FBE280813E
:10B6A000898391819A83A281AB83B381BC83E1E6D4
:10B6B000FBE280818D8391819E83A281AF83B381E0
:10B6C000B887EDE5FBE28081898791819A87A28125
:10B6D000AB87B381BC87E9E5FBE280818D879181EF
:10B6E0009E87A281AF87B381B88BE5E5FBE28081BD
:10B6F000898B91819A8BB280A380E1E5FBE2F08097
:10B70000E180D280C380EDE4FBE2A081AB8BB1810C
:10B71000BC8B128103810FB6F894DEBF0FBECDBF84
:10B720002BAB3CAB4DAB5EAB0E948C665EA95F93CE
:10B730004DA94F933CA93F932BA92F932F923F9252
:10B740004F925F926F927F928F929F922C812F9354
:10B750002B812F932A812F9329812F9328852F9333
:10B760002F812F932E812F932D812F932C852F9313
:10B770002B852F932A852F9329852F9328892F9303
:10B780002F852F932E852F932D852F93AF92BF92C8
:10B790002A892F9329892F93CF92DF92EF92FF92DC
:10B7A0000F931F932C892F932B892F939F938F9304
:10B7B0007F936F93A3E1B9E28C911F928F93E2E1A3
:10B7C000F9E280811F928F9385E79FE09F938F938B
:10B7D0000E9433940FB6F894DEBF0FBECDBFE8963B
:10B7E0000FB6F894DEBF0FBECDBFDF91CF911F9192
:10B7F0000F91FF90EF90DF90CF90BF90AF909F9010
:10B800008F907F906F905F904F903F902F90089512
:10B8100080E380936D130895CF93DF9360916D1350
:10B8200070E0C0E3D0E0C61BD70B65547D4EAE017F
:10B830000E946C93CE01DF91CF910895CF92DF9259
:10B84000EF92FF920F931F93CF93DF937C01C090F1
:10B850007013D090711360916D1370E0E601E09663
:10B86000C61BD70BC138D105D8F400E310E0061B86
:10B87000170B65547D4EA8010E946C936091B9121C
:10B880007091BA1280916E1390916F13680F791FA7
:10B89000A601C701800F911F0E946C93CE0102C0C8
:10B8A00080E090E0DF91CF911F910F91FF90EF909A
:10B8B000DF90CF90089590916D13980F90936D1332
:10B8C000089540917013509171134817590798F0DB
:10B8D00020916E1330916F13280F391F30936F131F
:10B8E00020936E13481B590B5093711340937013A0
:10B8F00081E090E0089580E090E0089590937113C6
:10B9000080937013089580916E1390916F138551F9
:10B910009D4E089580916D1390E085549D4E08953D
:10B9200081E090E02091B9123091BA122B5E324141
:10B9300011F480E090E008950E94905C892B61F002
:10B940006091B9127091BA124091701350917113B5
:10B950008BEE92E10C946C9320916E1330916F13E7
:10B9600021153105B9F08091701390917113C09633
:10B97000EBEEF2E1AF014B5B52414817590734F44B
:10B98000DF01A20FB31F4C914193F4CF10926F13BC
:10B9900010926E1308958091B9129091BA12089581
:10B9A0008091701390917113089590916D1380E3BD
:10B9B000891B089520E380916D13281B80917013DB
:10B9C00090917113820F911D08951F93CF93DF9370
:10B9D000EC0110916D13812F90E08C179D076CF096
:10B9E0000E94DA5C8C0F9D1F8138910530F41C1B7E
:10B9F00010936D1381E090E002C080E090E0DF9151
:10BA0000CF911F910895CF93DF93ECE1F9E211926A
:10BA1000119289E2EC34F807D1F7C4E1D9E260E091
:10BA200073E0CE010E949653229689E2CC31D8076A
:10BA3000B1F7DF91CF91089510926F1310926E13AA
:10BA4000109271131092701380E380936D138BEE3C
:10BA500092E19093BA128093B9120C94035DEF9225
:10BA6000FF920F931F93CF93DF9300D0CDB7DEB734
:10BA70008C0169837A830E941C5D6981E62E7A813C
:10BA8000F72E81E8E816F10418F080E8E82EF12C92
:10BA9000A701B8018091B9129091BA120E946C93DB
:10BAA000F0927113E0927013C7010F900F90DF9125
:10BAB000CF911F910F91FF90EF9008950F931F93D7
:10BAC000CF93DF938C01EB010E941C5D1093BA129F
:10BAD0000093B912D0937113C0937013DF91CF917B
:10BAE0001F910F91089520E3ECE1F9E2DC01019050
:10BAF0000D922A95E1F788E0E4E1F9E2DB0101909B
:10BB00000D928A95E1F7089520E3FC01ACE1B9E2DA
:10BB100001900D922A95E1F788E0FB01A4E1B9E2DA
:10BB200001900D928A95E1F70895E82FF0E0EE0F6D
:10BB3000FF1FE45EF64D7183608381E090E008951D
:10BB4000E82FF0E0EE0FFF1FE45EF64D808191815B
:10BB5000089590E0880F991F8C51974D0E9496533D
:10BB600081E090E0089590E0880F991F8C51974DE7
:10BB700008958115910511F00197F1F70895E0916D
:10BB80004F29F0915029908180914E298923089561
:10BB9000E0914C29F0914D29808190914E29892B7B
:10BBA0008083E0915129F0915229808190914E2912
:10BBB000892B80830895E0914C29F0914D29908143
:10BBC00080914E29809589238083E0915129F091BD
:10BBD0005229908180914E298095892380830895F0
:10BBE0001F93CF93DF93E0914C29F0914D299081E1
:10BBF00080914E29809589238083E0915129F0918D
:10BC00005229808190914E29892B80838FEB93E07C
:10BC10000E94B95D1FB7F894E0915129F091522923
:10BC2000908180914E2980958923808383E890E0DC
:10BC30000E94B95DE0914F29F0915029D081C091C7
:10BC40004E291FBF78948BE393E00E94B95DE09189
:10BC50004F29F0915029908180914E29982319F015
:10BC60008D2F8C2301C081E0DF91CF911F9108952A
:10BC7000509352294093512970934D2960934C2938
:10BC80009093502980934F2981E001C0880F2A9515
:10BC9000EAF780934E290C94F05DCF93DF93C82F81
:10BCA000DFB7F894E0915129F09152298081909169
:10BCB0004E29892B808383E090E00E94B95DCC23DC
:10BCC00051F0E0915129F0915229808190914E29B3
:10BCD00090959823908387E190E00E94B95DE09170
:10BCE0004F29F0915029808190914E29892309F4A0
:10BCF000C0E089E590E00E94B95DE0915129F091A2
:10BD00005229808190914E29909598239083DFBF8E
:10BD10008BE390E00E94B95D8C2FDF91CF91089565
:10BD2000CF93DF93C82FD8E08C2F81700E944D5E97
:10BD3000C6958111C068D150B9F78C2FDF91CF9192
:10BD400008958FEF0C94905EDF92EF92FF920F9325
:10BD50001F93CF93DF93E82EEB010E94F05D8111DA
:10BD60002FC080EF0E94905EF12C10E488EFD82E57
:10BD7000D10E81E00E944D5E082F81E00E944D5E51
:10BD8000882319F0002361F01DC0011109C01E15A0
:10BD900028F0888180FF04C0E11611F0F12E01E047
:10BDA000802F0E944D5E988196950111906898832E
:10BDB00011501D11DECF21961111D8CF8F2D03C048
:10BDC0008FEF01C08EEFDF91CF911F910F91FF9008
:10BDD000EF90DF900895FF920F931F93CF93DF931F
:10BDE000F82EEB010E94F05D209769F085E50E9436
:10BDF000905E8E01085F1F4F89910E94905EC01770
:10BE0000D107D1F703C08CEC0E94905E8F2DDF919B
:10BE1000CF911F910F91FF900C94905E0F931F9301
:10BE2000CF93DF93DB01EC9111969C911197F0E099
:10BE3000F92B803181F4BF016E7FE3E0660F771F3D
:10BE4000EA95E1F716969C911697ECE0F0E0E91B75
:10BE5000F109E60FF71FF7FF07C091E0EA019883A9
:10BE6000F195E195F10902C0EA011882883279F46E
:10BE700014968C91982F9076903649F086FF02C0E8
:10BE8000EE7F05C085FF02C0EC7F01C0E87FCF01D7
:10BE900044E0969587954A95E1F7D9018C93EF7028
:10BEA000E801E88380E0DF91CF911F910F91089521
:10BEB0000F931F93CF93DF93EC018B01B80188811F
:10BEC0000E94A45E888381508D3F30F4F801808108
:10BED000883211F0803191F7DF91CF911F910F914E
:10BEE0000895CF93DF93EC010E94F05DBE0184EBD7
:10BEF0000E94EB5E81E00E944D5EC82F0E94F05DC3
:10BF000081E0C11101C080E0DF91CF9108951F93BE
:10BF1000CF93DF9300D0CDB7DEB7182F69837A8334
:10BF20000E94F05D0E94BF5D69817A81882341F0A3
:10BF300084E40E94EB5E113029F00E94C85D02C0CB
:10BF400082E001C080E00F900F90DF91CF911F91B0
:10BF500008954F925F926F927F928F929F92AF92CD
:10BF6000BF92CF92DF92EF92FF920F931F93CF93E6
:10BF7000DF93CDB7DEB729970FB6F894DEBF0FBEBB
:10BF8000CDBF6C015B014A0189010E94F05DB601E1
:10BF90008EEB0E94EB5ECE0101967C013E019AE0A1
:10BFA000690E711C27010E94A15EF70181937F0138
:10BFB000E615F705C1F769E070E0C2010E94447917
:10BFC000811109C09401A501B201F60180810E948E
:10BFD0000E5F80E001C083E029960FB6F894DEBFC3
:10BFE0000FBECDBFDF91CF911F910F91FF90EF90CA
:10BFF000DF90CF90BF90AF909F908F907F906F9089
:10C000005F904F9008955F926F927F928F929F9270
:10C01000AF92BF92CF92DF92EF92FF920F931F9356
:10C02000CF93DF93CDB7DEB729970FB6F894DEBF75
:10C030000FBECDBF582E6B015A01890160E070E040
:10C040008EEB0E94EB5ECE0101967C014E019AE0E0
:10C05000890E911C37010E94A15EF70181937F0137
:10C06000E815F905C1F769E070E0C3010E94447961
:10C07000811108C09501A601B301852D0E940E5FB4
:10C0800080E001C083E029960FB6F894DEBF0FBEB2
:10C09000CDBFDF91CF911F910F91FF90EF90DF9077
:10C0A000CF90BF90AF909F908F907F906F905F9058
:10C0B00008950F931F93CF93DF93CDB7DEB72897E3
:10C0C0000FB6F894DEBF0FBECDBF182F062F98E035
:10C0D000ECE0F3E0DE01119601900D929A95E1F704
:10C0E000242F332727FD309541E752E0249FC001DC
:10C0F000259F900D349F900D112464E670E00E94FE
:10C10000568DCB0144E6049F800D911D1124FE0144
:10C110003196AE01475F5F4F619170E02617370798
:10C1200011F4019603C0E417F507B1F7112319F0D4
:10C1300091958195910928960FB6F894DEBF0FBEB0
:10C14000CDBFDF91CF911F910F910895EF92FF9294
:10C150000F931F93CF93DF93CDB7DEB72B970FB617
:10C16000F894DEBF0FBECDBFF82EE92E682F792FD1
:10C1700088E08F0D0E94875F882319F084E391E2A5
:10C1800043C066E471E48FE090E00E9411618E018B
:10C19000075F1F4F9801AE01465F5F4FBE01655FAD
:10C1A0007F4F8F2D9E2D0E94A95F8111E7CF88E0E0
:10C1B000ECE0F3E0DE01119601900D928A95E1F733
:10C1C000498521E732E0429FC001439F900D112431
:10C1D00064E670E00E94568D8A8594E6899F600D22
:10C1E000711D1124FE0131968191481303C06F5FC8
:10C1F0007F4F03C0E017F107B9F78B85882319F04B
:10C20000719561957109CB012B960FB6F894DEBF3D
:10C210000FBECDBFDF91CF911F910F91FF90EF9097
:10C220000895DC01CB0181159105A105B10529F027
:10C2300081509040A040B040D9F708959B01AC01D7
:10C240001092B90060E072E18AE790E00E946A8D86
:10C250002051310941095109569547953795279540
:10C260002093B800089594EA9093BC0040EA56E801
:10C2700061E070E09091BC0097FD0BC04150510906
:10C2800061097109411551056105710599F781E051
:10C2900008959091B900987F983011F09031B9F7D6
:10C2A0008093BB0084E88093BC0080EA96E8A1E01C
:10C2B000B0E02091BC0027FD08C00197A109B10999
:10C2C0000097A105B105A9F7E2CF8091B900887F59
:10C2D000883111F08034D9F680E0089524EA34E8FA
:10C2E00044E92093BC009091BC0097FFFCCF909153
:10C2F000B900987F983011F0903199F78093BB0086
:10C300003093BC009091BC0097FFFCCF9091B90096
:10C31000987F903211F0983539F44093BC00909199
:10C32000BC0094FDFCCFDDCF08950C94336184E90B
:10C330008093BC008091BC0084FDFCCF0895809365
:10C34000BB0084E88093BC008091BC0087FFFCCFD9
:10C350009091B900987F81E0983209F480E00895C7
:10C3600084EC8093BC008091BC0087FFFCCF80915F
:10C37000BB00089584E88093BC008091BC0087FFD7
:10C38000FCCF8091BB000895E0E1DC01FD91CD017F
:10C39000F0933F01E150C9F780913C018F7D80937C
:10C3A0003C0180913C01877F80933C01FB0180E14F
:10C3B000919190933E018150D9F780913C01806822
:10C3C00080933C0180913D0180FFFCCF4051510999
:10C3D00080913C01806280933C0180913C01877F89
:10C3E00080933C01141615069CF4FB0180E19191A9
:10C3F00090933E018150D9F780913C0180688093F1
:10C400003C0180913D0180FFFCCF40515109EACFB2
:10C41000F90180E190913E0191938150D9F781E03B
:10C4200090E008950F931F93CF93DF93EC018CE777
:10C430000E946E618CE70E949F618E01005F1F4F1A
:10C4400089910E949F61C017D107D1F7DF91CF91E9
:10C450001F910F910C949761813019F440E050E0E6
:10C4600002C040EC50E060E070E08CE790E00C949B
:10C47000BE11813019F44EE050E002C048E050E0B7
:10C4800060E070E08CE790E00C94BE1141E050E079
:10C4900060E070E08CE790E00E94BE116AE67AE00E
:10C4A00080E090E00C94116148E350E060E070E0BF
:10C4B0008CE790E00E94BE1149E350E060E070E03C
:10C4C0008CE790E00E94BE1144E150E060E070E033
:10C4D0008CE790E00E94BE1148E750E060E070E019
:10C4E0008CE790E00E94BE114EE550E060E070E005
:10C4F0008CE790E00E94BE114DE650E060E070E0F5
:10C500008CE790E00E94BE116CE17AE186E090E059
:10C510000E9411614CE050E060E070E08CE790E038
:10C520000E94BE1141E050E060E070E08CE790E0D6
:10C530000E94BE1146E050E060E070E08CE790E0C1
:10C540000E94BE116AE67AE080E090E00C941161EE
:10C55000CF93DF93CDB7DEB7A2970FB6F894DEBFC7
:10C560000FBECDBF81E1E0E4F9E0DE01529601901B
:10C570000D928A95E1F781E1E1E5F9E0DE0111969E
:10C5800001900D928A95E1F70E945462CE01429685
:10C590000E94126282E00E942C626AE67AE080E0E9
:10C5A00090E00E941161CE0101960E94126260E14A
:10C5B0007EEA88E290E00E94116180E00E94396288
:10C5C00060E17EEA88E290E00E9411614EE050E076
:10C5D00060E070E08CE790E00E94BE11A2960FB67A
:10C5E000F894DEBF0FBECDBFDF91CF910895CF92FB
:10C5F000DF92EF92FF920F931F93CF93DF9300D0C0
:10C600001F92CDB7DEB7F82E042F122F213031F054
:10C61000223031F0243031F0283031F090E005C084
:10C6200091E003C092E001C093E00C3059F00E306D
:10C6300011F4946007C0003111F4986003C0023116
:10C6400009F49C60613059F0623011F4906207C0C7
:10C65000633011F4906403C0643009F4906690680C
:10C66000692F70E023E030E0AE014F5F5F4F8F2D08
:10C6700090E00E94D51169E07AE180E090E00E94AC
:10C6800011618F2D8160F82E0E9433610E94B0618C
:10C6900089830E94B0618A83023119F40E94B061DB
:10C6A0008B830E94B06187FDF1CF0E94BA610E9426
:10C6B000976169E07AE180E090E00E9411618F2D3E
:10C6C0000E9433610E94B06189830E94B0618A83B5
:10C6D000023119F40E94BA618B830E94BA610E94F0
:10C6E000976139812A81023149F5832F90E0A0E0DA
:10C6F000B0E04B817727662731FF0EC030E0322F44
:10C700002227620F731F811D911D640F711D811DF2
:10C71000911D8C6F9F6F0BC030E0322F2227620F6C
:10C72000731F811D911D640F711D811D911D0E943C
:10C73000908A20E83FEF4FEF57E420C0632F70E06E
:10C74000762F6627620F711D882777FD8095982FB9
:10C750000E94908A0C3029F420E030EE4FEF54E430
:10C760000DC00E3029F420E038EF4FEF55E406C03D
:10C77000003131F420E03EEF4FEF56E40E94F189A2
:10C780002FE632E143E050E40E94728C6B017C01A1
:10C79000612F70E080E090E00E94908A9B01AC01E4
:10C7A000C701B6010E94F1890F900F900F90DF91A1
:10C7B000CF911F910F91FF90EF90DF90CF90089550
:10C7C000E6E4F1E080812081908130818295869538
:10C7D0008695837022952F70822B832B92959F7064
:10C7E000892B08950F931F93CF93DF9300D0CDB77C
:10C7F000DEB746E06CE080E00E94226789E180932A
:10C80000C4001092C50082E08093C00080E00E94C6
:10C81000AF670E944E6684B784B784B784B784B785
:10C82000E3EDF1E322E432E4318320833A968DB7DD
:10C830009EB70A97E817F907B8F382E699E09F9345
:10C840008F9381E391E19F938F930E9433940E9491
:10C8500087750E94425560E070E086E892E00E9491
:10C86000EA550E941E59E0911403F09115030995B1
:10C870000E94E06390E00E94C375CE0101960E9481
:10C8800083650F900F900F900F90882341F081E106
:10C8900091E19F938F930E9433940F900F90CE015C
:10C8A00001960E94B1530E9491658C010E948D6592
:10C8B000AE014F5F5F4FB8010E94796A0E94FD642C
:10C8C0000E945A6A0E9495650E94B36B84E091E1D0
:10C8D0009F938F930E9433948A811F928F9300E0DD
:10C8E00011E11F930F930E94339489811F928F93BC
:10C8F0001F930F930E9433948EEF90E19F938F9339
:10C900000E9433940E94C775E0915103F091520345
:10C910000995E0914303F09144030995E0912A03BE
:10C92000F0912B0309950E94BA6B182F0E94576A49
:10C930001F921F931F928F93809150038F9380912A
:10C940004F038F93809142038F93809141038F9384
:10C9500083EE90E19F938F930E943394E0915B0369
:10C96000F0915C030FB6F894DEBF0FBECDBF3097D9
:10C9700091F00995BC0180E890E00E94428D7F9380
:10C980006F9380ED90E19F938F930E9433940F906B
:10C990000F900F900F908EEC90E19F938F930E94D9
:10C9A000339460E070E08CED92E00E94EA5580EFF5
:10C9B00092E00E94977486EC90E19F938F930E947F
:10C9C00033940F900F900F900F900F900F90DF9176
:10C9D000CF911F910F9108957F936F939F938F93A2
:10C9E00080EC90E19F938F930E9433940F900F906F
:10C9F0000F900F900F900F9008951F93CF93DF9398
:10CA0000CDB7DEB7A0970FB6F894DEBF0FBECDBF8F
:10CA10008DE590E00E949F95182F282F35EF380F55
:10CA2000303108F0982F9095291709F461C08CE4F3
:10CA300091E19F938F930E943394E1E9F1E10F908C
:10CA40000F90DE01119684918D93319681E1E93941
:10CA5000F807C9F7F89448E050E069E770E0CE01C4
:10CA600001960E94A595E3E8F1E1DE01119684911B
:10CA70008D93319681E1E139F807C9F74EE050E036
:10CA80006BE670E0CE0101960E94A595E9E7F1E121
:10CA9000DE01119684918D93319681E1E338F80798
:10CAA000C9F74AE050E061E670E0CE0101960E94CD
:10CAB000A5956DEC7BEA8BE590E00E94BD9560E06A
:10CAC00070E089E590E00E94BD9560E088E590E027
:10CAD0000E94AF9560E070E08FE590E00E94BD9508
:10CAE0001AE16AE175EE8DE590E00E94BD957894BB
:10CAF000812FA0960FB6F894DEBF0FBECDBFDF9199
:10CB0000CF911F910895F89442E050E069E770E0FA
:10CB10000E948795789480E008958BE590E00C94CE
:10CB20009F9589E590E00C949F9588E590E00C94A2
:10CB30009795409161295091622960916329709184
:10CB4000642990E0A0E0B0E0480F591F6A1F7B1FE6
:10CB500040936129509362296093632970936429FB
:10CB600040915D2950915E2960915F297091602903
:10CB7000480F591F6A1F7B1F40935D2950935E2900
:10CB800060935F29709360292091012B2223A1F0EB
:10CB90004091592950915A2960915B2970915C29E3
:10CBA000480F591F6A1F7B1F4093592950935A29D8
:10CBB00060935B2970935C2908951F920F920FB6C2
:10CBC0000F9211240BB60F922F933F934F935F93C5
:10CBD0006F937F938F939F93AF93BF93EF93FF9345
:10CBE00080917413909175130196909375138093AF
:10CBF0007413809173138F5F809373138038A9F43B
:10CC0000109273138091612990916229A0916329F8
:10CC1000B09164290196A11DB11D80936129909363
:10CC20006229A0936329B09364298091012B882302
:10CC3000E1F0809172138F5F809372138038A9F4B2
:10CC4000109272138091592990915A29A0915B29D1
:10CC5000B0915C290196A11DB11D80935929909333
:10CC60005A29A0935B29B0935C290E947A58892B9A
:10CC700011F00E948D57FF91EF91BF91AF919F915D
:10CC80008F917F916F915F914F913F912F910F9075
:10CC90000BBE0F900FBE0F901F901895F894109236
:10CCA000B60016BC83EF87BD82E084BD94E095BDDD
:10CCB00095B395BB80936E0078940895809174131A
:10CCC0009091751320917413309175138217930707
:10CCD000A9F70895009751F022E330E000002150B9
:10CCE000310921153105D1F70197F4CF08950F933C
:10CCF0001F93CF93DF93EC010E945E668C010E942C
:10CD00005E66801B910B8C179D07C8F3DF91CF9156
:10CD10001F910F91089508950F931F9360916129BA
:10CD20007091622980916329909164290091612911
:10CD3000109162292091632930916429601771074D
:10CD40008207930759F71F910F9108951F920F9231
:10CD50000FB60F9211241092B2020F900FBE0F90D7
:10CD60001F9018951F920F920FB60F9211240BB6B9
:10CD70000F922F933F934F935F936F937F938F9374
:10CD80009F93AF93BF93EF93FF93E091A802F0912D
:10CD9000A9028081E091B302F091B402309709F0CA
:10CDA0000995FF91EF91BF91AF919F918F917F91E5
:10CDB0006F915F914F913F912F910F900BBE0F900C
:10CDC0000FBE0F901F9018951F920F920FB60F92E3
:10CDD00011241092BF020F900FBE0F901F90189554
:10CDE0001F920F920FB60F9211240BB60F922F9332
:10CDF0003F934F935F936F937F938F939F93AF93E3
:10CE0000BF93EF93FF93E091B502F091B60280815A
:10CE1000E091C002F091C102309709F00995FF91AD
:10CE2000EF91BF91AF919F918F917F916F915F91A2
:10CE30004F913F912F910F900BBE0F900FBE0F900F
:10CE40001F9018959DE0899FF0011124E855FD4F32
:10CE5000A281B3811C92A481B5816C93A681B78114
:10CE600088ED8C93A085B1854C9312861486138629
:10CE700008959DE0899FF0011124E855FD4F81E060
:10CE80008287A081B1816C933A9680818111FDCF18
:10CE900008951F93CF93DF93182FEB01FE01849128
:10CEA000882339F0FE016491812F0E943967219611
:10CEB000F5CFDF91CF911F9108951F93CF93DF930B
:10CEC000182FEB018881882369F08A3021F46DE006
:10CED000812F0E94396769916D30A1F3812F0E94E3
:10CEE0003967F0CFDF91CF911F910895CF93DF93F2
:10CEF000CDB7DEB79E01285F3F4F4E815F8160E472
:10CF000070E086E793E10E94F09466E773E18D811B
:10CF10000E945D67DF91CF910895CF93C82F8A302B
:10CF200031F46DE08091B6130E94396702C08D30F4
:10CF300029F06C2F8091B6130E94396780E090E051
:10CF4000CF9108959DE0899FF0011124E855FD4F90
:10CF5000748763870895682F80E00C943967809305
:10CF6000B6138AE992E09093CE318093CD31089543
:10CF700084B7877F84BF88E10FB6F8948093600000
:10CF8000109260000FBE08952FE088E190E00FB688
:10CF9000F894A895809360000FBE209360000895D8
:10CFA000A895089588E10FB6F894809360001092D8
:10CFB00060000FBE0895F89428E088E190E00FB675
:10CFC000F894A895809360000FBE20936000FFCF77
:10CFD00080916C2980916C2990E0089540E06FE188
:10CFE00081E491E00C944F6DE9E3F1E08081808170
:10CFF0008D7F80838DE090E00197F1F723E040E0A2
:10D000006FE182E491E00E94596D83E090E0019726
:10D01000F1F708959091390191FD0AC0282F8031D0
:10D0200008F02FE040E06FE085E491E00C94596D4A
:10D0300008958091390181FD0EC040E06FE181E4E7
:10D0400091E00E944F6D282F2F7E81E090E02130EB
:10D0500021F080E0089580E090E00895809139010A
:10D0600081FD10C040E06FE181E491E00E944F6DCE
:10D070008F3131F0982F9F7E915081E0923018F4DB
:10D0800080E0089581E008950E942E688823E1F3EE
:10D090000895CF93DF93C82F0E9444680E94EE67E3
:10D0A000D82FC81789F1C83019F40E94F46725C039
:10D0B000C93121F4863189F429E005C0C63169F40B
:10D0C000893159F426E040E06FE182E491E00E946A
:10D0D000596DE3E0F0E03197F1F72C2F40E06FE17C
:10D0E00082E491E00E94596DD83019F4E9E6F1E04C
:10D0F00002C0E3E0F0E03197F1F70E94EE678C1791
:10D1000019F083E490E002C080E490E0DF91CF91D9
:10D1100008950E9444681092012B0E94F467809148
:10D1200039018260809339018091842B8823D9F161
:10D1300080919400909195004091952B5091962B61
:10D1400084179507A0F48091612B9091622BA09198
:10D15000632BB091642B8C57914EAF4FBF4F809390
:10D16000612B9093622BA093632BB093642B20913F
:10D17000940030919500241B350B8091612B909188
:10D18000622BA091632BB091642B820F931FA11D82
:10D19000B11D8093612B9093622BA093632BB0936E
:10D1A000642B1092842B8091862B8823D9F1809157
:10D1B0009400909195004091992B50919A2B84174F
:10D1C0009507A0F48091692B90916A2BA0916B2B0D
:10D1D000B0916C2B8C57914EAF4FBF4F8093692B02
:10D1E00090936A2BA0936B2BB0936C2B209194009F
:10D1F00030919500241B350B8091692B90916A2BFF
:10D20000A0916B2BB0916C2B820F931FA11DB11DB0
:10D210008093692B90936A2BA0936B2BB0936C2B0C
:10D220001092862B08958091012B882381F08091A4
:10D230003A14811104C00E942E68811106C081E059
:10D240008093381481E090E008950E94896880E01E
:10D2500090E00895809194009091950090939A2B7E
:10D260008093992B21E02093862B8091390181FDB9
:10D2700008C08091390181FD1AC086E10E94496889
:10D2800016C02093002B809194009091950090936C
:10D29000962B8093952B2093842B809139018D7F41
:10D2A000809339018091002B8111FCCFE2CF81E086
:10D2B0008093012B08958091012B81110AC08091E8
:10D2C0003A14882321F081E08093391402C00E942F
:10D2D0002A6981E090E008951F93CF93DF931F9216
:10D2E000CDB7DEB78FB7898380913A14811126C0FC
:10D2F000F8948091012B882351F08091390181FDB0
:10D300001BC00E942E688823B9F080E003C00E94F1
:10D310005B6981E02091470191E02E3008F090E0B8
:10D32000192F119581110E941369107429F08981B8
:10D330008FBF81E090E004C089818FBF80E090E0E2
:10D340000F90DF91CF911F91089580913914882318
:10D3500021F00E942A691092391480913814882390
:10D3600021F00E9489681092381410923A1408959E
:10D370000F931F93AB0121E020933A140091452BAA
:10D380001091462B2091472B3091482B0F5F1F4F58
:10D390002F4F3F4F0093452B1093462B2093472B45
:10D3A0003093482B22E0260F27FF0CC08091FE2AE5
:10D3B0009091FF2A01969093FF2A8093FE2A0FEF07
:10D3C0001FEF07C0BC0187EB93E10E946C9300E064
:10D3D00010E00E94A569C8011F910F9108958093E4
:10D3E0003C1408950E94EE67823011F0823111F4EE
:10D3F00080E0089581E0089508958FEF80934E01B5
:10D4000022E044E060EF8CE691E00E94596D25E057
:10D4100041E06EE08CE290E00E94596D80E88093DC
:10D420006F018091460180936D0121E045E060E24B
:10D4300084E491E00C94596D8DEF93E00197F1F73E
:10D440000E94456D109275291092F7291092792A41
:10D450001092742910927329E9E3F1E080818E7FA4
:10D46000808380818D7F80838DE090E00197F1F74C
:10D4700080818160808323E040E06FE182E491E07D
:10D480000E94596D8DEF93E00197F1F780915D0156
:10D4900080915E010E94FD6960E070E082EC92E0A4
:10D4A0000E94EA550E942A6981E090E008958091E7
:10D4B0003B140895CF93DF931F92CDB7DEB78983D6
:10D4C0000E944468898180933B14282F40E06FE1DB
:10D4D00088E491E00F90DF91CF910C94596D0E94F8
:10D4E0005A6A8091390181FD03C086E00C94496835
:10D4F0000895FA0180936201909363016093600143
:10D50000709361013097C1F0808180936B018181BC
:10D5100080936A018281809369018381809368018D
:10D5200084818093670185818093660186818093E1
:10D530006501878180936401089582EC92E00E94E6
:10D540000B5681E080936C2980916D2990916E2912
:10D55000019690936E2980936D2981E090E0089563
:10D560008091742992E8899FF0011124EB58F64DBF
:10D5700010828F5F833018F48093742902C0109258
:10D580007429E091742982E8E89FF0011124EB5896
:10D59000F64D808181110C949D6A10926C2908953A
:10D5A0001F93CF93DF932091742912E8129F90016B
:10D5B0001124D901AB58B64D4C91411103C00E94C2
:10D5C000B06A93C05091390151FD8FC05091012B29
:10D5D000552309F48AC047FF16C00E94B06A8091A3
:10D5E000352B9091362BA091372BB091382B01968B
:10D5F000A11DB11D8093352B9093362BA093372B13
:10D60000B093382B72C04330B0F40E94B06A80915E
:10D61000312B9091322BA091332BB091342B01966A
:10D62000A11DB11D8093312B9093322BA093332BEE
:10D63000B093342B5AC050E0EA0122976C177D0753
:10D64000B0F40E94B06A80912D2B90912E2BA09166
:10D650002F2BB091302B0196A11DB11D80932D2B46
:10D6600090932E2BA0932F2BB093302B3EC0B9015B
:10D670006A58764D0E946C93E09174291E9FF001C8
:10D680001124EB50F64D8081809365290E94B06A89
:10D69000809147018093662990916B29992311F01D
:10D6A000891710F480936B296091662970E084E0FB
:10D6B0000E94955D6091652970E083E00E94955D10
:10D6C0004091492B50914A2B60914B2B70914C2BE0
:10D6D0004F5F5F4F6F4F7F4F4093492B50934A2BC3
:10D6E00060934B2B70934C2B02C0C0E0D0E0CE0176
:10D6F000DF91CF911F910895CF93DF93EC01888143
:10D7000099810097E9F08730954021F019821882BD
:10D7100083E026C06238C1F410926C290E941C5D1F
:10D720000E94835C60E870E00E94D06A18161906B7
:10D730006CF40E947E5CE0915503F09156030995CC
:10D7400087E095E09983888381E00AC08091692908
:10D7500090916A29019690936A2980936929F0CF64
:10D76000DF91CF91089591E090933A140E940A6856
:10D770000C94A5698091390181FD06C040E06FE0FD
:10D7800085E491E00C944F6D80E108950F931F9311
:10D79000CF93DF93182F21E020933A140091012BAF
:10D7A0008091390181FF16C080919400909195007D
:10D7B0009093962B8093952B2093842B2093002B72
:10D7C000809139018D7F809339018091002B8111E7
:10D7D000FCCF00E00E9444688091012B882309F46B
:10D7E0003FC08091862B8823D9F18091940090913D
:10D7F0009500E091992BF0919A2B8E179F07A0F43A
:10D800004091692B50916A2B60916B2B70916C2B1E
:10D810004C57514E6F4F7F4F4093692B50936A2B5B
:10D8200060936B2B70936C2B20919400309195003A
:10D830002E1B3F0B4091692B50916A2B60916B2BF3
:10D8400070916C2B420F531F611D711D4093692B0A
:10D8500050936A2B60936B2B70936C2B1092862BDA
:10D860008091390181FD03C089E10E94496886E009
:10D870000E94A05D892B51F00E94BA6BC82F86E0F0
:10D880000E94A05D81500E940A6802C0C0E0D0E002
:10D8900020919400309195003093982B2093972BF2
:10D8A00081E08093852BF894809139018260809388
:10D8B0003901809139018D7F8093390162E0610FD8
:10D8C00087EB93E10E94886D78942091FB2A309138
:10D8D000FC2A2F5F3F4F3093FC2A2093FB2A0E94A3
:10D8E000446845E060EE82E491E00E944F6D182F9D
:10D8F00086E00E94A05D892B19F08C2F0E940A6897
:10D90000002319F00E942A6902C00E948968809150
:10D91000852B8823D9F18091940090919500E09116
:10D92000972BF091982B8E179F07A0F44091652BB1
:10D930005091662B6091672B7091682B4C57514E1C
:10D940006F4F7F4F4093652B5093662B6093672BEF
:10D950007093682B20919400309195002E1B3F0B03
:10D960004091652B5091662B6091672B7091682BCD
:10D97000420F531F611D711D4093652B5093662B01
:10D980006093672B7093682B1092852B8091012BED
:10D99000882361F0209194003091950030939A2B68
:10D9A0002093992B81E08093862B07C023E040E0F1
:10D9B0006FE182E491E00E94596D0E94A5691130E7
:10D9C000E9F01330A9F480913D2B90913E2BA0916A
:10D9D0003F2BB091402B0196A11DB11D80933D2B93
:10D9E00090933E2BA0933F2BB093402B12E009C0A5
:10D9F000153031F0173029F411E003C010E001C0F8
:10DA000013E0812F90E0DF91CF911F910F91089546
:10DA1000CF93DF93EB010E94B869009729F4CE0100
:10DA20000E94C66B009751F02091FE2A3091FF2A88
:10DA30002F5F3F4F3093FF2A2093FE2ADF91CF9133
:10DA40000895CF93DF938091012B811104C00E9430
:10DA50005B69D1E001C0D0E00E94EE67863111F031
:10DA6000813119F4C091470109C040E06FE186E4BB
:10DA700091E00E944F6DC82FCC0FC80FD1110E94AA
:10DA800013698C2FDF91CF91089510923E1410925C
:10DA90003D14EFE6F0E08081806280830895FC0110
:10DAA0008081862390E002C0959587954A95E2F79C
:10DAB0000895F894FC015081362F30955323042E9D
:10DAC00001C0220F0A94EAF72623522B5083789440
:10DAD000089540917B01FC014193A0E8B1E050E83A
:10DAE000540F9D012F5F3F4F6C916193521711F0BE
:10DAF000D901F7CF4150E42FF0E0E058FE4F2181EB
:10DB0000FC01E058FF4F2083319621E020830895E7
:10DB100060938001E1E8F1E061589F012F5F3F4F82
:10DB2000DC014D91CD014083621711F0F901F5CF71
:10DB300008951F920F920FB60F9211240BB60F92F9
:10DB40002F933F934F935F936F937F938F939F9305
:10DB5000AF93BF93EF93FF93809147018093662922
:10DB60008091732922E8829FC00111248B58964D21
:10DB70000E94696D809173298F5F833018F48093C0
:10DB8000732902C0109273290E949D6AFF91EF9140
:10DB9000BF91AF919F918F917F916F915F914F91C5
:10DBA0003F912F910F900BBE0F900FBE0F901F90C3
:10DBB00018951F920F920FB60F9211240F900FBE5F
:10DBC0000F901F9018951F920F920FB60F9211246D
:10DBD0000F900FBE0F901F9018951F920F920FB6C7
:10DBE0000F9211240F900FBE0F901F9018951F9247
:10DBF0000F920FB60F9211241092002B0F900FBEB0
:10DC00000F901F9018951F920F920FB60F9211242C
:10DC10001092002B0F900FBE0F901F9018951F921F
:10DC20000F920FB60F9211248F9381E080936C298D
:10DC30008F910F900FBE0F901F9018951F920F920B
:10DC40000FB60F9211241092002B0F900FBE0F9061
:10DC50001F9018951F920F920FB60F9211248F9359
:10DC60009F9380913D1490913E14019690933E14A1
:10DC700080933D149F918F910F900FBE0F901F9036
:10DC80001895CF92DF92EF92FF920F931F93CF934D
:10DC9000DF937C018B016A018FE394E10E94AA5615
:10DCA000EC01009751F0EC81FD81309711F0C80133
:10DCB0000995CE010E945257F3CFA601B801C701C2
:10DCC000DF91CF911F910F91FF90EF90DF90CF9058
:10DCD0000C9434540F931F93CF93DF9300D0CDB7A0
:10DCE000DEB78091092B90910A2BA0910B2BB0915C
:10DCF0000C2B0196A11DB11D8093092B90930A2B2B
:10DD0000A0930B2BB0930C2B0E94D4708C018FE34B
:10DD100094E10E94AA56009779F0DC011296ED91E9
:10DD2000FC911397309729F089839A8309959A81FA
:10DD300089810E945257EFCF0115110549F0C801A2
:10DD40000F900F90DF91CF911F910F910C942B5456
:10DD50000F900F90DF91CF911F910F9108950E9426
:10DD6000C7750E941C5D0E94FB6E81E493E0909356
:10DD7000042B8093032B0E94D2702FEF31E040E000
:10DD80005EE160E074E082E090E00C949B70BC0186
:10DD90008FE394E10C940A57BC018FE394E10C9457
:10DDA000EF56CF93DF93EC014091052B5091062B5A
:10DDB0006091072B7091082B4F5F5F4F6F4F7F4F24
:10DDC0004093052B5093062B6093072B7093082BE1
:10DDD0000E94E770009761F00E949C5CE09145030F
:10DDE000F0914603BE0181E49EE6099581E090E052
:10DDF000DF91CF91089585E494E10C94A6560F939A
:10DE0000CF93DF93EC017B836A8318865F834E8315
:10DE1000BC0185E494E10E940A57E0914114F0911D
:10DE20004214309749F04C815D8101E020E030E000
:10DE300068858A819B810995DF91CF910F91089523
:10DE4000BC0185E494E10C94EF560F93DC01189625
:10DE50001C921897E0914114F0914214309759F0B8
:10DE600000E020E030E040E050E060E012968D916C
:10DE70009C91139709950F9108950F93DC01AB01C5
:10DE800014962D913C91159781E018968C931897D4
:10DE900015967C936E931497E0914114F09142147F
:10DEA000309739F000E061E012968D919C911397C4
:10DEB00009950F9108950F93DC01E0914114F091C1
:10DEC0004214309771F014964D915C91159701E0D2
:10DED0009A0118966C91189712968D919C911397B0
:10DEE00009950F910895E0914314F09144143097EF
:10DEF00009F009940895909344148093431408956D
:10DF00009093421480934114089585E494E10C9415
:10DF1000AA56EF92FF920F931F93CF93DF938C013A
:10DF2000EB017A0185E494E10E94AA560097D9F0AA
:10DF3000DC0112962D913C9113972C173D0781F42B
:10DF40001696ED91FC911797309769F09701AE0105
:10DF5000B801DF91CF911F910F91FF90EF9009943D
:10DF60000E945257E3CFDF91CF911F910F91FF9005
:10DF7000EF9008950895CF93DF93C8E7D4E16881C7
:10DF8000798120E030E04AED5FE682E694E10E948C
:10DF90002A590E94C575688179810E94428D20E0CE
:10DFA00030E04EEE5FE6BC0182E594E1DF91CF9177
:10DFB0000C942A59809178149091791420917614B8
:10DFC00030917714880F991F2817390708F4C90171
:10DFD00090937914809378140C94BB6FCF93DF9354
:10DFE0000E941C5D0E94835CEC01198218820E94D1
:10DFF000856F28813981009719F1FC014085442300
:10E00000F9F0FC0142815381F901EE0FFF1FEE0F81
:10E01000FF1FEC0FFD1F53834283FC014481558198
:10E020002F5F3F4FF901EE0FFF1FEE0FFF1FEC0FA9
:10E03000FD1F51834083398328830E945257D9CFD3
:10E04000C901880F991F880F991F02960E947E5C54
:10E0500088819981892B31F087E494E1DF91CF9118
:10E060000C940254DF91CF910895AF92BF92CF925A
:10E07000DF92EF92FF920F931F93CF93DF9300D025
:10E08000CDB7DEB76B010E94835CFC01008111817A
:10E090001A8309830C30110518F4E12CF12C0DC002
:10E0A0001F930F9380E899E09F938F930E94219490
:10E0B0000F900F900F900F9021C0E016F106F1F035
:10E0C0000E94835CF701EE0FFF1FEE0FFF1FE80FAA
:10E0D000F91FA280B3800E94835CFFEFEF1AFF0A52
:10E0E000F701EE0FFF1FEE0FFF1FE80FF91F408132
:10E0F0005181B501C6010E94896FDFCF0F900F904B
:10E10000DF91CF911F910F91FF90EF90DF90CF9013
:10E11000BF90AF9008950F93013059F4809172141D
:10E120009091731490937914809378140F910C94B8
:10E13000BB6F0F910895EF92FF920F931F93CF93B0
:10E14000DF938B01EA0179014EE253E0BC0187E4E1
:10E1500094E10E94E6531093731400937214D093C9
:10E160007514C0937414F0927714E09276148BE8CF
:10E1700090E7DF91CF911F910F91FF90EF900C945A
:10E18000806F82E694E10E94AE5982E594E10E949C
:10E19000AE5987E494E10C940054809178149091E6
:10E1A000791408950C944054CF93DF93E091320397
:10E1B000F09133030995EC01009729F06A817B8186
:10E1C00081E00E94955DCE01DF91CF9108950F937C
:10E1D0001F93CF93DF93EC01E0913403F09135036B
:10E1E00009958C016A817B8181E00E94955D81E0C7
:10E1F00090E0012B11F480E090E0DF91CF911F912E
:10E200000F910895E0913603F0913703099420E0CF
:10E2100030E00296FC0132974081442331F0FC014A
:10E2200031974081240F311DF4CFC9010895FC01BD
:10E23000208130E0322F22278181282B02C0220F3B
:10E24000331F6A95E2F7832F9927FA01E85CFC4FA8
:10E25000208130E08223932328E030E0241B350B1B
:10E2600002C0969587952A95E2F708956F927F925E
:10E270008F929F92AF92BF92CF92DF92EF92FF92D6
:10E280000F931F93CF93DF938C01EB016A01790108
:10E290002830310524F4A901B601CE014AC0590144
:10E2A00023E0B594A7942A95E1F74115510521F093
:10E2B0004801612C712C03C0D801FB0120C048E04B
:10E2C00050E0B601CE01860D971D0E941771F40132
:10E2D00081934F01FFEF6F1A7F0A6A147B047CF36E
:10E2E000C501B7FE02C080E090E0A7014770552746
:10E2F0004115510511F1080F191FB60118C0CF01C2
:10E300008C1B9D0B8A159B051CF481918D93F7CF77
:10E31000C501B7FE02C080E090E0A7014770552715
:10E320004115510551F0080F191F60E070E08C0F86
:10E330009D1F0E941771F8018083DF91CF911F917B
:10E340000F91FF90EF90DF90CF90BF90AF909F9094
:10E350008F907F906F9008958F929F92AF92BF920F
:10E36000CF92DF92EF92FF920F931F93CF93DF93A1
:10E3700000D0CDB7DEB70E94835C8C0182E090E0D4
:10E380000E94615C892B19F480E090E05DC0F80187
:10E39000818190E0982F88272081820F911D0E9413
:10E3A00051547C01009781F30E94835C4C01F7017A
:10E3B0002681822F86958695869590E0422F47701C
:10E3C00021E030E011F420E030E0820F931F0E9442
:10E3D000615C892BC9F2F70104811581C12CD12C14
:10E3E000F8018081882379F1F801A180B12CB60170
:10E3F00033E0759567953A95E1F7A6014770552783
:10E40000680D791D883168F09501CE0101960E9452
:10E410003671BE016F5F7F4FF80180810E94A95D58
:10E420000DC01A8219829501CE0101960E943671A3
:10E4300069817A81F80180810E94955DCA0CDB1C9C
:10E440000E5F1F4FCDCFC7010F900F90DF91CF917F
:10E450001F910F91FF90EF90DF90CF90BF90AF9002
:10E460009F908F900895DC0150E0E0E1F0E0E61B22
:10E47000F70BE21BF30B02C0440F551FEA95E2F7BE
:10E480008C91852B8C9311968C911197842B1196DE
:10E490008C9308956F927F928F929F92AF92BF92CA
:10E4A000CF92DF92EF92FF920F931F93CF93DF9360
:10E4B0008C016B01EA017901283031051CF4488197
:10E4C000C8015CC0390153E0759467945A95E1F72F
:10E4D0006115710521F04E01A12CB12C03C0D801AA
:10E4E000FE0127C0F40141914F0128E030E0B60160
:10E4F000C8018A0D9B1D0E943372FFEFAF1ABF0A3D
:10E50000A614B7047CF3C30177FE02C080E090E05C
:10E510009701277033272115310509F43FC0C80F33
:10E52000D91F488150E0B601621B730B685F7F4FB3
:10E530001CC0CF018C1B9D0B861597051CF4819187
:10E540008D93F7CFC30177FE02C080E090E0970182
:10E55000277033272115310509F1C80FD91F4881CC
:10E5600050E068E070E0621B730B02C05595479560
:10E570006A95E2F760E070E0800F911FDF91CF9124
:10E580001F910F91FF90EF90DF90CF90BF90AF90D1
:10E590009F908F907F906F900C943372DF91CF910A
:10E5A0001F910F91FF90EF90DF90CF90BF90AF90B1
:10E5B0009F908F907F906F9008956F927F928F922F
:10E5C0009F92AF92BF92CF92DF92EF92FF920F9302
:10E5D0001F93CF93DF9300D0CDB7DEB78C01FC0142
:10E5E0008681E82EE694E694E694F12C282F277095
:10E5F00081E090E011F480E090E0E80EF91EC701A0
:10E6000002960E94E55C009709F445C00E948A5C6E
:10E61000F8012281FC012083F8012381FC01218380
:10E620000E948A5C02965C01A70160E070E00E9493
:10E630007593F80104811581E12CF12CF80180819A
:10E64000882339F1F8018180912C670163E0D5942A
:10E65000C7946A95E1F73701F7E06F227724CA0C77
:10E66000DB1C883128F00E94B35D9401AC0108C026
:10E670000E94A05D9A8389839401AE014F5F5F4F32
:10E68000B301C6010E944A72E80CF91C0E5F1F4FCD
:10E69000D5CF81E090E00F900F90DF91CF911F9147
:10E6A0000F91FF90EF90DF90CF90BF90AF909F9031
:10E6B0008F907F906F900895E0915303F0915403F1
:10E6C0000994E0912C03F0912D030994E0915703F4
:10E6D000F09158030994E0915903F0915A03099479
:10E6E00080E090E008950895E0912403F0912503DF
:10E6F000099480E090E008950F931F93CF93DF93E8
:10E70000CDB7DEB7E0970FB6F894DEBF0FBECDBF32
:10E710000E94D05C8C010E94835CAE014F5F5F4F12
:10E72000602F0E944C7B882309F446C088A9980179
:10E73000281B3109C9010E94615C892BE9F12E81F6
:10E7400021110CC0BE016A5E7F4F88E10E94A95D65
:10E75000E0914703F091480309952EC08A859B8577
:10E760008D3C3BEA930711F0019631F5223019F008
:10E7700088E090E002C082E090E001979C012F5F6A
:10E780003F4F12161306F4F6E1E0F0E0EC0FFD1F28
:10E79000E80FF91F23852F3F81F3BE01645F7F4F90
:10E7A00089E10E94A95D89E10E94B35D62E179E29D
:10E7B0000E949F53892B31F6E0960FB6F894DEBF86
:10E7C0000FBECDBFDF91CF911F910F910895AF92F2
:10E7D000BF92CF92DF92EF92FF920F931F93CF934E
:10E7E000DF93CDB7DEB7E0970FB6F894DEBF0FBE6C
:10E7F000CDBF8C016B01CE0101967C0180E3F70156
:10E8000011928A95E9F781E089838CE00E94A05DEE
:10E810008C831D821F8280917C1491E0980F9093CD
:10E820007C14898783E0B82EB8868DEC9BEA9B87A1
:10E830008A8789E10E94B35D60E073E00E949F5384
:10E84000892B31F082E08E838FEF8C878D8709C012
:10E8500089E10E94B35DBC01CE010C960E949653E3
:10E86000BE828DEC9BEA9D8B8C8B62E179E2CE01BE
:10E8700046960E9496530E94835C9FA78EA70E9493
:10E88000D05C88ABC7010E94457AB82E90E00E9408
:10E89000E55C892B31F10E948A5CBC014B2DC701DC
:10E8A0000E94637AE0901A03F0901B030E94DA5CE6
:10E8B0005C010E948A5CB501F701099501151105FB
:10E8C00081F0009739F0019761F441E050E064E095
:10E8D00070E004C041E050E060E070E0C601F80183
:10E8E0000995E0960FB6F894DEBF0FBECDBFDF915D
:10E8F000CF911F910F91FF90EF90DF90CF90BF903D
:10E90000AF9008950E94C57580937C14E091240314
:10E91000F09125030994892B29F0E0912403F091CB
:10E92000250304C0E0912603F09127030994CF93B7
:10E93000DF93EC0189919991009729F060E070E0F4
:10E940000E94EA55F7CFDF91CF910895CF93DF93DF
:10E95000EC0189919991009719F00E943C55F9CFEB
:10E96000DF91CF910895CF93DF93EC017B836A838E
:10E970000E945E6699838883DF91CF910895FC01A0
:10E980008081918122813381820F931F91838083C3
:10E990000895CF93DF93EC010E945E66998388838C
:10E9A000DF91CF910895CF93DF93EC010E945E66D3
:10E9B00028813981821B930B9C012F5F3F4F81E09F
:10E9C00090E04A815B814217530710F080E090E0AD
:10E9D000DF91CF910895CF93DF93FC01C281D38162
:10E9E00080819181C80FD91F0E945E669E01281BFD
:10E9F000390BC901DF91CF910895CF93DF93EBE8F5
:10EA0000FBE2CDE4DBE2AFE7BBE211921192199297
:10EA10001992199219921D928BE2E33AF807A9F71D
:10EA2000DF91CF910895CF93DF93FC01E158F44D2E
:10EA300040819C01220F331F220F331F442301F119
:10EA4000A0919400B0919500FC01EE0FFF1FE557D7
:10EA5000F44D80819181AD01481B590BCA01E90138
:10EA6000C35BD44D488159816A817B81480F591F0E
:10EA7000611D711D488359836A837B83B183A083A1
:10EA8000F901E35BF44D6081718182819381DF91B3
:10EA9000CF91089560E070E0CB010895FC01EE0F86
:10EAA000FF1FEE0FFF1FE35BF44D40835183628332
:10EAB00073830895CF93DF932FE73BE2CDE4DBE24E
:10EAC000EBE8FBE2D9018D919D018823B9F04091DB
:10EAD00094005091950080819181BA01681B790B57
:10EAE00088819981AA81BB81860F971FA11DB11DC5
:10EAF00088839983AA83BB8351834083249632966B
:10EB0000BBE22B383B07F1F6DF91CF9108950C94CF
:10EB1000D4790F931F93FC01CB0140917D14509148
:10EB20007E14338322831583048371836083F0937F
:10EB30007E14E0937D14452B11F40E94EE7980E061
:10EB400090E01F910F91089580917D1490917E1413
:10EB50000097C1F010927E1410927D14DC0114967F
:10EB60006D917C9115971296ED91FC9113970995F3
:10EB7000E0917D14F0917E14309721F08081918195
:10EB80000C94EE7908950C94FF8F0C94FB8F84ED18
:10EB900092E00E9421568CEC92E00C942156CF9387
:10EBA000DF930E94905C892BA9F08CEC92E00E948C
:10EBB0003F56EC01009721F10E94D05C9983888335
:10EBC0000E94CB5C9B838A83CE0104960E940C5CDE
:10EBD0008CAB14C084ED92E00E943F56EC0100978C
:10EBE00079F002960E941E5C99838883BE016E5460
:10EBF0007F4FCE018E579F4F0E94735DCE0102C0A2
:10EC000080E090E0DF91CF910895BC016E547F4F7A
:10EC10008E579F4F0C94735DCF93DF93EC01BC0133
:10EC200084ED92E00E948956BE01892B19F084ED93
:10EC300092E009C08CEC92E00E948956892B39F051
:10EC4000BE018CEC92E0DF91CF910C946456DF9181
:10EC5000CF9108950F931F93CF93DF93EC01BC01E5
:10EC600084ED92E00E948956892B91F0FE0161911A
:10EC70007191CF010E942F5DBE016E547F4FCE0176
:10EC80008E579F4FDF91CF911F910F910C94845D10
:10EC9000BE018CEC92E00E948956892BD1F00E9433
:10ECA0001C5D688179818A819B810E942F5D8CA97E
:10ECB00090E00E94E55C0CA910E00E948A5CBE0115
:10ECC0006C5F7F4FA801DF91CF911F910F910C9442
:10ECD0006C93DF91CF911F910F910895CF93DF93A4
:10ECE000EC01BC0184ED92E00E948956892B19F059
:10ECF000CE0102960CC0BE018CEC92E00E948956B7
:10ED0000892B19F08A819B8102C080E090E0DF911D
:10ED1000CF910895FC01808191810895860F911D06
:10ED2000860F911D8E579F4F0895860F911D860F58
:10ED3000911D8E579F4FFC01808191810895089508
:10ED40008CED9AE10E946358892B21F08CED9AE1B9
:10ED50000C9450580895E091C81AF091C91A309750
:10ED600009F0099480E00895EF92FF920F931F93AA
:10ED7000CF93DF937C01EA01FC01808191810097B0
:10ED800041F08C30934071F1F7011182108283E0E1
:10ED9000F2C080E024E0829FF0011124E653F54E9A
:10EDA000118210828F5F8430A8F38093C71A8091FC
:10EDB0000212909103129093DB1A8093DA1A0E9448
:10EDC00035558093A32B60E470E08CED9AE10E94AE
:10EDD0003C580E94C17C8CE093E0F70191838083D2
:10EDE00081E0C9C06230D9F48091A42B9091A52B09
:10EDF000892B89F38091B52B863029F48091CD2B16
:10EE000081FD0E94A07681E00E94FE7D8091A42B6E
:10EE10009091A52B892BF9F20E94C478DCCF633046
:10EE200060F5611114C02097B1F2D093B230C09355
:10EE3000B13083E00E94FE7D8091A42B9091A52BA0
:10EE4000892B11F00E94AB760E94A076C4CF61306E
:10EE500011F6209709F4BFCFD093AE30C093AD30F8
:10EE600085E00E94FE7D8091A42B9091A52B892B9B
:10EE700009F4B1CF0E94AB76AECF6738E9F51092B6
:10EE8000C61A0AEC1AE18091C61A8430B8F4F80167
:10EE9000828193818C179D0749F4808191810E9422
:10EEA000CB7DF80111821082138212820C5F1F4FFA
:10EEB0008091C61A8F5F8093C61AE5CFECECF0E321
:10EEC000838194818C179D0719F414821382108218
:10EED000B09621E3EC34F20799F7E9E4F1E3818598
:10EEE00092858C179D0711F4158214823D9681E35B
:10EEF000EB3CF807A1F76FCF683809F06CCFCC5D19
:10EF0000DA4109F068CF8CED9AE10E946358892BB1
:10EF100009F461CF1092C61AE091C61AE43008F0E5
:10EF20005ACF20E2E29FF0011124ED54FF4C818D75
:10EF30008823D9F08CED9AE10E9450588091C61A2E
:10EF4000E0E28E9FC00111248D549F4C9093B2300B
:10EF50008093B13082E00E94FE7D8091A42B90913D
:10EF6000A52B892B11F00E94AB768091C61A8F5F7A
:10EF70008093C61AD1CFDF91CF911F910F91FF904F
:10EF8000EF9008959093C91A8093C81A089520911C
:10EF900002123091031260E0EAECFAE1643098F476
:10EFA000408151814817590759F4428153814217D2
:10EFB000530731F46093C51A118210820C94CB7DF3
:10EFC00034966F5FEBCF6093C51A089540E0EAEC8A
:10EFD000FAE14430A8F451E0540F20813181232B11
:10EFE00061F44093C41A918380832091021230917E
:10EFF0000312338322830C94E57D3496452FE9CFA9
:10F000004093C41A08952091021230910312FC011A
:10F01000358F248F778F668F08952091021230915B
:10F020000312FC0132872187748763870895CF9389
:10F03000DF93EA010E946E7D009749F02091021251
:10F0400030910312FC0132872187D487C387DF9177
:10F05000CF9108950F931F93CF93DF9300D000D0EB
:10F06000CDB7DEB78C01AB018FEF89838A838B83A9
:10F070008C83B801CE0101960E941778009719F091
:10F08000FC01158304830F900F900F900F90DF9178
:10F09000CF911F910F91089540E050E062E08CED18
:10F0A00092E00E94DB551092A52B1092A42B08959C
:10F0B000AC0161E08CED92E00C94BD55AC0160E0D8
:10F0C0008CED92E00C94BD550F931F93CF93DF937B
:10F0D0008A010E94ED7CEC01009759F080910212A8
:10F0E000909103129D8F8C8F1F8F0E8FCE010E94E7
:10F0F0005E78CE01DF91CF911F910F910895CF934C
:10F10000DF93A091B130B091B230109719F0ED01BA
:10F110006C9605C0C091AD30D091AE3029968091EB
:10F12000AC3086FF22C01092C31A40E0EAECFAE14C
:10F130004430B8F42081318114968D919C911597BB
:10F140002817390759F482819381009739F0409349
:10F15000C31A998388831B821A8205C034964F5F35
:10F16000E7CF4093C31A0E94A076888199810097C7
:10F1700041F04A815B816091A32BDF91CF910C9488
:10F18000DB55DF91CF9108950F931F93CF93DF93BA
:10F190008091B52B863009F071C08091A42B90919D
:10F1A000A52B8115954009F069C0C4E9D2E0D09340
:10F1B000A52BC093A42B02E00093AE2B14E910936F
:10F1C000AF2B1092D12B1092D02B0E94BB7C80953C
:10F1D00090959093D12B8093D02B1092B72B1092B7
:10F1E000B62B0E94AA7C809590959093B72B809324
:10F1F000B62B0E94AB76D093A52BC093A42B009383
:10F20000AE2B1093AF2BA091AF30B091B030FD0179
:10F21000E459FD4F8CE692E001900D920197E1F7E1
:10F220006CE672E084EC9BE20E94697C8091A82BE2
:10F230008093C42B8091A92B8093C52B8091AA2BFE
:10F240008093C62B8091AB2B8093C72B1092D12B30
:10F250001092D02B0E94BB7C809590959093D12BDF
:10F260008093D02B1092B72B1092B62B0E94AA7CC1
:10F27000809590959093B72B8093B62BDF91CF918B
:10F280001F910F910C94AB76FC01680F791F80E001
:10F2900048E1E617F70781F0219198E0322F3827EF
:10F2A000532F517030FD84278695513009F48068C2
:10F2B0002695915099F7EDCF08951F920F920FB6B2
:10F2C0000F9211240BB60F922F933F934F935F939E
:10F2D0006F937F938F939F93AF93BF93EF93FF931E
:10F2E00080919400909195009093902B80938F2B18
:10F2F00081E08093812B80917100807D80937100EB
:10F300000E94A4758091812B8823D9F1809194006B
:10F310009091950040918F2B5091902B84179507D9
:10F32000A0F48091552B9091562BA091572BB09122
:10F33000582B8C57914EAF4FBF4F8093552B9093C6
:10F34000562BA093572BB093582B209194003091BB
:10F350009500241B350B8091552B9091562BA09135
:10F36000572BB091582B820F931FA11DB11D809375
:10F37000552B9093562BA093572BB093582B10924C
:10F38000812BFF91EF91BF91AF919F918F917F91D1
:10F390006F915F914F913F912F910F900BBE0F9006
:10F3A0000FBE0F901F9018959FB7F894E1E7F0E01B
:10F3B0008081807D808388B38F6288BB10929000AB
:10F3C000E1E9F0E010821092920010929500109204
:10F3D00094008081856080839FBF08952FB7F89443
:10F3E000909399008093980088B38F6288BBE1E77F
:10F3F000F0E08081826080832FBF0895CF93DF93F8
:10F40000FC01DB0185E0EB0119928A95E9F7858122
:10F41000837011F082E08C938781837021F082E009
:10F4200012968C9312978581837081F08781837007
:10F4300069F023893489818592852817390731F449
:10F4400081E0848312961C92129701C014828581F8
:10F450008370823021F0833021F080E003C082E0AD
:10F4600001C088E011968C93119787818370823058
:10F4700021F0833021F080E003C082E001C088E009
:10F4800013968C93DF91CF910895CF93DF9300D0A3
:10F4900000D01F92CDB7DEB7BE016F5F7F4F0E94D5
:10F4A000FE7989819A81890F8D5F9B81890F9C816B
:10F4B000890F9D81890F0F900F900F900F900F90E3
:10F4C000DF91CF9108954F925F926F927F928F92CA
:10F4D0009F92AF92BF92CF92DF92EF92FF920F93E3
:10F4E0001F93CF93DF9300D000D000D0CDB7DEB70D
:10F4F0008C017B01BE016F5F7F4F4E830E94FE79BE
:10F50000B981AA815B804C808B2F90E003962A2FD3
:10F5100030E0820F931F850D911D642D70E0860FE2
:10F52000971F5D81850F911D4E8150E04817590747
:10F530000CF49AC0F801818180FB662460F8712C7C
:10F5400043E0660C771C4A95E1F7828180FB8824B2
:10F5500080F8912C54E0880C991C5A95E1F7862884
:10F5600080818770882A838180FBAA24A0F8B12C2F
:10F5700085E0AA0CBB1C8A95E1F78A28848180FB70
:10F58000CC24C0F8D12C96E0CC0CDD1C9A95E1F788
:10F590008C28F7018082F80145814370F4E04F9F89
:10F5A000A0011124F80186818370F0E18F9FC001D2
:10F5B0001124482BF8018781F0E48F9FC0011124AA
:10F5C000482BF7014183F8018085F7018283B2302F
:10F5D00059F4F8018185F7018383F8018285F701E9
:10F5E000848395E0C92E02C083E0C82EB0E080E09D
:10F5F00090E0200F311FDB2EDC0C0197BA1761F071
:10F60000A901480F591FFA01B384A7014D0D511DDF
:10F61000FA01B082BF5FEFCF9D2DF2E05F120EC006
:10F62000D701AD0DB11DF80183898C9381E08D0D5B
:10F63000D701A80FB11D9E5F84898C9340E020E024
:10F6400030E0060F171F842F890F21503109441510
:10F6500061F0D801A20FB31F55965C91D701A80F96
:10F66000B11D5C934F5FEFCF80E026960FB6F89404
:10F67000DEBF0FBECDBFDF91CF911F910F91FF90E5
:10F68000EF90DF90CF90BF90AF909F908F907F9042
:10F690006F905F904F900895BF92CF92DF92EF925C
:10F6A000FF920F931F93CF93DF937C01D62EEA0135
:10F6B00082E0861708F0B1C0F701808186FBBB2489
:10F6C000B0F89181292F269526952370C92EC294D2
:10F6D000C694C69453E0C522382F3770388383FB15
:10F6E000332730F9398384FB332730F93A8385FB9C
:10F6F000882780F98B83BC822D83892F8295837024
:10F700008E83CF8282818887222389F1338184810D
:10F7100090E0982F8827830F911D9A87898787010A
:10F720000B5F1F4F223071F460E073E0CE010B9647
:10F730000E949653F70186818B8785818C870E5FA7
:10F740001F4F20C02330F1F4F7013D9680E090E098
:10F750003E2F2F2F4291DE01A80FB91F1B964C930D
:10F76000019688309105B1F7032F122F0BC0870146
:10F770000D5F1F4F60E073E0CE010B960E94965321
:10F780001A861986CC20B9F1B1100DC0F80120817C
:10F79000818190E0982F8827820F911D9C8B8B8B05
:10F7A0000E5F1F4F04C089859A859C8B8B8BF2E07E
:10F7B000CF120EC060E073E0CE0145960E949653D2
:10F7C000F80181818D8B80818E8B0E5F1F4F1BC056
:10F7D000F3E0CF1218C0085F1F4FF80180E090E0FF
:10F7E0002291DE01A80FB91F55962C9301968830FF
:10F7F0009105B1F708C060E073E0CE0145960E9424
:10F8000096531C8A1B8AC8018E199F092D2D281B0F
:10F810002FA71EA70DA7D81608F480E0DF91CF917F
:10F820001F910F91FF90EF90DF90CF90BF900895C0
:10F83000FB0141505109460F571FE417F50778F4B3
:10F84000208130E0322F22276181260F311D820F67
:10F85000931F8217930708F401963296EECFE417B0
:10F86000F50751F4208130E0322F2227820F931FB9
:10F870008217930708F401960895CF93DF93C09100
:10F88000AF2BD0E064972091AE2B30E0322F2227AF
:10F89000C20FD31F48E050E068EB7BE29E01280FC7
:10F8A000311DC9010E94187CAE0160EC7BE20E9410
:10F8B000187C009721F098278927982702C08FEF9E
:10F8C0009FEFDF91CF9108959093F51A8093F41AEA
:10F8D0000895FC015381560F5093AB2B872F992726
:10F8E0004281480F4093AA2BA181A093A92BE081CC
:10F8F000E093A82B242F30E02817390748F481E043
:10F900008A0F8093A92B811103C0EF5FE093A82B8E
:10F91000852F90E077278617970788F44F5F4093ED
:10F92000AA2B41110CC08091A92B8F5F8093A92B2A
:10F93000811105C08091A82B8F5F8093A82B08951B
:10F94000AB01BC0180E090E00E94187C98278927D9
:10F950009827089544E150E06CEA7BE280E090E073
:10F960000E94187C009721F09827892798270895EE
:10F970008FEF9FEF089586E00C943D7C81E10C941D
:10F980003D7C80E0E82FF0E0EE0FFF1FED5CFE4CC9
:10F99000118210828F5F8430A8F380E090E2899F0B
:10F9A000F0011124ED54FF4C118E8F5F8430B0F3C1
:10F9B00080E094E09093EF1A8093EE1A80E09DE04F
:10F9C000989FF0011124E75BFE4C158214828F5F33
:10F9D0008A30B0F38093ED1A0895CF932091EE1AF8
:10F9E0003091EF1A2F5F3F4F21154DE7340710F08C
:10F9F00020E030E1522F432FE3EBF0E3C0E0C430CE
:10FA000059F0A18DAA2329F0A481B581A417B507C7
:10FA100049F3CF5FB096F3CF3093EF1A2093EE1AED
:10FA20001092ED1A20E0E0E0F0E02430E8F430E25B
:10FA3000239FD0011124AD54BF4C59963C91599746
:10FA4000311104C02093ED1AFD0110C0373041F48C
:10FA5000309739F05A964C915A97328D341708F0F6
:10FA6000DF012F5FFD01E1CF2093ED1A309799F16F
:10FA700022E0218F2091F01A24872091F11A258706
:10FA80002091F21A26872091F31A278728ED34E077
:10FA9000338B228B358B248B21E030E0318B208B14
:10FAA000138E228F23E0208F168A20E1278B20914E
:10FAB000EE1A3091EF1A3227232732273583248319
:10FAC00077836683DC014D915D916D917C914083DC
:10FAD000518362837383CF01CF910895CF93DF93D6
:10FAE0002091EE1A3091EF1A2F5F3F4F21154DE70D
:10FAF000340710F020E030E1522F432FEDE4F1E322
:10FB0000C0E0CA3041F0A081B181CF5F3D96A4171B
:10FB1000B507B9F7E9CF3093EF1A2093EE1A40E01A
:10FB20005DE04A30A0F4A1E0A40F549FF00111243D
:10FB3000E75BFE4C24813581232B39F44093ED1A89
:10FB4000309741F480E090E023C04A2FEACF409301
:10FB5000ED1AF8CF2091EE1A3091EF1A32272327B1
:10FB600032273583248377836683009729F41082B4
:10FB700011821282138209C0EC0188819981AA81C5
:10FB8000BB8180839183A283B38380E48087CF018C
:10FB9000DF91CF91089540E04430A0F4E42FF0E0ED
:10FBA00051E0540FEE0FFF1FED5CFE4C20813181C0
:10FBB0002817390729F44093ED1A1182108208950D
:10FBC000452FEACF4093ED1A089540E0443098F471
:10FBD000E42FF0E051E0540FEE0FFF1FED5CFE4C00
:10FBE00020813181232B29F44093ED1A9183808366
:10FBF0000895452FEBCF4093ED1A0895AF92BF9231
:10FC0000CF92DF92EF92FF920F931F93CF93DF93E8
:10FC1000C091B130D091B230843009F4DCC124ED10
:10FC20003BE23093B0302093AF303093A72B20933A
:10FC3000A62B833059F4898D8F70833009F06BC007
:10FC400088899989892B09F0DFC67FC0823009F045
:10FC500080C08091F31A8F5F8093F31A811113C0D3
:10FC60008091F21A8F5F8093F21A81110CC08091FB
:10FC7000F11A8F5F8093F11A811105C08091F01AFB
:10FC80008F5F8093F01A1092A52B1092A42B1092E4
:10FC9000483110924731298D822F8D7F853041F474
:10FCA0008A8D8F5F8A8F843109F0AEC6198EACC6FB
:10FCB000222309F4A9C688899989892B09F441C0AE
:10FCC0008A8D9FEF980F9A8F81119EC68B8D8830F9
:10FCD00031F09FEF920F923048F4853039F4198E4D
:10FCE00080E88093AC300E947F7847C5853038F437
:10FCF00093E0082E01C0990F0A94EAF701C090E33F
:10FD00009A8F8F5F8B8F822F8F708330A1F048F492
:10FD1000813009F44FC3823009F076C61092CD2BA2
:10FD20004CC3863009F4C8C4883009F4C5C4843093
:10FD300009F06AC6C1C484E08093AC300E947F7829
:10FD40004EC52F70233009F05FC688E08093AC3039
:10FD500009C5853019F5E091AD30F091AE30848160
:10FD60009581892B09F450C61092B2301092B130AF
:10FD700088EC9BE29093B0308093AF309093A72BA8
:10FD80008093A62B10924831109247311092A52BE8
:10FD90001092A42B88E08093AC301BC18091AC2BD7
:10FDA000853409F031C60091AE2B10E0102F0027EA
:10FDB0008091AF2B080F111D8091A42B9091A52B42
:10FDC0008017910708F420C61093A52B0093A42B4D
:10FDD0008091B22B8F7309F017C68091B32B8111DC
:10FDE00013C68091433190914431C0915D03D0910D
:10FDF0005E038C179D0759F440914531509146316F
:10FE000020915F033091600342175307A1F02091C6
:10FE1000BC2B3091BD2B2817390709F0F5C520916F
:10FE2000BE2B3091BF2B80914531909146312817E0
:10FE3000390709F0E9C50E94AA7C019609F0E4C5DA
:10FE40008091B52B863009F429C18131E9F18130E7
:10FE500009F0DAC58091C02B883009F0D5C5109221
:10FE6000C02B8091C22B9091C32B873F3FEF93070C
:10FE700010F0099601C008969093C32B8093C22B73
:10FE80008091B82B9091B92BA091BA2BB091BB2B3C
:10FE90008093BC2B9093BD2BA093BE2BB093BF2B14
:10FEA0008091433190914431A0914531B0914631D8
:10FEB0008093B82B9093B92BA093BA2BB093BB2B04
:10FEC00080E48093B42B7DC50C5111091093A52BB0
:10FED0000093A42B88EC9BE29093B0308093AF30DA
:10FEE0008091C62B9091C72B892B29F00E94BE7C54
:10FEF000019609F089C52091C22B3091C32B2115A1
:10FF0000310509F481C589E491E39093AE30809383
:10FF1000AD30A090C02BB090C12B40915F035091A9
:10FF200060036091610370916203A0916303B091DB
:10FF300064030091B82B1091B92BE090BA2BF0908C
:10FF4000BB2BE091AD30F091AE3081E3EB3CF80794
:10FF500008F05AC584819581009721F12817390747
:10FF600009F586819781009719F0A816B906D1F492
:10FF7000808191818C179D0729F4C280D380C4169B
:10FF8000D506B1F08617970729F4C280D380CA1628
:10FF9000DB0671F00817190729F482819381E816AE
:10FFA000F90631F03D96F093AE30E093AD30C9CF15
:10FFB0001092B2301092B13082E08093AC3088EC75
:10FFC0009BE29093A72B8093A62B1092483110921E
:10FFD00047310E947F788091473190914831009756
:10FFE00009F412C59C01245E3F4F3093A52B20934A
:10FFF000A42B3093AE2B2093AF2BE091AD30F0913A
:020000021000EC
:10000000AE3020852093B42B21E12093B52B0896A8
:100010009827892798279093C52B8093C42B1092FB
:10002000C72B1092C62B848195819093C12B80930E
:10003000C02B868197819093C32B8093C22B809194
:10004000433190914431A0914531B0914631809334
:10005000B82B9093B92BA093BA2BB093BB2B808174
:100060009181A281B3818093BC2B9093BD2BA093EF
:10007000BE2BB093BF2B84ED9BE29093B030809366
:10008000AF300E94BE7C80959095009711F48FEF61
:100090009FEF9093C72B8093C62B93C40E94BB7C89
:1000A000019609F0B1C48091C22B9091C32B0097A7
:1000B00009F4AAC42091C02B3091C12B2115310520
:1000C00009F4A2C44091B82B5091B92B6091BA2B7E
:1000D0007091BB2BECECF0E3C3EBD0E3F080FF209E
:1000E000A9F0AC81BD818A179B0781F4AE81BF81E5
:1000F0002A173B0759F4A881B9814A175B0731F4E5
:10010000AA81BB816A177B0709F46FC1A096B096DC
:10011000A1E3C333DA0711F72091CD2B2F732230DF
:10012000D9F49093EB1A8093EA1A40E0443090F4AB
:10013000E42FF0E0EE0FFF1FED5CFE4C20813181DB
:100140004F5F8217930791F71092ED1A20E0C0E0FD
:10015000D0E07EC04093ED1A8091CD2B82FD54C437
:1001600084E18093CD2B88E290E09093A52B80933F
:10017000A42B80E58093CC2B8091C72B9091CB2B27
:100180009093C72B3091C62B9091CA2B9093C62B7E
:100190003093CA2B2091C52B9091C92B9093C52BDE
:1001A0002093C92B9091C42B9093ED1A4091C82BAA
:1001B0004093C42B9093C82B8F5F8093CB2B8111DE
:1001C0000FC081E0830F8093CA2B811109C081E0A9
:1001D000820F8093C92B811103C09F5F9093C82B1E
:1001E0008091C02B9091C12B9093EB1A8093EA1AC7
:1001F0002091C22B3091C32B3093C12B2093C02B65
:100200009093C32B8093C22B8091B82B9091B92BE4
:10021000A091BA2BB091BB2B8093BC2B9093BD2B9C
:10022000A093BE2BB093BF2B80914331909144316A
:10023000A0914531B09146318093B82B9093B92B62
:10024000A093BA2BB093BB2BA1C3373089F02F5F9B
:100250002430C0F430E2239FC0011124FC01ED548E
:10026000FF4C318D3111F1CF2093ED1AEF010CC00D
:10027000209721F0428D3A8D341748F7EC01CD5488
:10028000DF4CE5CF2093ED1A209709F4BDC3D0933E
:10029000B230C093B13083E08A8F888F1E8A84E0A9
:1002A0008F8B1B8E8091C22B9091C32B9D838C834F
:1002B0008091C02B9091C12B9F838E838091B82B0E
:1002C0009091B92BA091BA2BB091BB2B88839983C5
:1002D000AA83BB8381E0898F8091F01A8C878091FB
:1002E000F11A8D878091F21A8E878091F31A8F8789
:1002F00081E090E0998B888B8091C72B8B878091D0
:10030000C62B8A878091C52B89878091C42B8887CB
:1003100081E090E00E9468858091CC2B282F207F7F
:1003200030E0213531050CF445C082958F7090E0A6
:100330000597880F991F880F991F3091EC1A20E0BC
:10034000E22FF0E0E817F9078CF5E455F44D30A5FD
:10035000311105C02093ED1A1092EC1A2BC03130E8
:1003600011F42F5FEDCF3230E1F441A54430C9F4F0
:100370002093ED1A3093EC1A82A590E0982F8827ED
:1003800023A5822B9093EB1A8093EA1A893DA4E06F
:100390009A0710F088ED94E09B8B8A8B9D8B8C8B59
:1003A00009C041A5442311F0240FCACF2093ED1AB0
:1003B0003093EC1A80E18093CD2B8091CD2B82601D
:1003C0008093CD2B82E08093D42B84E08093D52B37
:1003D0008093D62B88ED8093D72B8CE290E090937E
:1003E000A52B8093A42B80E67EC2D093B230C0931D
:1003F000B1301092AC309091CD2B92FF03C0198E8A
:1004000080E21AC28091CC2B82958F70880F880F62
:100410008093ED1A081B1109045111091093A52BA3
:100420000093A42B8F2D8F70823029F4892F8F7326
:10043000823139F41FC0813021F4892F8F738230CB
:10044000C9F0012B19F4892F8370A1F02091C42BDE
:10045000888528133EC22091C52B8985281339C26F
:100460002091C62B8A85281334C22091C72B8B85F7
:1004700028132FC294FF4AC06889798961157105D4
:1004800009F444C0CE010C960E94697C3091C82BBF
:100490008091A82B38133AC02091C92B8091A92BA9
:1004A000281334C09091CA2B8091AA2B98132EC088
:1004B0008091CB2B4091AB2B841328C03C872D8798
:1004C0009E878F878B8D81111AC02E89888D9A8D7A
:1004D000891B922F969596959695891B280F2E8BA2
:1004E00087FD81959F89392F36953695931B980FF7
:1004F0009F8B822F869586958695890F888F81E0C0
:100500008093AC30888D8A8F198A188A498D842F00
:100510008F7090E0FC013197E830F10508F074C26B
:10052000E057FF4F0C94AB8D8091AC3080FF14C02E
:1005300083E0898F80E48093AC30198A188A809197
:10054000A42B9091A52B009709F408C122E42093D5
:10055000AC300E94688502C18091CD2B8F738230B0
:1005600009F052C227CF8091AC3080FF70C08091DB
:10057000CD2B8F73823109F06AC08091CC2B282F4C
:10058000207F30E0213531050CF445C082958F7015
:1005900090E00597880F991F880F991F3091EC1AEA
:1005A00020E0E22FF0E0E817F9078CF5E455F44D70
:1005B00030A5311105C02093ED1A1092EC1A2BC012
:1005C000313011F42F5FEDCF3230E1F441A54430EA
:1005D000C9F42093ED1A3093EC1A82A590E0982F7D
:1005E000882723A5822B9093EB1A8093EA1A893DE2
:1005F00024E0920710F088ED94E09B8B8A8B9D8B12
:100600008C8B09C041A5442311F0240FCACF20933D
:10061000ED1A3093EC1A83E0898F8091C42B888780
:100620008091C52B89878091C62B8A878091C72BA3
:100630008B8781E090E00E94688582E48093AC30F3
:10064000198A188A1092A52B1092A42B87C080E2D9
:100650008093AC300E947F78E091B130F091B2305D
:10066000118E7ACD8091CD2B80FF28C044FD26C00D
:1006700088899989892B09F0C7C18091A42B909111
:10068000A52B01960E9468852091AC30822F806155
:100690008093AC308091A42B9091A52B892B19F0DD
:1006A00022612093AC300E947F7881E090E0998BAA
:1006B000888B88E0898F1B8E81E10CC185FF1CC06F
:1006C0008091D22B90E0982F88272091D32B822BDA
:1006D0002091AF303091B030280F391F3093B030B7
:1006E0002093AF302091A42B3091A52B281B390BE0
:1006F0003093A52B2093A42B8091A42B9091A52B14
:10070000009749F044FD07C02091AC30226020934F
:10071000AC300E9468858091CE2B90E0982F88277E
:100720002091CF2B820F911D9093EB1A8093EA1AA0
:100730002C893D892817390710F0892B21F4309333
:10074000EB1A2093EA1A8091EA1A9091EB1A9B8B8C
:100750008A8B8091AC30837009F456C11092483175
:10076000109247310E947F788091AC3085FF07C09E
:100770001092483110924731198E84E1ABC084FF4A
:100780000AC0109248311092473181E090E0998B75
:10079000888B84E08FCF20914731309148312115EB
:1007A0003105E1F080FF02C0198A188A8889998989
:1007B000009781F48A899B898217930720F490938C
:1007C0004831809347318091473190914831998BDE
:1007D000888B04C090934831809347311B8E809161
:1007E000A62B9091A72B9093B0308093AF3080913F
:1007F000473190914831892B59F088899989009720
:1008000039F088969093A52B8093A42B88E10BC098
:100810008091AC3081FFF8C088E290E09093A52BE6
:100820008093A42B80E18093CD2B5CC08091AC3071
:1008300080FFEAC0198E80E18093AC300E947F78FF
:10084000E3C08091A42B9091A52B009711F00E94FA
:1008500068859091CD2B8091AC3090FF0BC080FFCC
:1008600006C087E0898F1A8E198A188A19C086E017
:10087000898F16C080FF1EC085E0898F198A188A6B
:10088000C3C08091A42B9091A52B009711F00E94DA
:1008900068858091CD2B80FF0DC087E0898F1A8EEF
:1008A00081E090E00E94688580E18093AC300E94F6
:1008B0007F780FC08091A42B9091A52B892B49F4B0
:1008C000A3C08091AC3080FF9FC087E0898F1A8ED3
:1008D0009BC080E18093CD2B88E290E09093A52B84
:1008E0008093A42B80E58093CC2B88858093C82BA4
:1008F00089858093C92B8A858093CA2B8B858093A9
:10090000CB2B8C858093C42B8D858093C52B8E85B6
:100910008093C62B8F858093C72B86E08093B52B61
:100920008C819D819093C12B8093C02B8E819F8160
:100930009093C32B8093C22B80914331909144318B
:10094000A0914531B09146318093B82B9093B92B4B
:10095000A093BA2BB093BB2B88819981AA81BB81CC
:100960008093BC2B9093BD2BA093BE2BB093BF2B39
:10097000898D84FF05C01092CF2B1092CE2B06C01C
:1009800084E08093CE2B88ED8093CF2B80E48093FE
:10099000B42B8091A42B9091A52B9093AE2B809398
:1009A000AF2B1092D32B1092D22B1092D12B1092EE
:1009B000D02B0E94BB7C809590959093D12B8093F7
:1009C000D02B85E48093AC2B1092AD2B1092B32BDF
:1009D0001092B22B8091F41A9091F51A019690938F
:1009E000F51A8093F41A9093B02B8093B12B109248
:1009F000B72B1092B62B0E94AA7C8095909590936D
:100A0000B72B8093B62B04C01092A52B1092A42B69
:100A10001092AC30DF91CF911F910F91FF90EF902A
:100A2000DF90CF90BF90AF9008959827892798279F
:100A300008950E94B18D0895FC018091A62B90919C
:100A4000A72B2CEA30E3281B390BAB0126173707FD
:100A50000CF4A9011416150654F450934831409330
:100A60004731E817F90719F0BF010C946C9308950A
:100A700080E880936100109261000E94F2630E94FE
:100A800052550E94D0678091532990915429009724
:100A900029F001979093542980935329C0905529A8
:100AA000D0905629E0905729F09058290E948C66E2
:100AB000C616D706E806F90611F30E948C66609305
:100AC0005529709356298093572990935829D7CF49
:100AD0002091B1303091B230BC01C90108960E941A
:100AE000697CE091B130F091B2308091A82B808781
:100AF0008091A92B81878091AA2B82878091AB2B33
:100B0000838708952F923F924F925F926F927F92C8
:100B10008F929F92AF92BF92CF92DF92EF92FF920D
:100B20000F931F93CF93DF93CDB7DEB763970FB6C5
:100B3000F894DEBF0FBECDBF7C011B016A01FC0132
:100B400017821682838181FF66C3BE016F5F7F4F6C
:100B50004B01F7019381F10193FD859193FF819101
:100B60001F01882309F453C3853239F493FD85911D
:100B700093FF81911F01853239F4B70190E00E9403
:100B8000EF9356016501E5CF10E0512C20E02032B3
:100B9000A0F48B3269F030F4803259F0833269F47A
:100BA00020612CC08D3239F0803339F4216026C0A9
:100BB0002260246023C0286021C027FD27C030EDBB
:100BC000380F3A3078F426FF06C0FAE01F9F300D48
:100BD0001124132F13C06AE0569E300D1124532E9A
:100BE00020620CC08E3221F426FD11C3206406C0A1
:100BF0008C3611F4206802C0883641F4F10193FD6F
:100C0000859193FF81911F018111C1CF9BEB980FBB
:100C1000933018F42061805E06C09BE9980F9330F2
:100C200008F0AAC12F7E26FF16E02F73722E85369C
:100C300021F4F22FF0647F2E08C0863621F4622F53
:100C40006068762E02C01111115077FE07C01C3368
:100C500048F444244394410E27E00BC0183030F48C
:100C6000212F06C027E04CE3442E03C027E017E005
:100C7000412C560174E0A70EB11CF6016081718110
:100C800082819381042DA4010E9474926C010981D8
:100C900000FF02C003FF06C071FC07C072FC08C061
:100CA000612C08C03DE2632E05C02BE2622E02C01B
:100CB00090E2692E802F8C7099F1662011F084E00B
:100CC00001C083E0851510F0512C0BC0581A73FC3D
:100CD00008C0B70180E290E00E94EF935A94C9F7F0
:100CE000F3CF662029F0B701862D90E00E94EF93A4
:100CF00003FD03C00DE911E102C009E911E1F72D7F
:100D0000F0717F2EF8018491882309F476C2711066
:100D10008052B70190E00E94EF930F5F1F4FF2CF18
:100D200077FE0FC04C0C04FF04C08A81813309F4A4
:100D30004A94141474F5F8E0F41578F588E0482E18
:100D40002CC076FC2AC0812F90E08C159D059CF06C
:100D50006CEFC6166FEFD60674F0772D7068772E9D
:100D60000AC0E2E0F0E0EC0FFD1FE10FF11D808111
:100D7000803319F411501111F4CF77FE0EC04424C2
:100D80004394410E812F90E0C816D9062CF41C190B
:100D900004C04424439401C010E077FE07C01C1433
:100DA0001D043CF496012F5F3F4F05C025E030E065
:100DB00002C021E030E0662011F02F5F3F4F112389
:100DC00031F0412F50E04F5F5F4F240F351F452D0D
:100DD00050E02417350714F4521A01C0512C872D06
:100DE000897049F4552039F0B70180E290E00E9403
:100DF000EF935A94F7CF662029F0B701862D90E043
:100E00000E94EF9373FC09C0552039F0B70180E3CD
:100E100090E00E94EF935A94F7CF77FE5FC09C2D2D
:100E20008D2DD7FE02C090E080E0692E782E40E044
:100E300050E0C601841991099D878C879601261977
:100E40003709280D391D812F90E0EE27FF27E81B79
:100E5000F90BFF87EE87FFEF6F167F0669F4B70186
:100E60008EE290E02B8B3A8B488B598B0E94EF934C
:100E7000598948893A892B89C614D70454F06C855E
:100E80007D85661577052CF4F901E40FF51F818146
:100E900001C080E371E0671A71084F5F5F4FEE8514
:100EA000FF856E167F066CF0B70190E02B8B3A8BB6
:100EB000488B598B0E94EF932B893A89488959892D
:100EC000CACF6C147D0439F49A81963318F49533A3
:100ED00011F404FF81E3B70190E04BC08A818133B4
:100EE00009F00F7EB70190E00E94EF93111105C049
:100EF00074FE18C085E490E017C0B7018EE290E060
:100F00000E94EF9382E066246394680EF401E80F78
:100F1000F11D8081B70190E00E94EF93115041F3E1
:100F2000862DF1CF85E690E0B7010E94EF93D7FCC4
:100F300005C0C114D10439F404FF05C0D194C19493
:100F4000D1088DE201C08BE2B70190E00E94EF93DF
:100F500080E36AE0C616D1042CF08F5FFAE0CF1A66
:100F6000D108F7CFB70190E00E94EF93B701C60117
:100F7000C0960E94EF9341C1833631F0833779F0F8
:100F8000833509F058C021C0560172E0A70EB11C8C
:100F9000F6018081898301E010E0640114C05601EC
:100FA000F2E0AF0EB11CF601C080D18026FF03C075
:100FB000612F70E002C06FEF7FEFC6012B8B0E94A4
:100FC0009B938C012B892F7715C05601F2E0AF0E51
:100FD000B11CF601C080D18026FF03C0612F70E0F4
:100FE00002C06FEF7FEFC6012B8B0E945D938C01D7
:100FF0002B892068722E23FD1AC0852D90E00817DA
:101000001907A8F4B70180E290E00E94EF935A9488
:10101000F4CFF60177FC859177FE81916F01B701DE
:1010200090E00E94EF9351105A940150110901155C
:10103000110579F7E2C0843611F0893651F5560171
:1010400027FF09C0F4E0AF0EB11CF6016081718189
:10105000828193810AC0F2E0AF0EB11CF60160817B
:101060007181882777FD8095982F022F0F7697FF43
:1010700008C090958095709561957F4F8F4F9F4FD9
:1010800000682AE030E0A4010E942995C82EC81803
:101090003EC0022F853721F40F7E2AE030E01DC0CC
:1010A000097F8F3691F018F4883559F0B0C0803739
:1010B00019F0883711F0ABC0006104FF09C004606B
:1010C00007C024FF08C0066006C028E030E005C065
:1010D00020E130E002C020E132E0560107FF09C004
:1010E000F4E0AF0EB11CF6016081718182819381C1
:1010F00008C0F2E0AF0EB11CF6016081718180E0A2
:1011000090E0A4010E942995C82EC8180F7706FF09
:101110000BC0202F2E7FC11650F404FF0AC002FD21
:1011200008C0202F2E7E05C0DC2C202F03C0DC2C15
:1011300001C0D12E24FF0DC0FE01EC0DF11D8081F8
:10114000803311F4297E09C022FF06C0D394D394C2
:1011500004C0822F867809F0D39423FD13C020FFAA
:1011600006C01C2DD51418F4150D1D19D52CD51439
:1011700068F4B70180E290E02B8B0E94EF93D39448
:101180002B89F5CFD51410F45D1801C0512C24FF24
:1011900012C0B70180E390E02B8B0E94EF932B8964
:1011A00022FF17C021FF03C088E590E002C088E756
:1011B00090E0B7010CC0822F867859F021FD02C063
:1011C00080E201C08BE227FD8DE2B70190E00E9432
:1011D000EF93C11638F4B70180E390E00E94EF93DB
:1011E0001150F7CFCA94F401EC0DF11D8081B701C5
:1011F00090E00E94EF93C110F5CF552009F4C2CCC6
:10120000B70180E290E00E94EF935A94F6CFF70185
:101210008681978102C08FEF9FEF63960FB6F89497
:10122000DEBF0FBECDBFDF91CF911F910F91FF9019
:10123000EF90DF90CF90BF90AF909F908F907F9076
:101240006F905F904F903F902F9008955058BB271C
:10125000AA270ED04EC23FD230F044D220F031F453
:101260009F3F11F41EF4FFC10EF4E095E7FBF5C1BA
:10127000E92F50D280F3BA176207730784079507E6
:1012800018F071F49EF568C20EF4E0950B2EBA2F9B
:10129000A02D0B01B90190010C01CA01A00111247C
:1012A000FF27591B99F0593F50F4503E68F11A1628
:1012B000F040A22F232F342F4427585FF3CF4695B9
:1012C00037952795A795F0405395C9F77EF41F16DB
:1012D000BA0B620B730B840BBAF09150A1F0FF0FA5
:1012E000BB1F661F771F881FC2F70EC0BA0F621F91
:1012F000731F841F48F4879577956795B795F79581
:101300009E3F08F0B3CF9395880F08F09927EE0F12
:10131000979587950895DFD158F080E891E009F41A
:101320009EEFE0D128F040E851E059F45EEF09C0AB
:101330009AC112C2E92FE078EDD168F3092E052A8F
:10134000C1F3261737074807590738F00E2E07F85C
:10135000E02569F0E025E0640AC0EF6307F8009437
:1013600007FADB01B9019D01DC01CA01AD01EF9370
:1013700047D0BFD10AD05F91552331F02BED3FE02C
:1013800049E450FD49EC63CF0895DF93DD27B92F81
:10139000BF7740E85FE31616170648075B0710F4AF
:1013A000D92FE5D19F938F937F936F934AD3E0E337
:1013B000F1E06CD19ED12F913F914F915F919ED2E0
:1013C000DD2349F09058A2EA2AED3FE049EC5FE3C3
:1013D000D0785D274DDFDF918CC11BD108F481E00F
:1013E00008950CD086C17ED140F075D130F021F443
:1013F0005F3F19F032C15111B0C135C18BD198F3A3
:101400009923C9F35523B1F3951B550BBB27AA2785
:1014100062177307840738F09F5F5F4F220F331FF7
:10142000441FAA1FA9F333D00E2E3AF0E0E830D0C3
:1014300091505040E695001CCAF729D0FE2F27D0C6
:10144000660F771F881FBB1F261737074807AB0794
:10145000B0E809F0BB0B802DBF01FF2793585F4F09
:101460002AF09E3F510568F0F8C077C15F3FECF36A
:10147000983EDCF3869577956795B795F7959F5FCE
:10148000C9F7880F911D9695879597F90895E1E022
:10149000660F771F881FBB1F621773078407BA0781
:1014A00020F0621B730B840BBA0BEE1F88F7E095DC
:1014B000089519F40EF0D1C04FC1D5C033D1C8F38F
:1014C0009638C0F707F80F92E8942BE33AEA48EB16
:1014D0005FE716D20F920F920F924DB75EB70F9241
:1014E000CED1EDE5F1E0D2D04F915F91EF91FF9138
:1014F000E595EE1FFF1F49F0FE57E0684427EE0F09
:10150000441FFA95E1F74195550B3AD10F9007FE2C
:101510002EC1089597FB0EF4A9D03EC0E89409C0EF
:1015200097FB3EF490958095709561957F4F8F4F16
:101530009F4F9923A9F0F92F96E9BB279395F6952C
:10154000879577956795B795F111F8CFFAF4BB0FAA
:1015500011F460FF1BC06F5F7F4F8F4F9F4F16C00E
:10156000882311F096E911C0772321F09EE8872F98
:10157000762F05C0662371F096E8862F70E060E054
:101580002AF09A95660F771F881FDAF7880F9695CD
:10159000879597F90895E894F92F96EBFF2381F04A
:1015A000121613061406440B9395F69587957795B6
:1015B000679557954040FF23B9F71BC099270895B9
:1015C000882351F49850D2F7872B762F652F542F0C
:1015D000432F322F20E0B1F3121613061406440BEA
:1015E00088233AF09A95440F551F661F771F881F6E
:1015F000CAF755234AF4440F551F11F460FF04C085
:101600006F5F7F4F8F4F9F4F880F9695879597F904
:101610000895990F0008550FAA0BE0E8FEEF161683
:101620001706E807F907C0F012161306E407F507D6
:1016300098F0621B730B840B950B39F40A2661F04A
:10164000232B242B252B21F408950A2609F4A140ED
:10165000A6958FEF811D811D089597F99F6780E8FA
:1016600070E060E008959FEF80EC0895909580957C
:101670007095609550954095309521953F4F4F4F0F
:101680005F4F6F4F7F4F8F4F9F4F0895DF93CF93E3
:101690001F930F93FF92EF92DF927B018C0168946E
:1016A00005C0DA2EEF012AD1FE01E894A59125911B
:1016B000359145915591AEF3EF01DADDFE019701C9
:1016C000A801DA9479F7DF90EF90FF900F911F91C6
:1016D000CF91DF91089500240A9416161706180674
:1016E0000906089500240A94121613061406050626
:1016F0000895092E0394000C11F4882352F0BB0FB7
:1017000040F4BF2B11F460FF04C06F5F7F4F8F4F19
:101710009F4F089557FD9058440F551F59F05F3F54
:1017200071F04795880F97FB991F61F09F3F79F003
:1017300087950895121613061406551FF2CF469585
:10174000F1DF08C0161617061806991FF1CF869507
:101750007105610508940895E894BB2766277727EB
:10176000CB0197F9089555DF08F48FEF08959B0199
:10177000AC0160E070E080E89FE333CE6ECF64C1DF
:10178000D1DFE8F39923D9F3940F511DBBF39150A6
:10179000504094F059F0882332F0660F771F881F6D
:1017A00091505040C1F79E3F510544F7880F911D5D
:1017B0009695879597F908955F3FACF0983E9CF019
:1017C000BB27869577956795B79508F4B160939593
:1017D000C1F7BB0F58F711F460FFE8CF6F5F7F4F81
:1017E0008F4F9F4FE3CFB9CF0AD029ED3BE54EEDA8
:1017F0005EE378C00EF028C136CF68942ECF92DF1A
:10180000C8F39923D1F3C6F3DF93CF931F930F93BC
:10181000FF92C92FDD2788232AF02197660F771FB3
:10182000881FDAF720E030E040E85FEB9FE388397B
:1018300020F0803E30F021968F7709DDE5E8F1E079
:1018400003C005DDE2EBF1E021DF8B01BE01EC011D
:10185000FB2E6F5771097595771F880B990B60DE0A
:1018600028E132E741E35FE349D0AF2D9801AE01B3
:10187000FF900F911F91CF91DF91FADC3ACFFA01DF
:10188000DC01AA0FBB1F9B01AC01BF5728F4222724
:101890003327442750781FC0B75188F4AB2F00245A
:1018A000469537952795011CA395D2F3002069F042
:1018B000220F331F441FB395DAF30DD0C7CC61302C
:1018C0007105A0E88A07B94630F49B01AC01662790
:1018D000772788279078309621F0208331834283C0
:1018E000538308950BD005CFF6DE28F0FBDE18F009
:1018F000952309F0B2CEB7CE11242FCF0BDFA0F382
:10190000959FD1F3950F50E0551F629FF001729F94
:10191000BB27F00DB11D639FAA27F00DB11DAA1FB3
:10192000649F6627B00DA11D661F829F2227B00D00
:10193000A11D621F739FB00DA11D621F839FA00D8B
:10194000611D221F749F3327A00D611D231F849FDB
:10195000600D211D822F762F6A2F11249F57504032
:101960008AF0E1F088234AF0EE0FFF1FBB1F661FCD
:10197000771F881F91505040A9F79E3F510570F086
:101980006CCEEBCE5F3FECF3983EDCF3869577951B
:101990006795B795F795E7959F5FC1F7FE2B880F81
:1019A000911D9695879597F90895FA01EE0FFF1FFF
:1019B00030962105310599F16115710561F4803882
:1019C000BFE39B0749F168949038810561F0803846
:1019D000BFEF9B0741F0992342F5FF3FE105310539
:1019E000210511F1E8940894E795D901AA2329F477
:1019F000AB2FBE2FF85FD0F310C0FF5F70F4A69539
:101A0000E0F7F73950F019F0FF3A38F49F779F93D9
:101A10000CD00F9007FC905808953EF024CE60E063
:101A200070E080E89FE308954FE79F775F934F93BF
:101A30003F932F93E4DE2F913F914F915F9152DFBF
:101A40003DCD9B01AC014ECF9F3F31F0915020F432
:101A5000879577956795B795880F911D969587958A
:101A600097F90895DB018F939F930E94D68DBF91C4
:101A7000AF91A29F800D911DA39F900DB29F900DDD
:101A800011240895AA1BBB1B51E107C0AA1FBB1F4D
:101A9000A617B70710F0A61BB70B881F991F5A95FA
:101AA000A9F780959095BC01CD01089597FB072E6D
:101AB00016F4009407D077FD09D00E94428D07FCF0
:101AC00005D03EF4909581959F4F0895709561954E
:101AD0007F4F0895A1E21A2EAA1BBB1BFD010DC06A
:101AE000AA1FBB1FEE1FFF1FA217B307E407F507CE
:101AF00020F0A21BB30BE40BF50B661F771F881FAA
:101B0000991F1A9469F760957095809590959B013F
:101B1000AC01BD01CF010895052E97FB1EF4009482
:101B20000E94A38D57FD07D00E946A8D07FC03D049
:101B30004EF40C94A38D50954095309521953F4FD0
:101B40004F4F5F4F089590958095709561957F4FA9
:101B50008F4F9F4F0895EE0FFF1F0590F491E02DDA
:101B60000994692796276927782787277827089572
:101B70000E94C08D332312F48A1B9B0B0C94D18DD1
:101B8000A29FB001B39FC001A39F700D811D1124BE
:101B9000911DB29F700D811D1124911D08950E9409
:101BA000C08DB7FF0895821B930B08950E94C08DCE
:101BB000A59F900DB49F900DA49F800D911D1124A1
:101BC0000895B7FF0C94D68D0E94D68D821B930B7F
:101BD0000895DF93CF931F930F939A9DF02D219F2C
:101BE000F00D8B9DF00D8A9DE02DF10D039FF00D02
:101BF000029FE00DF11D4E9DE00DF11D5E9DF00D6B
:101C00004F9DF00D7F936F93BF92AF925F934F9371
